:100000000C948E080C94AD080C94AD080C94D10A95
:100010000C94070B0C94AD080C94AD080C94AD082F
:100020000C94AD080C94AD080C94AD080C94AD087C
:100030000C94AD080C94AD080C94AD080C94610EB2
:100040000C94AD080C94AD080C94AD080C94AD085C
:100050000C94A2590C94AE500C94AD080C94AD08BD
:100060000C94AD080C9484510C94AD080C94785108
:100070000C94AD080C94AD080C94AD080C94AD082C
:100080000C9465650C94AD080C94AD080C94AD0807
:100090000C94C2510C94AD080C94B6510C94AD085C
:1000A0000C94AD080C94AD080C94AD080C94AD08FC
:1000B0000C94AD080C94AD080C94AD080C94AD08EC
:1000C0000C94AD080C94AD080C94AD080C94AD08DC
:1000D0000C94AD080C94AD080C94AD080C94AD08CC
:1000E0000C94AD080C945B590C9465590C945159BF
:1000F0000C940B590C9496590C9487590C947B5979
:100100000C946F590C94AD080C94AD080C94AD0888
:100110000C94AD080C94AD080C94AD080C94AD088B
:10012000084AD73B3BCE016E84BCBFFDC12F3D6C5E
:1001300074319ABD56833DDA3D00C77F11BED9E4C4
:10014000BB4C3E916BAAAABE000000803F076342F1
:1001500036B79BD8A71A39685618AEBAAB558C1D5E
:100160003CB7CC5763BD6DEDFD753EF6177231BFE0
:10017000000000803F08000000BE922449123EAB00
:10018000AAAA2ABECDCCCC4C3E00000080BEABAAB1
:10019000AAAA3E00000000BF000000803F0000004F
:1001A0000000084178D3BB4387D1133D190E3CC3EF
:1001B000BD4282AD2B3E68EC8276BED98FE1A93E6E
:1001C0004C80EFFFBE01C4FF7F3F000000000050E5
:1001D0003A20256C642050612020252D372E326670
:1001E000206D0A002563002563004932433A200050
:1001F000256300256C642050612020252D372E3288
:1002000066206D00256C6420432000256300545F48
:1002100052483D252D342E3166200052483D252D73
:10022000342E31662000256300256300507772313B
:100230003D25730A0044656275673D3078252D7849
:100240000A00496E7075742050313D25730A0048CC
:10025000554D5F5057525F414C574159533D25739F
:100260000A0025730A006175746F0A004C6F6720DD
:100270006D6F64653D00496E74722E205365633A5C
:1002800020202050303D252D372E33662050313D23
:10029000252D372E33660A00496E74722E20546F56
:1002A00074616C3A2050303D252D6C642050313DF6
:1002B000252D6C640A005553425F5057523D2573FB
:1002C0000A00565F4D43553D252D352E32660A00F6
:1002D000565F494E3D252D352E32660A0052657017
:1002E0006F7274204D61736B3D3078252D6C7820D2
:1002F000005265706F727420496E74657276616C1D
:100300003D252D640A0052494D4520616464723DCB
:10031000252D642E252D640A004E65696768626F7D
:1003200072207461626C652073697A653D25640A88
:1003300000545820506F7765723D25640A00436869
:10034000616E3D25640A004932433A200049443D2C
:100350000053797374656D2053756D6D6172790A00
:100360000025630025630043757272656E74207208
:1003700065706F727420696E74657276616C3D256C
:100380002D64207365630A004E6577207265706F77
:10039000727420696E74657276616C3D252D6420DF
:1003A0007365630A002563005573696E6720726583
:1003B000706F72743D3078252D6C7820004E657713
:1003C000207265706F72743D3078252D6C78200036
:1003D000256300256300256300256300204F5343F8
:1003E00043414C3D2564200020467573653A2065E5
:1003F000653D253032782068663D25303278206CA6
:10040000663D25303278206C623D25303278004DD3
:1004100043553D2530366C7800256300252D31305D
:100420006C7520252D31306C7520252D31306C7583
:1004300020252D31306C75200A007478206C656E93
:1004400020202020207268206D69737320202020D6
:100450007268207374616C652020207268206D6959
:1004600073630A002563004F4B0A00256300256370
:1004700000256300256300445F434F4D50415353B3
:100480003D307825780A00445F414343454C3D3078
:100490007825780A00445F505245533D30782578DE
:1004A0000A00445F5057525F313D307825780A008A
:1004B000445F4145533D307825780A00445F503110
:1004C0005F4C45443D307825780A00445F50305FEA
:1004D0004C45443D307825780A00445F4556454EEA
:1004E000543D307825780A00445F504F5745523DBF
:1004F000307825780A00445F4C45443D30782578B3
:100500000A00445F4F573D307825780A00445F5019
:100510004B543D6E307825780A00445F54583D3086
:100520007825780A00445F52583D307825780A00D3
:10053000445F4F5045523D307825780A004375722C
:1005400072656E742064656275673D307825580A5F
:10055000004E65772064656275673D307825580ADE
:100560000025730A0025372E33662025372E336683
:100570000025352E326620004572726F72203020C1
:10058000566F6C74004E6F7420737570706F727458
:1005900065640A004572726F72203020566F6C7469
:1005A000004572726F72203020566F6C7400257394
:1005B0000A00545820506F7765723D25640A004345
:1005C00068616E3D25640A005465737420362025E9
:1005D000730A005465737420352025730A0054652E
:1005E000737420342025730A0054657374203320FB
:1005F00025730A005465737420322025730A005451
:1006000065737420312025730A0025730A00257351
:100610000A0025730A0025730A005854414C5F54A0
:1006200052494D3D25640025730A00525F50413DFB
:1006300009093078256C7800525F503D09093078FF
:10064000256C7800525F41333D09093078257800E8
:10065000525F41323D09093078257800525F4131BF
:100660003D09093078257800525F565F494E3D09B3
:10067000093078257800525F52483D0909307825C5
:100680007800525F555054494D453D0930782578E2
:1006900000525F50315F543D09093078257800528F
:1006A0005F50313D09093078257800525F50305F46
:1006B000543D09093078257800525F50303D0909D2
:1006C0003078257800525F565F4D43553D093078AC
:1006D000257800525F545F4D43553D0930782578A9
:1006E00000525F54313D09093078257800525F543B
:1006F0003D09093078257800525F4536343D0909B7
:100700003078257800525F49443D090930782578D2
:1007100000525F50412000525F502000525F413331
:100720002000525F41322000525F41312000525F71
:10073000565F494E2000525F52482000525F55508C
:1007400054494D452000525F50315F542000525FA4
:1007500050312000525F50305F542000525F5030C3
:100760002000525F565F4D43552000525F545F4D4D
:1007700043552000525F54312000525F54200052F4
:100780005F4536342000525F4944200025303278DE
:100790000025372E33662025372E33662025352E4B
:1007A00030660025352E32662000204E6576657253
:1007B0002D7573656420737461636B203E2025641E
:1007C0002062797465730A00557074696D6520251F
:1007D0006420646179732C20253032643A253032EC
:1007E000643A253032640A0074657374205B6F6666
:1007F000667C317C327C337C347C355D202020204B
:10080000202020202D2074657374206D6F64657323
:100810000A0D00776474205B6F6E7C6F66667C7473
:100820006573745D20202020202020202020202D92
:10083000207761746368646F670A0D007570677272
:1008400020202020202020202020202020202020A8
:1008500020202020202020202D207265626F6F74C0
:100860002076696120626F6F746C6F616465720AD3
:100870000D00626F6F742020202020202020202077
:1008800020202020202020202020202020202D205B
:100890007265626F6F740A0D0070777273205B640B
:1008A0006565707C666F7263655F69646C655D2009
:1008B00020202020202D206D637520736C656570CD
:1008C000206D6F64650A0D00726573742065657034
:1008D000726F6D202020202020202020202020202A
:1008E000202020202D20726573746F72652065654D
:1008F00070726F6D0A0D007031205B6F6E7C6F66D9
:10090000665D202020202020202020202020202064
:100910002020202D2064697361626C652070756CE5
:10092000736520703120746F207361766520706F5D
:100930007765720A0D0070777231205B6F6E7C6F85
:1009400066665D20202020202020202020202020DE
:1009500020202D2070696E31207077720A0D00748E
:10096000787077205B31352D305D202020202020CD
:1009700020202020202020202020202D20545820FE
:100980005077722E2048696768657374203020287C
:100990003364426D290A0D0073732020202020202B
:1009A0002020202020202020202020202020202047
:1009B000202020202D2073797374656D2073756D50
:1009C0006D6172790A0D0072732020202020202092
:1009D0002020202020202020202020202020202017
:1009E0002020202D20726164696F207374617473FC
:1009F0000A0D007269205B696E745D202020202042
:100A00002020202020202020202020202020202DD9
:100A1000207265706F727420696E74657276616C95
:100A20000A0D007265205B6D61736B5D20202020D4
:100A30002020202020202020202020202020202DA9
:100A4000206D6F7465207265706F727420736574A9
:100A500074696E670A0D006F772020202020202007
:100A60002020202020202020202020202020202086
:100A70002020202D206F6E652D77697265207365AB
:100A80006E736F72730A0D006C6F67205B61757413
:100A90006F7C6F6E7C6F66665D202020202020209A
:100AA000202020202D206D6F746573206461746197
:100AB000206F6E205553420A0D006E65205B666CF8
:100AC0007573685D202020202020202020202020F9
:100AD0002020202020202D206E65696768626F72BB
:100AE000207461626C650A0D0065727220202020FE
:100AF00020202020202020202020202020202020F6
:100B000020202020202D206572726F7220696E6671
:100B10006F0A0D006D6375202020202020202020EA
:100B200020202020202020202020202020202020C5
:100B30002D206D637520696E666F0A0D0069642053
:100B40005B72657365745D202020202020202020AA
:100B50002020202020202020202D20696420686172
:100B60006E646C696E670A0D0068756D70205B6F4E
:100B70006E7C6F66665D20202020202020202020B3
:100B800020202020202D2068756D696469747920EB
:100B90007065726D2073656E736F72207077720A64
:100BA0000D0068756D20202020202020202020208E
:100BB00020202020202020202020202020202D2028
:100BC00068756D69646974792073656E736F720AF4
:100BD0000D006465205B6D61736B5D20202020201B
:100BE00020202020202020202020202020202D20F8
:100BF00064656275670A0D006368616E205B313160
:100C00002D32365D20202020202020202020202072
:100C1000202020202D204368616E2031312D323676
:100C20002028322E3430352D32343830204D687A39
:100C3000290A0D0063616C69205B5B765F696E7CDD
:100C400061317C61325D20766F6C747C7265736596
:100C5000747C6E6F6E655D202D2063616C696272BD
:100C60006174650A0D00616463202020202020202B
:100C70002020202020202020202020202020202074
:100C800020202D2073686F7720765F696E2C20619D
:100C9000312C20613220766F6C74616765730A0DA8
:100CA00000616573205B6F6E7C6F66665D2020203F
:100CB000202020202020202020202020202D2069DE
:100CC0006E746567726574790A0D007520202020A6
:100CD0002020202020202020202020202020202014
:100CE000202020202020202D20757074696D650A39
:100CF0000D007620202020202020202020202020D1
:100D000020202020202020202020202020202D20D6
:100D100076657273696F6E0A0D00682020202020AE
:100D200020202020202020202020202020202020C3
:100D30002020202020202D2068656C700A0D0025C1
:100D40006300756E6B6E6F776E20636D640A004E84
:100D50004844433032313620004C3347343230304F
:100D6000442000484D433538383320004144584C26
:100D70003334352000424D50303835200048494842
:100D8000363133302000415432344D41432000206D
:100D90002573002025362E3266200025303278005B
:100DA000202573002025362E3266204F6E2D426F8F
:100DB0006172640025303278000A00452025642ED7
:100DC000256420636C6F636B20256C7520637075E0
:100DD00020256C75206C706D20256C7520697271F2
:100DE00020256C7520676C656420256C7520796CF6
:100DF000656420256C7520726C656420256C7520F7
:100E0000747820256C75206C697374656E20256C70
:100E1000752073656E736F727320256C7520736512
:100E20007269616C20256C750A00532025642E259B
:100E30006420636C6F636B20256C752074782025AB
:100E40006C7520727820256C752072747820256C62
:100E5000752072727820256C75207265786D6974C2
:100E600020256C752061636B747820256C75206E6D
:100E70006F61636B747820256C752061636B727889
:100E800020256C752074696D65646F757420256C00
:100E9000752062616461636B727820256C752074C3
:100EA0006F6F6C6F6E6720256C7520746F6F736841
:100EB0006F727420256C752062616473796E63684B
:100EC00020256C752062616463726320256C752037
:100ED000636F6E74656E74696F6E64726F702025D7
:100EE0006C752073656E64696E6764726F7020251F
:100EF0006C75206C6C747820256C75206C6C727825
:100F000020256C750A00257325730A004F6E6C69E5
:100F10006E650A000A002C20636865636B207261AD
:100F2000746520257520487A0025732025732C20B0
:100F30006368616E6E656C20257520706F776572D1
:100F4000202575000A0025783A004D414320616450
:100F50006472657373200052616E646F6D20455535
:100F600049363420616464726573732067656E6509
:100F700072617465640A000A2A2A2A2A2A2A2A42E5
:100F80006F6F74696E672025732A2A2A2A2A2A2AF3
:100F90000A00020000FFFE00000141544D45474198
:100FA00031323872666131006C6F63616C686F73E7
:100FB0007400454550524F4D20697320636F727223
:100FC0007570742C20726577726974696E6720770A
:100FD0006974682064656661756C74732E0A006EAE
:100FE000616E00696E660000407A10F35A00A072CC
:100FF0004E18090010A5D4E80000E8764817000054
:10100000E40B54020000CA9A3B000000E1F5050021
:101010000080969800000040420F000000A086016A
:10102000000000102700000000E80300000000643A
:1010300000000000000A00000000000100000000A5
:10104000002C76D888DC674F0823DFC1DFAE59E17A
:10105000B1B796E5E3E453C63AE651997696E8E6E9
:10106000C28426EB898C9B62ED407C6FFCEFBC9CBC
:101070009F40F2BAA56FA5F490055A2AF75C936BCE
:101080006CF9676DC11BFCE0E40D47FEF520E6B589
:1010900000D0ED902E0300943577050080841E0863
:1010A0000000204E0A000000C80C333333330F9881
:1010B0006E12831141EF8D2114893BE65516CFFE48
:1010C000E6DB18D1844B381BF77C1D901DA4BBE4D4
:1010D00024203284725E228100C9F124ECA1E53D16
:1010E00027494E46494E4954594E414ECDCCCC3DF0
:1010F0000AD7233C17B7D13877CC2B329595E62405
:101100001FB14F0A000020410000C84200401C46A9
:1011100020BCBE4CCA1B0E5AAEC59D7411241FBE06
:10112000CFEFD1E4DEBFCDBF16E0A0E0B2E0E0E05B
:10113000F2E001E00BBF02C007900D92A43EB107A0
:10114000D9F71DE2A4EEB6E001C01D92AE3AB10798
:10115000E1F70E94684F0C94FE800C94000029E097
:10116000FC0120935700C895802D0895E091D31776
:10117000F0E0EF71F070E85DF74E80838091D31757
:101180008F5F8093D3178091E82488608093E82450
:1011900045EF54E0CA0161E10E94B04080E090E078
:1011A00008954F925F926F927F928F929F92AF922B
:1011B000BF92CF92DF92EF92FF920F931F93DF9334
:1011C000CF93CDB7DEB760970FB6F894DEBF0FBEF2
:1011D000CDBF3B010E948D55E82FF0E0EE0FFF1FC1
:1011E000E356F84E808191810196918380838091AE
:1011F000E4069091E50681FD74980E9478474C01C1
:1012000089E097E00E94A7410AC0C8010296B30195
:101210000E947D3E009701F5C8010E946D42082F93
:10122000192F0115110589F721C1C8010296B301D3
:101230000E94743ED4018C918150F801808780E037
:1012400091E0A0E0B0E081879287A387B48789E02E
:1012500097E0B8010E942E42C8010D9660E074E646
:1012600048E55AE098010E946C4484E00E94AC4832
:10127000D80115969C938E93149783E00E94AC48F6
:101280002C01F80197838683D401AC908085A81A3D
:10129000BB24CC24DD2486E0AA0CBB1CCC1CDD1CAA
:1012A0008A95D1F7618572858385948520EC30E03D
:1012B00040E050E00E941F7A672F782F892F9927EE
:1012C000A60EB71EC81ED91EF801A186B286C38617
:1012D000D486D4018C9180878091E4069091E506B4
:1012E00081FD08C08091CE0480FD04C081FFB6C09E
:1012F0001D9BB4C0EDB7FEB772970FB6F894FEBF52
:101300000FBEEDBFEDB6FEB60894E11CF11C80E007
:1013100092E092838183C4010196D70113969C9336
:101320008E931297F301808114968C9314971596DF
:101330001C921597818116968C93169717961C927E
:10134000D4018C91F70180871186D80114968D9174
:101350009C9115979387828755864486BB27AD2D30
:101360009C2D8B2D97878687C601B50124E630E03A
:1013700040E050E00E941F7A672F782F892F99272D
:101380000E94657AF701718B608B0E94D67D209157
:10139000B1048DB79EB742960FB6F8949EBF0FBEAC
:1013A0008DBF2223A9F000D000D0EDB7FEB7319653
:1013B00087EE91E0ADB7BEB712969C938E931197CE
:1013C000228313820E94E87D0F900F900F900F9060
:1013D0008091711C86FF42C00E945E4DC40104963C
:1013E0000E941D4DEDB7FEB73C970FB6F894FEBFB7
:1013F0000FBEEDBF31967E010894E11CF11CADB724
:10140000BEB71296FC92EE92119780E190E0938322
:1014100082838CE392E095838483D80114968D9126
:101420009C9115979783868316968D919C9117971B
:1014300091878087D4018C91828713860E94467E93
:10144000EDB7FEB73C960FB6F894FEBF0FBEEDBFEA
:1014500082E00E943A4DC7010E941D4D8091E40632
:101460009091E50681FF0DC0749A0BC08EE595E062
:101470000E943B41082F192F0115110509F0D5CE07
:10148000EDCF60960FB6F894DEBF0FBECDBFCF9103
:10149000DF911F910F91FF90EF90DF90CF90BF9061
:1014A000AF909F908F907F906F905F904F90089536
:1014B000EF92FF92CF93DF93E82EE7017E01F92EA2
:1014C000E7018091E4069091E50687FF2FC08DB774
:1014D0009EB70C970FB6F8949EBF0FBE8DBFEDB7A9
:1014E000FEB731968FE492E0ADB7BEB712969C93EB
:1014F0008E9311978A81828313828B8184831582D4
:101500008885868317828C819D81918780878E81D3
:101510009F81938782870E94D67D2DB73EB7245F37
:101520003F4F0FB6F8943EBF0FBE2DBF89E097E046
:10153000BE010E94F5418EE595E0BE010E94614129
:10154000DF91CF91FF90EF90089587EE93E08115A2
:10155000910511F00197F1F708958823E9F0529869
:101560005A981DBA80916900806280936900EA9A56
:101570008091CE049091CF0493FF12C053985B9852
:10158000EB9A80916900806880936900809168007F
:101590008160809368000895109269005A9AEA98D1
:1015A00008951F920F920FB60F9211248F939F935D
:1015B000AF93BF938091680080FF20C08091C824C2
:1015C0009091C924A091CA24B091CB240196A11D69
:1015D000B11D8093C8249093C924A093CA24B093CA
:1015E000CB248091E4069091E50690FF07C07498A3
:1015F00082E090E09093A4048093A304BF91AF9104
:101600009F918F910F900FBE0F901F9018951F9272
:101610000F920FB60F9211248F939F93AF93BF93A6
:101620008091680080FF20C08091CC249091CD24CF
:10163000A091CE24B091CF240196A11DB11D80931D
:10164000CC249093CD24A093CE24B093CF2480912A
:10165000E4069091E50691FF07C0739882E090E060
:101660009093A4048093A304BF91AF919F918F9115
:101670000F900FBE0F901F90189580937C00809163
:101680007B00877F80937B0080917C00806C8093BF
:101690007C0085E080937A0080917A008068809356
:1016A0007A0080917B0087FFFCCF80917B0085FFD3
:1016B000FCCF80917A00806480937A0080917A00D8
:1016C00086FDFCCF109279001092780084E090E0C3
:1016D00060E070E020917A00206420937A002091ED
:1016E0007A0026FDFCCF2091780030917900620FBE
:1016F000731F019779F710927C0080917A008F77A1
:1017000080937A00769567957695679580E090E06E
:101710000E94A277089580E00E943D0B2091A504CD
:101720003091A6044091A7045091A8040E948078AB
:1017300021EE3AE744E95EE30E947076089580E185
:1017400080935101809351019091510195FF03C005
:101750008F5F8F31B9F76BE4869FB0011124882722
:1017600077FD8095982F0E94A47720E030E64FE91E
:1017700054E40E94707620E030E04AE754E40E948E
:101780003A7708958091C80484FF4BC080917B0014
:10179000886080937B0089EC80937C0085E0809357
:1017A0007A0080917A00806880937A0080917B0033
:1017B00087FFFCCF80917B0085FFFCCF80917A0072
:1017C000806480937A0080917A0086FDFCCF8091BE
:1017D0007A00806480937A0080917A0086FDFCCF45
:1017E000609178007091790080E090E00E94A2778B
:1017F00027ED33EA40E95FE30E94807826E636E68B
:1018000048E853E40E946F766093A8177093A91775
:101810008093AA179093AB1780917A008F7780936B
:101820007A0008956F927F928F929F92AF92BF92AB
:10183000CF92DF92EF92FF920F931F93DF93CF939C
:10184000CDB7DEB72A970FB6F894DEBF0FBECDBF77
:101850003C011092EC068FEF898364EEC62E67E19F
:10186000D62E00E010E052E0E52EF12CEC0EFD1E2D
:101870004E010894811C911C4AE0A42EB12CAC0EA0
:10188000BD1E3FC00830110509F441C0C401B701B5
:101890002A870E946A4A89812A858F3F11F08E3FEC
:1018A00019F48093EC0634C06114710479F4C70113
:1018B0000E94844A8093E524F701ADEDB4E2819162
:1018C0008D93EA15FB05D9F721E022C0C7010E94DC
:1018D000844AF6018083D701F80133E0EE0FFF1F41
:1018E0003A95E1F7E00FF11FE452F84E8D918193A4
:1018F000AA15BB05D9F70F5F1F4F89E090E0C80E0E
:10190000D91E202F8981882309F0BCCF01C028E08F
:10191000822F2A960FB6F894DEBF0FBECDBFCF91AF
:10192000DF911F910F91FF90EF90DF90CF90BF90CC
:10193000AF909F908F907F906F90089500D089EB2B
:101940009DE0EDB7FEB7928381830E94E87D0F9002
:101950000F9008952F923F924F925F926F927F92D5
:101960008F929F92AF92BF92CF92DF92EF92FF92AF
:101970000F931F93DF93CF9300D000D0CDB7DEB786
:101980008C01009741F489E290E06BE270E04AE25A
:1019900050E027E00AC08130910549F489E290E0E7
:1019A0006BE270E04AE250E026E00E944649C8013E
:1019B0000E94120CF801E651F94F808301151105C0
:1019C000A1F014EEC12E17E1D12E00E010E04F017E
:1019D000BBE96B2EBDE07B2EA3E94A2EADE05A2E6B
:1019E000FFE82F2EFDE03F2EFAC08DED94E20E941D
:1019F000B64B9C01B901882777FD8095982F0E94EE
:101A0000A477C82EE92EEDEDAE2EE4E2BE2E04EB57
:101A10001DE0D5018D915D0100D000D0EDB7FEB77E
:101A20003196ADB7BEB712961C930E931197828371
:101A300013826B837C830E94E87D0F900F900F9040
:101A40000F906B817C81B5EEAB16B4E2BB0609F753
:101A500000D000D000D00DB71EB70F5F1F4F24EA93
:101A60003DE0EDB7FEB7328321838C2D9E2D20E023
:101A700030E048EC52E40E943A77D80112966D9318
:101A80007D938D939C9315970E94E87DEDB7FEB7EB
:101A900036960FB6F894FEBF0FBEEDBF8091E524D9
:101AA000882319F08EE792E002C087E892E000D028
:101AB00000D020EA3DE0ADB7BEB712963C932E931E
:101AC000119714969C938E9313970E94E87D0F9024
:101AD0000F900F900F900E949E0C88C0780173E0C9
:101AE000EE0CFF1C7A95E1F7E00EF11EECEDF7E14C
:101AF000EE0EFF1EC7010E94B64B9C01B90188275C
:101B000077FD8095982F0E94A4775C0120E030E05B
:101B1000D7018D917D0100D000D0EDB7FEB7319691
:101B2000ADB7BEB712967C926E92119782831382E4
:101B300029833A836B837C830E94E87D29813A81E3
:101B40002F5F3F4F0F900F900F900F906B817C8114
:101B500028303105E9F600D000D000D0EDB6FEB651
:101B60000894E11CF11CEDB7FEB7528241828A2D28
:101B70009B2D20E030E048EC52E40E943A77D701F8
:101B800012966D937D938D939C9315970E94E87D9B
:101B9000EDB7FEB736960FB6F894FEBF0FBEEDBF99
:101BA000D6018C91882319F08EE792E002C087E875
:101BB00092E000D000D0EDB7FEB73282218294834C
:101BC00083830E94E87D0F900F900F900F900E94EA
:101BD0009E0C0F5F1F4F29E030E0C20ED31ED401D0
:101BE0008C9190E0081719070CF478CF0F900F90A4
:101BF0000F900F90CF91DF911F910F91FF90EF9079
:101C0000DF90CF90BF90AF909F908F907F906F901C
:101C10005F904F903F902F900895DF93CF9300D027
:101C2000CDB7DEB78091DE2489838091E4248A8356
:101C3000CE0101960E948F3E0F900F90CF91DF91C1
:101C40000895CF93DF93EC018091DD248F3FB1F5B0
:101C50008091DE248F3F91F58091DF248F3F71F5D5
:101C60008091E0248F3F51F58091E1248F3F31F541
:101C70008091E2248F3F11F58091E3248F3FF1F4AE
:101C80008091E4248F3FD1F489E290E06BE270E030
:101C90004AE250E027E00E94464980E090E00E943E
:101CA000120CC651D94F88838DED94E268E170E043
:101CB00049E050E00E94387F0E940D0EDF91CF91E5
:101CC00008951F920F920FB60F920BB60F92112428
:101CD0001F932F933F934F935F936F937F938F93B4
:101CE0009F93AF93BF93EF93FF938091E82482601B
:101CF0008093E8248091CE0486FD2B9A8091CE04B7
:101D000087FD2B9A8091A3049091A40418161906BC
:101D100014F4749A739A8091E4069091E50685FF15
:101D200002C0749873988091660590916705019739
:101D30009093670580936605009709F07EC08091B7
:101D40001807909119070196909319078093180727
:101D5000209173203091742040917520509176200D
:101D60002F5F3F4F4F4F5F4F20937320309374206E
:101D7000409375205093762020E130E03093670542
:101D8000209366052091CE0420FD02C01D9B05C056
:101D90001092E8061092E70606C021E030E030938A
:101DA000E8062093E7066091CC047091CD0461159C
:101DB000710599F001960E943E7A009771F4779828
:101DC0008091E4069091E50693FF07C0749884E043
:101DD00090E09093A4048093A3046091CC0470914C
:101DE000CD046115710579F080911807909119075C
:101DF0000E943E7A009739F481E195E062E140E08B
:101E000050E00E94B0408091CE0486FD2B988091D6
:101E1000CE049091CF0491FF10C00E948D558A315D
:101E200019F0182F1F5F01C01BE00E94D153812FB2
:101E300090E00E94A5550E946F5480E895E060E014
:101E400040E050E00E94B040FF91EF91BF91AF9110
:101E50009F918F917F916F915F914F913F912F91C2
:101E60001F910F900BBE0F900FBE0F901F901895F3
:101E70008091D31790918720891B08950E94380F75
:101E8000882379F0E0918720F0E0EF71F070E85D51
:101E9000F74E208130E0809187208F5F80938720EC
:101EA00002C02FEF3FEFC9010895CF93DF93EC01FC
:101EB00010920C0710920B0788819981009731F0DE
:101EC00022E0853D920709F0B9C009C00E94380F91
:101ED000882341F485ED92E099838883B3C0613112
:101EE00009F0B0C0F89478940E943E0F90E090936F
:101EF000100780930F078D3009F47CC08F3F31F3BA
:101F00008231910569F18F37910521F08830910573
:101F100009F053C080911307909114071816190601
:101F20000CF060C06091A82D7091A92D88E090E020
:101F30000E94AA7D6091A82D7091A92D80E290E069
:101F40000E94AA7D6091A82D7091A92D88E090E053
:101F50000E94AA7D809113079091140701973EC0BB
:101F60006091A82D7091A92D8DE090E00E94AA7D2E
:101F7000109212071092110714C088579F4DFC0150
:101F800080816091A82D7091A92D90E00E94AA7D7A
:101F900080911107909112070196909312078093F8
:101FA000110780911107909112072091130730912A
:101FB0001407821793070CF315C06091A82D709138
:101FC000A92D0E94AA7D809113079091140720915A
:101FD0000F07FC01E857FF4D2083019690931407EB
:101FE0008093130780911307909114078F33910505
:101FF00009F06CCF10928720809187208093D317AF
:102000008091130790911407FC01E857FF4D10824F
:1020100090930C0780930B071092140710921307EC
:102020008091E6249091E724009709F44FCF6091C6
:102030000D0740E050E00E94B04048CF198218825E
:1020400083E001C081E0DF91CF9108957894809181
:10205000E7069091E806009731F08091CE049091C8
:10206000CF0492FF03C083B7817F03C083B7817F12
:10207000866083BFF89483B7816083BF7894889526
:1020800083B78E7F83BF78940895CF93DF93EC015D
:1020900088819981009721F02AE08F3A920799F47C
:1020A0000E94BF520E94261080919E0E90919F0E1A
:1020B00065E840E050E00E94B0408FEA9AE09983E2
:1020C000888381E003C01982188283E0DF91CF9179
:1020D0000895CF93DF930E94BF5280EB0E94364C4D
:1020E0008823B1F40E949C4C8091711C9091721CC9
:1020F00081609093721C8093711C00D086E89DE0F3
:10210000EDB7FEB7928381830E94E87D0F900F9018
:102110008EB1C82FD0E0C470D070729A0E94BF52A6
:102120008EE40E94364C8823B1F40E949C4C80912E
:10213000711C9091721C82609093721C8093711C30
:1021400000D08DE79DE0EDB7FEB7928381830E94BA
:10215000E87D0F900F90209709F472980E94BF526B
:102160008EEE0E94364C8823B1F40E949C4C8091E4
:10217000711C9091721C84609093721C8093711CEE
:1021800000D085E79DE0EDB7FEB7928381830E9482
:10219000E87D0F900F9086EA0E94364C8823B1F4B8
:1021A0000E949C4C8091711C9091721C886090934D
:1021B000721C8093711C00D08CE69DE0EDB7FEB7D9
:1021C000928381830E94E87D0F900F900E94BF52FE
:1021D0008CE30E94364C8823B1F40E949C4C809181
:1021E000711C9091721C80619093721C8093711C81
:1021F00000D083E69DE0EDB7FEB7928381830E9415
:10220000E87D0F900F900E94BF5282ED0E94364CE5
:102210008823B1F40E949C4C8091711C9091721C97
:1022200080629093721C8093711C00D089E59DE0C0
:10223000EDB7FEB7928381830E94E87D0F900F90E7
:10224000C7E0D0E00E94BF528CE70E94364C882342
:10225000B9F40E949C4C8091711C9091721C806416
:102260009093721C8093711C00D08FE49DE0EDB7B9
:10227000FEB7928381830E94E87D0F900F9002C089
:10228000219701F70E949C4C0E949E0CDF91CF91F8
:102290000895DF93CF9300D0CDB7DEB74A8369832B
:1022A0000E94724C6981862F0E94A44C4A81842F1F
:1022B0000E94A44C0E949C4C0F900F90CF91DF91F4
:1022C0000895AF92BF92DF92EF92FF920F931F9308
:1022D000DF93CF9300D00F92CDB7DEB7082FD22E69
:1022E0004A835B8369830E94724C6981862F0E94B6
:1022F000A44C802F81600E94994C4A815B81042FFD
:10230000152FAA24BB24ED2CFF240894E108F10822
:102310000FC0AE14BF0419F40E94BF4C02C00E944B
:10232000B54CF80180830894A11CB11C0F5F1F4FAE
:10233000AD1478F30E949C4C0F900F900F90CF91AA
:10234000DF911F910F91FF90EF90DF90BF90AF90C2
:102350000895AF92BF92CF92DF92EF92FF920F93C8
:102360001F93DF93CF93CDB7DEB760970FB6F89486
:10237000DEBF0FBECDBFB82EA42E662309F455C014
:10238000AE014F5F5F4F80E1DA011D928A95E9F758
:1023900080EB68E928E00E946111BB2059F000D071
:1023A00088E892E0EDB7FEB7928381830E94D67DE4
:1023B0000F900F908E010F5F1F4F38E0E32EF12C2E
:1023C000EC0EFD1E2FE8C22E22E0D22ED8018D91F8
:1023D0008D0100D000D0EDB7FEB73196ADB7BEB7D6
:1023E0001296DC92CE921197828313820E94D67D40
:1023F0000F900F900F900F900E151F0539F700D01A
:1024000000D0EDB7FEB7319684E992E0ADB7BEB724
:1024100012969C938E9311978885828313820E94D3
:10242000D67D0F900F900F900F90AA2009F457C0FF
:10243000AE014F5F5F4F80E1FA0111928A95E9F793
:1024400080EB60E828E00E946111BB2069F000D0B9
:102450008AE992E0ADB7BEB712969C938E9311971E
:102460000E94D67D0F900F908E010F5F1F4F90E15D
:10247000E92EF12CEC0EFD1E8FE8C82E82E0D82E3E
:10248000F80181918F0100D000D0EDB7FEB73196F1
:10249000ADB7BEB71296DC92CE92119782831382AB
:1024A0000E94D67D0F900F900F900F900E151F0574
:1024B00039F700D000D0EDB7FEB7319684E992E04D
:1024C000ADB7BEB712969C938E9311978885828381
:1024D00013820E94D67D0F900F900F900F90609600
:1024E0000FB6F894DEBF0FBECDBFCF91DF911F9125
:1024F0000F91FF90EF90DF90CF90BF90AF90089535
:102500000F931F93DF93CF9300D0CDB7DEB71A821E
:1025100019828EEE6AEA8E010F5F1F4FA80122E03A
:102520000E946111398120E08A8190E0822B932BF7
:1025300090934918809348188EEE6CEAA80122E027
:102540000E946111398120E08A8190E0822B932BD7
:1025500090934B1880934A188EEE6EEAA80122E001
:102560000E946111398120E08A8190E0822B932BB7
:1025700090934D1880934C188EEE60EBA80122E0EA
:102580000E946111398120E08A8190E0822B932B97
:1025900090935B1880935A188EEE62EBA80122E0AC
:1025A0000E946111398120E08A8190E0822B932B77
:1025B00090935D1880935C188EEE64EBA80122E086
:1025C0000E946111398120E08A8190E0822B932B57
:1025D00090935F1880935E188EEE66EBA80122E060
:1025E0000E946111398120E08A8190E0822B932B37
:1025F00090934F1880934E188EEE68EBA80122E05E
:102600000E946111398120E08A8190E0822B932B16
:1026100090935118809350188EEE6AEBA80122E037
:102620000E946111398120E08A8190E0822B932BF6
:1026300090935518809354188EEE6CEBA80122E00D
:102640000E946111398120E08A8190E0822B932BD6
:1026500090935718809356188EEE6EEBA80122E0E7
:102660000E946111398120E08A8190E0822B932BB6
:1026700090935918809358180F900F90CF91DF9135
:102680001F910F9108952F923F924F925F926F92F8
:102690007F928F929F92AF92BF92CF92DF92EF92F2
:1026A000FF920F931F93DF93CF93CDB7DEB76C9755
:1026B0000FB6F894DEBF0FBECDBFA82E4A8B2B8F6E
:1026C000FE01319683E0DF011D928A95E9F7809142
:1026D0006C18882339F46C8F0E94801281E08093FB
:1026E0006C186C8D662309F475C08EEE64EF4EE2B3
:1026F0000E94491169E07AE180E090E00E94234C59
:102700008EEE66EFAE014F5F5F4F22E00E946111D7
:10271000698170E080E090E0982F872F762F662700
:102720002A8130E040E050E0622B732B842B952B04
:1027300020915E1830915F1840E050E0621B730BEF
:10274000840B950B20915C1830915D1840E050E0AF
:102750000E941F7A7B018C013FE015950795F79445
:10276000E7943A95D1F760915618709157188827D9
:1027700077FD8095982F2BE0660F771F881F991F94
:102780002A95D1F72091581830915918442737FDD0
:102790004095542F2E0D3F1D401F511F0E94877AD8
:1027A0002E0D3F1D3093531820935218285F3F4F32
:1027B00014E0359527951A95E1F779010027F7FC84
:1027C0000095102FE0926018F09261180093621843
:1027D00010936318BA2DB295BB0FBB0FB07CBC5CD5
:1027E000B9872A2D30E03E8B2D8B63E070E00A2CF8
:1027F00002C0660F771F0A94E2F7882777FD80955D
:10280000982F25E335E040E050E00E941F7ADC017C
:10281000CB010296A11DB11D8A879B87AC87BD871E
:1028200020E533EC40E050E004C0559547953795DE
:102830002795AA94D2F72E873F87488B598B188605
:102840001C821D821E821F8248E050E08D899E8975
:10285000481B590B5C8B4B8B69C18EEE64EF49852D
:102860000E9449116A857B858C859D850E94234C39
:102870008EEE66EFAE014F5F5F4F23E00E94611165
:102880008091521890915318805A9F401C01442403
:1028900037FC4094542CC201B101A20191010E9465
:1028A0001F7A6F8B788F898F9A8F20914C18309177
:1028B0004D18442737FD4095542FC201B1010E94A5
:1028C0001F7A7B018C01BDE015950795F794E7947D
:1028D000BA95D1F722E030E040E050E0E20EF31E7E
:1028E000041F151F6F89788D898D9A8DACE09595A1
:1028F000879577956795AA95D1F720914E183091D5
:102900004F18442737FD4095542F0E941F7ABC0171
:10291000992777FD9095892FE60EF71E081F191F3E
:10292000E2E015950795F794E794EA95D1F780E0F2
:1029300090E8A0E0B0E0E80EF91E0A1F1B1F2091EE
:102940005A1830915B1840E050E0C801B7010E946E
:102950001F7A3B014C017FE09694879477946794AB
:102960007A95D1F7A980BB24CC24DD246501BB2452
:10297000AA248A8190E0A0E0B0E0BA2FA92F982F76
:102980008827A82AB92ACA2ADB2A8B8190E0A0E0EE
:10299000B0E0A82AB92ACA2ADB2A0B8804C0D59439
:1029A000C794B794A7940A94D2F720914A1830910B
:1029B0004B18442737FD4095542FC201B1010E94A6
:1029C0001F7A7B018C014BE015950795F794E794EE
:1029D0004A95D1F78091481890914918AA2797FDF8
:1029E000A095BA2F32E0880F991FAA1FBB1F3A95F6
:1029F000D1F7E80EF91E0A1F1B1F209150183091C5
:102A00005118442737FD4095542F6F89788D898D53
:102A10009A8D0E941F7A27E19595879577956795FE
:102A20002A95D1F7E60EF71E081F191F0D8804C05E
:102A3000EE0CFF1C001F111F0A94D2F722E030E0B9
:102A400040E050E0E20EF31E041F151F82E01595D2
:102A50000795F794E7948A95D1F7AE18BF08C00A96
:102A6000D10AC601B5012E853F85488959890E9442
:102A70001F7A97FD0BC0660F771F881F991FA4014F
:102A800093010E94657A79018A010AC0A401930129
:102A90000E94657A79018A01EE0CFF1C001F111F4C
:102AA000552717FD5A95412F302F2F2DCA01B901F7
:102AB0000E941F7A2EED3BE040E050E00E941F7A1A
:102AC0005B016C01C801B70123E433EE4FEF5FEF08
:102AD0000E941F7ABC01992777FD9095892F615339
:102AE000714F8F4F9F4F5601DD24B7FCD094CD2CF2
:102AF0006A0D7B1D8C1D9D1D44E0959587957795EE
:102B000067954A95D1F76E0D7F1D801F911F2C810F
:102B10003D814E815F81260F371F481F591F2C832F
:102B20003D834E835F8338853F5F388748855A8968
:102B3000451708F492CE552391F0252F30E040E060
:102B400050E06C817D818E819F810E94657A209307
:102B500064183093651840936618509367188B8DEE
:102B60008823C9F160916418709165188091661886
:102B700090916718611571058105910561F10E94B9
:102B8000A47720E836EE45EC57E40E943A7721E03E
:102B90003EED42E45EE30E94E378562F472F382F44
:102BA000292F60E070E080E89FE3DA01F9012B2F24
:102BB0003A2F4F2F5E2F0E946F762BE43AE34DEBB6
:102BC00057E30E943A77609368187093691880936E
:102BD0006A1890936B186C960FB6F894DEBF0FBE10
:102BE000CDBFCF91DF911F910F91FF90EF90DF90BC
:102BF000CF90BF90AF909F908F907F906F905F909D
:102C00004F903F902F900895DF93CF9300D000D046
:102C100000D0CDB7DEB7FE01319686E0DF011D9210
:102C20008A95E9F78091B217882399F486EA61E3DF
:102C300040E00E94491186EA6CE24AE00E94491194
:102C400081E08093B2176CE77EE380E090E00E9421
:102C5000234C86EA6DE248E00E9449116CE77EE36E
:102C600080E090E00E94234C86EA62E3AE014F5F71
:102C70005F4F26E00E94611186EA6DE247E00E9404
:102C800049119A8180E0498150E0482B592B50939B
:102C9000AD174093AC179C8180E02B8130E0282B4E
:102CA000392B3093AF172093AE177E8160E08D8172
:102CB00090E0862B972B9093B1178093B0176DB748
:102CC0007EB7685070400FB6F8947EBF0FBE6DBFE0
:102CD000EDB7FEB731966EE972E0ADB7BEB71296AA
:102CE0007C936E9311975383428335832483978318
:102CF00086830E94D67D6DB77EB7685F7F4F0FB623
:102D0000F8947EBF0FBE6DBF26960FB6F894DEBF57
:102D10000FBECDBFCF91DF910895CF92DF92EF929A
:102D2000FF920F931F93DF93CF9300D000D000D07A
:102D3000CDB7DEB78E010F5F1F4F86E0F80111920D
:102D40008A95E9F78CE362E041E00E9449118CE347
:102D500060E048E50E94491162E174E380E090E0A0
:102D60000E94234C8CE363E0A80126E00E946111DD
:102D70008CE362E043E00E944911998180E00A817E
:102D800010E0082B192B10939317009392179B8137
:102D900080E06C8170E0682B792B709395176093BD
:102DA00094173D8120E08E8190E0822B932B9093AD
:102DB000971780939617882777FD8095982F0E9404
:102DC000A4776B017C01B801882777FD8095982F47
:102DD0000E94A4779B01AC01C701B6010E94E37673
:102DE0002DB73EB72C5030400FB6F8943EBF0FBE03
:102DF0002DBF0DB71EB70F5F1F4F2CEA32E0EDB7A6
:102E0000FEB7328321832091921730919317F801F6
:102E1000338322832091941730919517358324832F
:102E200020919617309197173783268320EE3EE244
:102E300045E652E40E94807820E030E044E353E429
:102E40000E947076F80160877187828793870E945D
:102E5000D67D2DB73EB7245F3F4F0FB6F8943EBFE7
:102E60000FBE2DBF26960FB6F894DEBF0FBECDBFA6
:102E7000CF91DF911F910F91FF90EF90DF90CF9056
:102E80000895CF93DF93EC0188819981009731F009
:102E90002AE08839920709F071C00BC08DEE96E0E8
:102EA00060E870E00E94664388E99AE0998388832D
:102EB00069C08DEE96E00E949143009709F462C0CC
:102EC0008091E4069091E50694FF3FC08091711CCB
:102ED00082FF3BC083E061E048E021E00E944313B1
:102EE0008DB79EB70A970FB6F8949EBF0FBE8DBFE1
:102EF000EDB7FEB731968FEC91E0ADB7BEB7129645
:102F00009C938E9311978091641890916518A0916D
:102F10006618B091671882839383A483B5838091E8
:102F2000681890916918A0916A18B0916B188683FF
:102F30009783A087B1870E94E87D8DB79EB70A96D8
:102F40000FB6F8949EBF0FBE8DBF8091E40690919E
:102F5000E50695FF06C08091711C83FF02C00E94A8
:102F600004168091E4069091E50696FF97CF809134
:102F7000711C84FF93CF0E948D1690CF1982188206
:102F800083E001C081E0DF91CF910895CF92DF927D
:102F9000FF920F931F93CF93DF93729A8091CE0489
:102FA00083FD06C0C0E5D0E00E94A50A2197E1F7A5
:102FB0008EE40E94364C8823B1F080917720909166
:102FC0007820A0917920B0917A200196A11DB11DA1
:102FD0008093772090937820A0937920B0937A20E3
:102FE00021E030E084C0C0E5D0E00E94A50A21972E
:102FF000E1F78FE40E94364C0E94B54CF82E829582
:103000008695869583708130A9F420917B2030913C
:103010007C2040917D2050917E202F5F3F4F4F4F6D
:103020005F4F20937B2030937C2040937D205093F2
:103030007E2016C08230A0F020917F203091802029
:1030400040918120509182202F5F3F4F4F4F5F4F23
:1030500020937F20309380204093812050938220C2
:103060000E94B54C1F2D1F7300E0080F111D0E9418
:10307000B54C0E94BF4C20E0E901C80FD11DD69588
:10308000C795D695C7950E949C4C8091CE0483FF2E
:103090007298B80180E090E00E94A27720E134E0CD
:1030A00048EC5BE30E94807860936D1870936E1813
:1030B00080936F1890937018BE0180E090E00E949A
:1030C000A27724EA3CEF44E25CE30E94807820E0AF
:1030D00030E040E252E40E946F766093E9247093FE
:1030E000EA248093EB249093EC2420E030E0C901A3
:1030F000DF91CF911F910F91FF90DF90CF900895B6
:103100007298729A8EE40E94364C80EA0E94A44C17
:1031100080E00E94A44C80E00E94A44C8FE40E94B6
:10312000364C0E94B54C8295869586958370813089
:10313000A9F420917B2030917C2040917D205091FA
:103140007E202F5F3F4F4F4F5F4F20937B20309368
:103150007C2040937D2050937E2016C08230A0F0CA
:1031600020917F20309180204091812050918220B9
:103170002F5F3F4F4F4F5F4F20937F203093802032
:10318000409381205093822000D000D0EDB7FEB74D
:10319000319621EC32E0ADB7BEB712963C932E9338
:1031A0001197828313820E94D67D0F900F900F900B
:1031B0000F908EE40E94364C80E80E94A44C80E080
:1031C0000E94A44C80E00E94A44C0E949C4C80E091
:1031D00090E0089500D082E49DE0ADB7BEB71296AE
:1031E0009C938E9311970E94E87D2091B1040F90DB
:1031F0000F902223A9F000D000D0EDB7FEB7319692
:103200008FE39DE0ADB7BEB712969C938E93119756
:10321000228313820E94E87D0F900F900F900F90F1
:10322000089500D08AE19DE0EDB7FEB792838183D7
:103230000E94E87D82EF9CE0EDB7FEB79283818328
:103240000E94E87D8BEC9CE0EDB7FEB79283818312
:103250000E94E87D81EA9CE0EDB7FEB7928381830E
:103260000E94E87D86E69CE0EDB7FEB792838183FD
:103270000E94E87D84E39CE0EDB7FEB792838183F2
:103280000E94E87D88EF9BE0EDB7FEB792838183D3
:103290000E94E87D82ED9BE0EDB7FEB792838183CB
:1032A0000E94E87D82EA9BE0EDB7FEB792838183BE
:1032B0000E94E87D89E69BE0EDB7FEB792838183AB
:1032C0000E94E87D8DE39BE0EDB7FEB7928381839A
:1032D0000E94E87D84E19BE0EDB7FEB79283818395
:1032E0000E94E87D89EE9AE0EDB7FEB79283818374
:1032F0000E94E87D8AEB9AE0EDB7FEB79283818366
:103300000E94E87D88E89AE0EDB7FEB7928381835A
:103310000E94E87D87E59AE0EDB7FEB7928381834E
:103320000E94E87D83E29AE0EDB7FEB79283818345
:103330000E94E87D83EF99E0EDB7FEB79283818329
:103340000E94E87D87EC99E0EDB7FEB79283818318
:103350000E94E87D88E999E0EDB7FEB7928381830A
:103360000E94E87D8FE599E0EDB7FEB792838183F7
:103370000E94E87D86E399E0EDB7FEB792838183F2
:103380000E94E87D87EF98E0EDB7FEB792838183D6
:103390000E94E87D88EC98E0EDB7FEB792838183C8
:1033A0000E94E87D89E998E0EDB7FEB792838183BA
:1033B0000E94E87D82E798E0EDB7FEB792838183B3
:1033C0000E94E87D8CE398E0EDB7FEB7928381839D
:1033D0000E94E87D83E198E0EDB7FEB79283818398
:1033E0000E94E87D88EE97E0EDB7FEB79283818377
:1033F0000E94E87D0F900F90089581ED92E00E9469
:103400000F7E08952F923F924F925F926F927F921C
:103410008F929F92AF92BF92CF92DF92EF92FF92E4
:103420000F931F93CF93DF9360917320709174205B
:103430008091752090917620A0907320B090742098
:10344000C0907520D090762060907320709074208A
:10345000809075209090762020907320309074207A
:1034600040907520509076202DB73EB72A503040BE
:103470000FB6F8943EBF0FBE2DBFCDB7DEB7219675
:1034800028EC37E0EDB7FEB732832183A0E8EA2EBF
:10349000A1E5FA2EA1E00A2F112DA80197010E94A3
:1034A000657A3B832A83C601B501A80197010E9472
:1034B000657AF0E1EF2EFEE0FF2E012D112DA8011F
:1034C00097010E94657A332727FD30953D832C8331
:1034D000C401B301A80197010E94657AECE3EE2EC6
:1034E000F12C012D112DA80197010E94657A332737
:1034F00027FD30953F832E83C201B101A8019701BA
:103500000E94657A772767FD7095798768870E94A2
:10351000E87D2DB73EB7265F3F4F0FB6F8943EBF0C
:103520000FBE2DBFDF91CF911F910F91FF90EF90B4
:10353000DF90CF90BF90AF909F908F907F906F90D3
:103540005F904F903F902F900895EEEAFDE28081CA
:10355000918122E482349207B9F000D000D08AEA47
:1035600097E0ADB7BEB712969C938E931197EE5A23
:10357000FD421496FC93EE9313970E94E87D0F9002
:103580000F900F900F9008953A96B1E4E53FFB0736
:10359000F0F208958F929F92AF92BF92CF92DF92F6
:1035A000EF92FF920F931F938C9A0E948B0B00D087
:1035B00000D000D023EA37E0ADB7BEB712963C93F7
:1035C0002E931197EDB7FEB763837483858396833B
:1035D0000E94E87D8DB79EB706960FB6F8949EBF01
:1035E0000FBE8DBF81E00E943D0B2091A904309158
:1035F000AA044091AB045091AC040E9480787B01F6
:103600008C0182E00E943D0B2091AD043091AE040C
:103610004091AF045091B0040E948078B62EC72E1E
:10362000D82EA92E83E00E943D0B9B01AC01ADB7C3
:10363000BEB71E970FB6F894BEBF0FBEADBFEDB7B5
:10364000FEB7319681E997E012969C938E9311977D
:10365000C701A02FB12F82839383A483B5830B2D41
:103660001C2DC801AD2DBA2D86839783A087B18705
:1036700022873387448755870E94E87D8C98EDB771
:10368000FEB73E960FB6F894FEBF0FBEEDBF0E9488
:103690009E0C1F910F91FF90EF90DF90CF90BF9005
:1036A000AF909F908F9008950F931F93CF93DF93C8
:1036B000882389F08DED94E26FEF70E049E050E0EF
:1036C0000E94607D8DED94E268E170E049E050E099
:1036D0000E94387F1CC0CDEDD4E20CE817E0899140
:1036E00000D000D0EDB7FEB73196ADB7BEB7129699
:1036F0001C930E931197828313820E94E87D0F9092
:103700000F900F900F90B4E2C53EDB0741F70E9487
:103710009E0CDF91CF911F910F910895EF92FF9230
:103720000F931F936091B6047091B70480E090E00E
:103730000E94527D65EF72E00E94677D009709F05C
:1037400096C086E294E9A0E0B0E08093C80490932C
:10375000C904A093CA04B093CB0488EC94E06EE053
:1037600070E044E050E00E94387F8CE390E090935A
:10377000CD048093CC048CEC94E062E170E042E0F4
:1037800050E00E94387F8AE090E09093CF048093CD
:10379000CE048EEC94E064E170E042E050E00E94E0
:1037A000387F1092E5061092E40684EE96E060E021
:1037B00070E042E050E00E94387F0F2EF2E2EF2EE0
:1037C000FFEFFF2EFCEC0F2FFBE31F2FF02DE092FD
:1037D000A904F092AA040093AB041093AC0489EA04
:1037E00094E066E070E044E050E00E94387FE092B0
:1037F000AD04F092AE040093AF041093B0048DEAD0
:1038000094E06AE070E044E050E00E94387F87ED89
:1038100094E3AFEEBCE38093A5049093A604A09339
:10382000A704B093A80485EA94E062E070E044E065
:1038300050E00E94387F1092E90689EE96E066E13A
:1038400070E041E050E00E94387F8AE18093E90611
:1038500080ED94E067E170E041E050E00E94387F45
:1038600081E00E94541B80E090E00E94210E1F9195
:103870000F91FF90EF900895882309F44BC1809138
:10388000C80480FF0BC000D086E897E0EDB7FEB714
:10389000928381830E94E87D0F900F908091C804ED
:1038A00081FF0BC000D08FE797E0EDB7FEB79283A2
:1038B00081830E94E87D0F900F908091C80482FF61
:1038C0000BC000D08AE797E0EDB7FEB79283818303
:1038D0000E94E87D0F900F908091C80483FF0BC079
:1038E00000D084E797E0EDB7FEB7928381830E9412
:1038F000E87D0F900F908091C80484FF0BC000D02A
:103900008BE697E0EDB7FEB7928381830E94E87D56
:103910000F900F908091C80485FF0BC000D082E605
:1039200097E0EDB7FEB7928381830E94E87D0F9008
:103930000F908091C80486FF0BC000D08CE597E003
:10394000EDB7FEB7928381830E94E87D0F900F90C0
:103950008091C80487FF0BC000D084E597E0EDB7E5
:10396000FEB7928381830E94E87D0F900F90809133
:10397000C8049091C904A091CA04B091CB0490FFEF
:103980000BC000D08EE497E0EDB7FEB79283818341
:103990000E94E87D0F900F908091C8049091C90417
:1039A000A091CA04B091CB0491FF0BC000D086E473
:1039B00097E0EDB7FEB7928381830E94E87D0F9078
:1039C0000F908091C8049091C904A091CA04B0914D
:1039D000CB0492FF0BC000D08CE397E0EDB7FEB7AD
:1039E000928381830E94E87D0F900F908091C8049C
:1039F0009091C904A091CA04B091CB0493FF0BC06D
:103A000000D086E397E0EDB7FEB7928381830E94F2
:103A1000E87D0F900F908091C8049091C904A09107
:103A2000CA04B091CB0494FF0BC000D08EE297E0A3
:103A3000EDB7FEB7928381830E94E87D0F900F90CF
:103A40008091C8049091C904A091CA04B091CB049C
:103A500095FF0BC000D088E297E0EDB7FEB79283E8
:103A600081830E94E87D0F900F908091C80490910F
:103A7000C904A091CA04B091CB0496FF0BC000D03A
:103A800082E297E0EDB7FEB7928381830E94E87DE2
:103A90000F900F908091C8049091C904A091CA041E
:103AA000B091CB0497FF0BC000D08CE197E0EDB74D
:103AB000FEB7928381830E94E87D0F900F908091E2
:103AC000C8049091C904A091CA04B091CB04A0FF8E
:103AD0000BC000D087E197E0EDB7FEB792838183FA
:103AE0000E94E87D0F900F908091C8049091C904C6
:103AF000A091CA04B091CB04A1FF14C200D081E10F
:103B000097E0EDB7FEB7928381830E94E87D0F9026
:103B10000F9008C200D000D000D085E097E0EDB74C
:103B2000FEB79283818381E090E0A0E0B0E08383E0
:103B30009483A583B6830E94E87D8DB79EB70696D1
:103B40000FB6F8949EBF0FBE8DBF0E949E0C00D092
:103B500000D000D088EF96E0EDB7FEB79283818366
:103B600082E090E0A0E0B0E083839483A583B683F5
:103B70000E94E87D8DB79EB706960FB6F8949EBF5B
:103B80000FBE8DBF0E949E0C00D000D000D08DEEE5
:103B900096E0EDB7FEB79283818384E090E0A0E0E9
:103BA000B0E083839483A583B6830E94E87D8DB7BC
:103BB0009EB706960FB6F8949EBF0FBE8DBF0E94AB
:103BC0009E0C00D000D000D081EE96E0EDB7FEB79D
:103BD0009283818388E090E0A0E0B0E083839483C7
:103BE000A583B6830E94E87D8DB79EB706960FB673
:103BF000F8949EBF0FBE8DBF0E949E0C00D000D0D7
:103C000000D083ED96E0EDB7FEB79283818380E12B
:103C100090E0A0E0B0E083839483A583B6830E9404
:103C2000E87D8DB79EB706960FB6F8949EBF0FBE7F
:103C30008DBF0E949E0C00D000D000D085EC96E095
:103C4000EDB7FEB79283818380E290E0A0E0B0E020
:103C500083839483A583B6830E94E87D8DB79EB746
:103C600006960FB6F8949EBF0FBE8DBF0E949E0CA5
:103C700000D000D000D089EB96E0EDB7FEB792837C
:103C8000818380E490E0A0E0B0E083839483A58307
:103C9000B6830E94E87D8DB79EB706960FB6F8945E
:103CA0009EBF0FBE8DBF0E949E0C00D000D000D0E2
:103CB0008BEA96E0EDB7FEB79283818380E890E0CF
:103CC000A0E0B0E083839483A583B6830E94E87D5F
:103CD0008DB79EB706960FB6F8949EBF0FBE8DBFE8
:103CE0000E949E0C00D000D000D08FE996E0EDB786
:103CF000FEB79283818380E091E0A0E0B0E083830F
:103D00009483A583B6830E94E87D8DB79EB70696FF
:103D10000FB6F8949EBF0FBE8DBF0E949E0C00D0C0
:103D200000D000D081E996E0EDB7FEB792838183A1
:103D300080E092E0A0E0B0E083839483A583B68323
:103D40000E94E87D8DB79EB706960FB6F8949EBF89
:103D50000FBE8DBF0E949E0C00D000D000D082E824
:103D600096E0EDB7FEB79283818380E094E0A0E017
:103D7000B0E083839483A583B6830E94E87D8DB7EA
:103D80009EB706960FB6F8949EBF0FBE8DBF0E94D9
:103D90009E0C00D000D000D086E796E0EDB7FEB7CD
:103DA0009283818380E098E0A0E0B0E083839483F5
:103DB000A583B6830E94E87D8DB79EB706960FB6A1
:103DC000F8949EBF0FBE8DBF0E949E0C00D000D005
:103DD00000D088E696E0EDB7FEB79283818380E05D
:103DE00090E1A0E0B0E083839483A583B6830E9432
:103DF000E87D8DB79EB706960FB6F8949EBF0FBEAE
:103E00008DBF0E949E0C00D000D000D08CE596E0C3
:103E1000EDB7FEB79283818380E090E2A0E0B0E04E
:103E200083839483A583B6830E94E87D8DB79EB774
:103E300006960FB6F8949EBF0FBE8DBF0E949E0CD3
:103E400000D000D000D080E596E0EDB7FEB79283B9
:103E5000818380E090E4A0E0B0E083839483A58335
:103E6000B6830E94E87D8DB79EB706960FB6F8948C
:103E70009EBF0FBE8DBF0E949E0C00D000D000D010
:103E800084E496E0EDB7FEB79283818380E090E80A
:103E9000A0E0B0E083839483A583B6830E94E87D8D
:103EA0008DB79EB706960FB6F8949EBF0FBE8DBF16
:103EB0000E949E0C00D000D000D088E396E0EDB7C1
:103EC000FEB79283818380E090E0A1E0B0E083833D
:103ED0009483A583B6830E94E87D8DB79EB706962E
:103EE0000FB6F8949EBF0FBE8DBF0E949E0C00D0EF
:103EF00000D000D08BE296E0EDB7FEB792838183CD
:103F000080E090E0A2E0B0E083839483A583B68351
:103F10000E94E87D8DB79EB706960FB6F8949EBFB7
:103F20000FBE8DBF0E949E0C08952F923F924F921C
:103F30005F926F927F928F929F92AF92BF92CF9239
:103F4000DF92EF92FF920F931F93DF93CF9300D0F6
:103F5000CDB7DEB79A838983DC018D919C9111974F
:103F6000009711F00C9495336091B6047091B704EA
:103F700088E890E20E94527D88E890E260E470E078
:103F80000E94707D009759F46091A82D7091A92D21
:103F90008AE090E00E94AA7D81E00C949A338130FF
:103FA000910549F420908820332444245524662424
:103FB00077244301BFC18230910599F43091882064
:103FC00020918920932F80E0820F911D1C01892F61
:103FD000880F880B482E582E682E782E882E982E03
:103FE000A9C18330910509F09CC020918820A09040
:103FF000892080908A2030E040E050E060E070E06E
:1040000080E090E000E10E940C72F22E132FE42E6B
:10401000D52EC62EB72E282E992E2A2D30E040E020
:1040200050E060E070E080E090E008E00E940C72F8
:104030002F0DB1E02F1508F0B0E0310FE1E031179E
:1040400008F0E0E0B30FF1E0B31708F0F0E0EF2B79
:104050004E0D31E04E1508F030E0E40FF1E0E417CA
:1040600008F0F0E03F2B5D0D41E05D1508F040E009
:10407000A32FA50F31E0A51708F030E0432B6C0DFE
:1040800031E06C1508F030E0F42FF60F41E0F61740
:1040900008F040E0342B7B0D41E07B1508F040E058
:1040A000532F570F31E0571708F030E0432B820DA4
:1040B00031E0821508F030E0480F61E0481708F061
:1040C00060E0362B990D930F022F080D11E00217B7
:1040D00008F010E01B0F81E01B1708F080E0B82FFC
:1040E000BE0F71E0BE1708F070E07A0F61E07A173A
:1040F00008F060E06F0F31E06F1708F030E0350F27
:1041000021E0351708F020E0240F81E0241708F0A3
:1041100080E018014B2E572E662E732E822E982E7D
:10412000FEC0843091050CF4FCC020918820A09042
:10413000892070908A2080908B2030E040E050E011
:1041400060E070E080E090E008E10E940C72F22EE6
:10415000132FE42ED52EC62EB72E282E992E2A2DBB
:1041600030E040E050E060E070E080E090E000E1AE
:104170000E940C722F0DF1E02F1508F0F0E0310FC6
:10418000E1E0311708F0E0E0F30FA1E0F31708F0E9
:10419000A0E0EA2B4E0D31E04E1508F030E0E40FC0
:1041A000A1E0E41708F0A0E03A2B5D0D41E05D15B9
:1041B00008F040E0B32FB50F31E0B51708F030E05C
:1041C000432B6C0D31E06C1508F030E0A42FA60FE6
:1041D00041E0A61708F040E0342B7B0D41E07B1551
:1041E00008F040E0532F570F31E0571708F030E048
:1041F000432B820D31E0821508F030E0480F61E07A
:10420000481708F060E0362B990E930E122F180D08
:1042100081E0121708F080E0282E2F0E81E02F1683
:1042200008F080E0F82EFE0E81E0FE1608F080E037
:10423000E82EEB0E81E0EB1608F080E0D82EDA0EC7
:1042400081E0DA1608F080E0C82EC50E81E0C516C0
:1042500008F080E0B82EB40E81E0B41608F080E0DB
:10426000980E272D30E040E050E060E070E080E004
:1042700090E008E00E940C72210FE1E0211708F0A5
:10428000E0E0320DF1E0321508F0F0E0E30FA1E0DC
:10429000E31708F0A0E0FA2B4F0D31E04F1508F0BE
:1042A00030E0F40FA1E0F41708F0A0E03A2B5E0D27
:1042B00041E05E1508F040E0A32FA50F31E0A517FF
:1042C00008F030E0432B6D0D31E06D1508F030E063
:1042D000542F560F41E0561708F040E0342B7C0D68
:1042E00041E07C1508F040E0632F670F31E067176D
:1042F00008F030E0432B8B0D31E08B1508F030E0F7
:10430000480F71E0481708F070E0372B990D222E06
:104310003E2E4F2E5A2E652E762E842E932E990EDB
:1043200009C0AAE02A2E3324442455246624772485
:10433000882499240E949E0CB22DB33689F4E32D73
:10434000E23371F4F42DF93659F4552049F466201E
:1043500039F4772029F4882019F4992009F46AC5E2
:104360009101A201B301C401F3E6AF2EE2E3BE2E38
:1043700009E6C02EDD24EE24FF2400E010E00E94B8
:104380007D72823008F074C2822D853689F4932DB7
:10439000923771F4442061F4552051F4662041F4C1
:1043A000772031F4882021F4992011F40C94482FBF
:1043B0009101A201B301C40115E6A12EB2E7BB2E03
:1043C000CC24DD24EE24FF2400E010E00E947D7266
:1043D000823008F009C1A22DA53681F4B32DB43680
:1043E00069F4442059F4552049F4662039F47720C3
:1043F00029F4882019F4992009F4E9C69101A20151
:10440000B301C401A5E6AA2EF4E6BF2ECC24DD2418
:10441000EE24FF2400E010E00E947D72823008F05C
:1044200063C0E22DE53781F4332071F4442061F458
:10443000552051F4662041F4772031F4882021F48E
:10444000992011F40C944A2A9101A201B301C401EC
:10445000E5E7AE2EBB24CC24DD24EE24FF2400E0CF
:1044600010E00E947D72823010F5F22DF83611F0C6
:104470000C949333332011F00C949333442011F0B7
:104480000C949333552011F00C949333662011F063
:104490000C949333772011F00C949333882011F00F
:1044A0000C949333992011F00C949333AEC7822D62
:1044B000863779F4332069F4442059F4552049F4BF
:1044C000662039F4772029F4882019F4992009F41A
:1044D000F1C7922D943611F00C949333A32DA1368D
:1044E00011F00C9493337BC0B22DB73789F4E32DD0
:1044F000EF3671F4442061F4552051F4662041F404
:10450000772031F4882021F4992011F40C94D22DD5
:104510009101A201B301C40107E7A02E1FE6B12E4D
:10452000CC24DD24EE24FF2400E010E00E947D7204
:104530008230B8F5F22DF43681F4832D893669F492
:10454000442059F4552049F4662039F4772029F4A1
:10455000882019F4992009F473C7922D953611F02B
:104560000C949333A32DAE3611F00C949333442066
:1045700011F00C949333552011F00C949333662072
:1045800011F00C949333772011F00C94933388201E
:1045900011F00C949333992011F00C9493330C94F4
:1045A000302EB22DB13389F4E32DE03771F444207D
:1045B00061F4552051F4662041F4772031F48820CD
:1045C00021F4992011F40C94C12EF22DF33311F043
:1045D0000C949333832D813711F00C949333442042
:1045E00011F00C94933395C0922D983789F4A32D34
:1045F000A43671F4B42DB13659F4552049F466202F
:1046000039F4772029F4882019F4992009F40EC48C
:104610009101A201B301C401B8E7AB2EA4E6BA2E02
:10462000F1E6CF2EDD24EE24FF2400E010E00E940E
:104630007D72823008F083C0E22DE33789F4F32DD8
:10464000F23771F4442061F4552051F4662041F4AE
:10465000772031F4882021F4992011F40C9414303F
:104660009101A201B301C401E3E7AE2E02E7B02E2F
:10467000CC24DD24EE24FF2400E010E00E947D72B3
:10468000823020F5822D893611F00C949333932DCE
:10469000923711F00C949333442011F00C9493331F
:1046A000552011F00C949333662011F00C94933341
:1046B000772011F00C949333882011F00C949333ED
:1046C000992011F00C9493330C94C12FA22DA33791
:1046D00089F4B32DB33771F4442061F4552051F4BB
:1046E000662041F4772031F4882021F4992011F4D8
:1046F0000C942330E22DE33611F00C949333F32D18
:10470000F43611F00C949333842D813611F00C940F
:104710009333552011F00C949333662011F00C94D0
:104720009333772011F00C949333882011F00C947C
:104730009333992011F00C9493330C943932922DC9
:10474000923791F4A32DA23779F4B42DB53661F4E4
:10475000552051F4662041F4772031F4882021F46B
:10476000992011F40C94F52C9101A201B301C4011C
:1047700012E7A12EB2E7BB2EA5E6CA2EDD24EE2459
:10478000FF2400E010E00E947D728230C0F5E22D2F
:10479000E33789F4F32DF53671F4842D813659F41D
:1047A000552049F4662039F4772029F4882019F43B
:1047B000992009F48FC6922D923611F00C94933300
:1047C000A32DA53611F00C949333B42DB43611F00B
:1047D0000C949333552011F00C949333662011F010
:1047E0000C949333772011F00C949333882011F0BC
:1047F0000C949333992011F00C949333E8C4E22D78
:10480000E33689F4F32DFD3671F4842D883659F49E
:10481000552049F4662039F4772029F4882019F4CA
:10482000992009F40BC3922D9D3611F00C9493330B
:10483000A32DA53711F00C949333B42DB83611F095
:104840000C949333552011F00C949333662011F09F
:104850000C949333772011F00C949333882011F04B
:104860000C949333992011F00C9493330C944932A7
:10487000E22DE63391F4F32DF93679F4842D853762
:1048800061F4952D953649F4662039F4772029F4A2
:10489000882019F4992009F4BCC59101A201B30143
:1048A000C401F6E3AF2EE9E6BE2E05E7C02E15E6FD
:1048B000D12EEE24FF2400E010E00E947D728230B1
:1048C00008F04BC1A22DA13391F4B32DB13379F48B
:1048D000E42DE13761F4552051F4662041F477204E
:1048E00031F4882021F4992011F40C94582D910171
:1048F000A201B301C401B1E3AB2EA1E3BA2EF1E7EB
:10490000CF2EDD24EE24FF2400E010E00E947D7213
:10491000823008F085C0F22DF73691F4832D8F3662
:1049200079F4942D9C3661F4552051F4662041F4BD
:10493000772031F4882021F4992011F40C94A22CD2
:104940009101A201B301C401E7E6AE2E0FE6B02E3D
:104950001CE6C12EDD24EE24FF2400E010E00E94BE
:104960007D72823020F5A22DA43611F00C94933381
:10497000B32DB33611F00C949333E42DEC3611F0D3
:104980000C949333552011F00C949333662011F05E
:104990000C949333772011F00C949333882011F00A
:1049A0000C949333992011F00C949333C8C7F22DD3
:1049B000F53791F4832D833679F4942D9D3661F487
:1049C000552051F4662041F4772031F4882021F4F9
:1049D000992011F40C94582DA22DA03311F00C94B1
:1049E0009333B32DB13311F00C949333E42DE137AD
:1049F00011F00C949333552011F00C9493336620EE
:104A000011F00C949333772011F00C949333882099
:104A100011F00C949333992011F00C949333E5C763
:104A2000F22DF43791F4832D8F3679F4942D9F363F
:104A300061F4A52DA23649F4662039F4772029F4D3
:104A4000882019F4992009F4D1C59101A201B3017C
:104A5000C401B4E7AB2EAFE6BA2EFFE6CF2EE2E6F6
:104A6000DE2EEE24FF2400E010E00E947D728230F2
:104A7000D0F5B22DB03791F4E32DE53679F4F42D6D
:104A8000F23761F4552051F4662041F4772031F477
:104A9000882021F4992011F40C94482F822D84371A
:104AA00011F00C949333932D943611F00C949333AE
:104AB000A42DA73711F00C949333552011F00C94CA
:104AC0009333662011F00C949333772011F00C94FB
:104AD0009333882011F00C949333992011F00C94A7
:104AE00093330C942C33B22DB93691F4E32DEC367C
:104AF00079F4F42DF13661F4852D833649F466207E
:104B000039F4772029F4882019F4992009F4C3C1D5
:104B1000922D9E3611F00C949333A32DA13611F0F3
:104B20000C949333B42DB83611F00C949333E52DD7
:104B3000E33611F00C949333662011F00C94933308
:104B4000772011F00C949333882011F00C94933358
:104B5000992011F00C9493331EC5F22DF33799F47C
:104B6000832D823781F4942D973769F4A52DA037D2
:104B700051F4662041F4772031F4882021F4992003
:104B800011F40C940E2F9101A201B301C40103E7AB
:104B9000A02E12E7B12EB7E7CB2EA0E7DA2EEE2437
:104BA000FF2400E010E00E947D72823008F09FC078
:104BB000B22DB03799F4E32DED3681F4F42DF537AD
:104BC00069F4852D883651F4662041F4772031F45C
:104BD000882021F4992011F40C94F82D9101A20160
:104BE000B301C401F0E7AF2EEDE6BE2E05E7C02EFF
:104BF00018E6D12EEE24FF2400E010E00E947D7222
:104C00008230D0F5922D903791F4A32DAC3679F403
:104C1000B42DB53661F4E52DE83649F4662039F453
:104C2000772029F4882019F4992009F4EEC3F22D95
:104C3000F13611F00C949333832D8D3611F00C94D2
:104C40009333942D953711F00C949333A52DA836FA
:104C500011F00C949333662011F00C949333772069
:104C600011F00C949333882011F00C949333992015
:104C700011F00C949333ABC7B22DB33799F4E32DF5
:104C8000E53681F4F42DF23769F4852D803751F43F
:104C9000662041F4772031F4882021F4992011F422
:104CA0000C949432922D913311F00C949333A32DE4
:104CB000A23711F00C949333B42DB73711F00C9444
:104CC0009333E52DE03711F00C949333662011F007
:104CD0000C949333772011F00C949333882011F0C7
:104CE0000C949333992011F00C949333ABC0F22DB4
:104CF000F73791F4832D803779F4942D983761F448
:104D0000A52DA43749F4662039F4772029F48820AA
:104D100019F4992009F419C49101A201B301C40145
:104D2000B7E7AB2EA0E7BA2EF8E7CF2EE4E7DE2EEA
:104D3000EE24FF2400E010E00E947D728230D8F55E
:104D4000B22DB43799F4E32DE33781F4F42DF53621
:104D500069F4852D823751F4662041F4772031F4CF
:104D6000882021F4992011F40C94BE2E922D9437B2
:104D700011F00C949333A32DA33711F00C949333BB
:104D8000B42DB53611F00C949333E52DE43711F0C2
:104D90000C949333662011F00C949333772011F028
:104DA0000C949333882011F00C949333992011F0D4
:104DB0000C9493331FC4F22DF23791F4832D873670
:104DC00079F4942D903761F4A52DA53749F4662028
:104DD00039F4772029F4882019F4992009F47EC544
:104DE000B22DBC3611F00C949333E32DE13611F063
:104DF0000C949333F42DF43711F00C949333852DE8
:104E0000883711F00C949333662011F00C9493338F
:104E1000772011F00C949333882011F00C94933385
:104E2000992011F00C9493330C94F0320E940416E4
:104E30000C9495330E9469100C9495330E948D1642
:104E40000C9495336091B6047091B70480E090E0C3
:104E50000E94527D8C016CEF72E00E94677D00978A
:104E600019F477980C949533C8016FEF72E00E94A3
:104E7000677D009719F4779A0C949533779903C05E
:104E80008CEF92E002C08FEF92E000D000D021E6DC
:104E900035E00C9482336091B6047091B70480E0E1
:104EA00090E00E94527D8C0166E173E00E94677D74
:104EB000009709F052C06091B6047091B70480E089
:104EC00090E00E94527D8C01009711F40C94953370
:104ED00069E173E00E94677D009729F482E29FEF09
:104EE000ACECBBE30BC0C8016FE173E00E94677DCF
:104EF000009789F482E29FEFACECBAE38093A904B7
:104F00009093AA04A093AB04B093AC0489EA94E014
:104F100066E070E0DCC0C8010E94457C7B018C012A
:104F200020E030E0A9010E943677882391F081E0EB
:104F30000E943D0B9B01AC01C801B7010E943A776A
:104F40006093A9047093AA048093AB049093AC047B
:104F5000DDCF00D081EA95E08CC0C80164E273E047
:104F60000E94677D009709F052C06091B60470916D
:104F7000B70480E090E00E94527D8C01009711F40C
:104F80000C94953369E173E00E94677D009729F4E2
:104F900082E29FEFACECBBE30BC0C8016FE173E0B2
:104FA0000E94677D009769F482E29FEFACECBAE360
:104FB0008093AD049093AE04A093AF04B093B0047B
:104FC0001DC0C8010E94457C7B018C0120E030E0BF
:104FD000A9010E9436778823B1F082E00E943D0B40
:104FE0009B01AC01C801B7010E943A776093AD0400
:104FF0007093AE048093AF049093B0048DEA94E074
:105000006AE070E064C000D084E995E066C0C80141
:1050100067E273E00E94677D009709F06AC06091C3
:10502000B6047091B70480E090E00E94527D8C013C
:10503000009711F40C94953369E173E00E94677D49
:10504000009769F487ED94E3AFEEBCE38093A50489
:105050009093A604A093A704B093A80434C0C801F9
:105060006FE173E00E94677D009741F400D085E80E
:1050700095E0EDB7FEB79283818335C0C8010E94E9
:10508000457C1B012C0120E030E0A9010E9436770D
:10509000882301F180E00E943D0B7B018C01C2015D
:1050A000B10121EE3AE744E95EE30E946F76A80180
:1050B00097010E943A776093A5047093A6048093A9
:1050C000A7049093A80485EA94E062E070E044E0CD
:1050D00050E01EC200D088E795E0ADB7BEB712968B
:1050E0009C938E9311970E94E87D0F900F900C94E3
:1050F00095330E948B0B00D000D000D021E735E023
:10510000EDB7FEB732832183ADB7BEB713966D936B
:105110007D938D939C9316970E94E87DEDB7FEB723
:1051200036960FB6F894FEBF0FBEEDBF81E00E9429
:105130003D0B2091A9043091AA044091AB045091F9
:10514000AC040E9480787B018C0182E00E943D0BC0
:105150009B01AC018DB79EB70A970FB6F8949EBF1E
:105160000FBE8DBFCDB6DEB60894C11CD11C85E63E
:1051700095E0ADB7BEB712969C938E9311978E2D86
:105180009F2DA02FB12FF60182839383A483B58333
:10519000CA01B9012091AD043091AE044091AF0431
:1051A0005091B0040E948078D60116966D937D933D
:1051B0008D939C9319970E94E87DEDB7FEB73A96C0
:1051C0000FB6F894FEBF0FBEEDBF0C94293360916B
:1051D000B6047091B70480E090E00E94527D009781
:1051E00061F160E070E040E150E00E94377B209187
:1051F000E4063091E5062617370799F17093E50626
:105200006093E40684EE96E060E070E042E050E0F7
:105210000E94387F8091E4069091E50600D000D08E
:1052200021E535E0ADB7BEB712963C932E931197AA
:1052300014969C938E9313970EC08091E4069091E0
:10524000E50600D000D02DE335E0EDB7FEB73283A0
:105250002183948383830E94E87D0F900F900F90A9
:105260000F900E949E0C00D000D080E395E0ADB777
:10527000BEB712969C938E93119781E090E014969E
:105280009C938E9313970E94E87D85E295E0EDB79D
:10529000FEB79283818382E090E0948383830E94AF
:1052A000E87D8AE195E0ADB7BEB712969C938E93E8
:1052B000119784E090E014969C938E9313970E942C
:1052C000E87D8DE095E0EDB7FEB79283818388E0BD
:1052D00090E0948383830E94E87D82E095E0ADB7FF
:1052E000BEB712969C938E93119780E190E014962E
:1052F0009C938E9313970E94E87D86EF94E0EDB720
:10530000FEB79283818380E290E0948383830E943E
:10531000E87D88EE94E0ADB7BEB712969C938E936D
:10532000119780E490E014969C938E9313970E94BB
:10533000E87D8AED94E0EDB7FEB79283818380E843
:1053400090E0948383830E94E87D8BEC94E0ADB77A
:10535000BEB712969C938E93119780E091E01496BD
:105360009C938E9313970E94E87D8CEB94E0EDB7AD
:10537000FEB79283818380E092E0948383830E94CE
:10538000E87D80EB94E0ADB7BEB712969C938E9308
:10539000119780E094E014969C938E9313970E944B
:1053A000E87D82EA94E0EDB7FEB79283818380E0E6
:1053B00098E0948383830E94E87D85E994E0ADB70B
:1053C000BEB712969C938E93119780E090E114964D
:1053D0009C938E9313970E94E87D87E894E0EDB745
:1053E000FEB79283818380E090E2948383830E945E
:1053F000E87D87E794E0ADB7BEB712969C938E9395
:10540000119780E090E40C9488330E9411190C9459
:10541000953380918C20843329F480E061E040E072
:105420000E94A9112091B104222311F40C94953308
:1054300000D000D0EDB7FEB7319684E794E020C0ED
:105440006091B6047091B70480E090E00E94527DB4
:1054500069E173E00E94677D009711F481E001C06B
:1054600080E00E94541B2091B104222311F40C947B
:10547000953300D000D0EDB7FEB7319681E794E0C8
:10548000ADB7BEB712969C938E9311972283138269
:105490000C948C330E94021A2091B104222311F43F
:1054A0000C94953300D000D0EDB7FEB731968EE660
:1054B00094E0E6CF0E94FD192091B104222311F45B
:1054C0000C94953300D000D0EDB7FEB731968BE643
:1054D00094E0D6CF6091B6047091B70480E090E07C
:1054E0000E94527D8C016CEF72E00E94677D0097F4
:1054F00099F48091CE049091CF0484609093CF046E
:105500008093CE048EEC94E064E170E042E050E0E1
:105510000E94387F0C949533C8016FEF72E00E94AF
:10552000677D4091CE045091CF04009711F44B7FDA
:1055300080C342FF03C08CEF92E002C08FEF92E085
:1055400000D000D02EEA35E084C36091B60470919B
:10555000B70480E090E00E94527D0E94497C803137
:1055600050F48093E90690E00E94185789EE96E087
:1055700066E170E027C000D000D0EDB7FEB73196ED
:1055800082EB95E0ADB7BEB712969C938E931197C0
:105590008091E90629C06091B6047091B70480E05B
:1055A00090E00E94527D0E94497C982F9B50903140
:1055B00060F48093D00490E00E94905580ED94E0D8
:1055C00067E170E041E050E0A3CF00D000D0EDB73C
:1055D000FEB731968FEB95E0ADB7BEB712969C93B0
:1055E0008E9311978091D004828351CF0C94000048
:1055F0000C9495336091B6047091B70480E090E00C
:105600000E94527D8C016CE273E00E94677D0097DE
:1056100039F4219A8091CE049091CF0480616ECFAD
:10562000C8016EE273E00E94677D009739F4229A08
:105630008091CE049091CF04806260CFC80160E376
:1056400073E00E94677D009739F4239A8091CE041D
:105650009091CF04806452CFC80162E373E00E944E
:10566000677D009739F4239A8091CE049091CF04FE
:10567000806844CFC80164E373E00E94677D0097AF
:10568000D1F48091CE049091CF0491609093CF0497
:105690008093CE048EEC94E064E170E042E050E050
:1056A0000E94387F81E195E062E140E050E00E9495
:1056B000B0400C949533C80166E373E00E94677DA7
:1056C000009771F4E3EBF7E111921192B7E1E33D3A
:1056D000FB07D1F78091CE049091CF0492600ECF5A
:1056E000C8016FEF72E00E94677D4091CE04509137
:1056F000CF040097B1F44F705C7F5093CF04409378
:10570000CE042B9A8EEC94E064E170E042E050E02D
:105710000E94387F8091D42490E00E94A5550C947B
:10572000953344FF03C08CEF92E002C08FEF92E00C
:1057300000D000D02FEF35E0EDB7FEB732832183E4
:10574000948383830E94E87D8091CE040F900F9014
:105750000F900F9085FF03C08CEF92E002C08FEF97
:1057600092E000D000D024EF35E0ADB7BEB712967E
:105770003C932E93119714969C938E9313970E94AB
:10578000E87D8091CE040F900F900F900F9086FFD0
:1057900003C08CEF92E002C08FEF92E000D000D007
:1057A00029EE35E0EDB7FEB73283218394838383FE
:1057B0000E94E87D8091CE040F900F900F900F9083
:1057C00087FF03C08CEF92E002C08FEF92E000D021
:1057D00000D02EED35E0ADB7BEB712963C932E93B8
:1057E000119714969C938E9313970E94E87D809155
:1057F000CE049091CF040F900F900F900F9090FFD8
:1058000003C08CEF92E002C08FEF92E000D000D096
:1058100023ED35E0EDB7FEB7328321839483838394
:105820000E94E87D8091CE049091CF040F900F905C
:105830000F900F9091FF03C08CEF92E002C08FEFAA
:1058400092E000D000D028EC35E0ADB7BEB712969C
:105850003C932E93119714969C938E9313970E94CA
:10586000E87D8091CE049091CF040F900F900F901F
:105870000F9091FF5AC788E393E00E940F7E03EBDD
:1058800017E18BE0C82ED12CB0E4EB2EB3E0FB2E59
:10589000F801819191918F0100D000D000D0EDB737
:1058A000FEB73196ADB7BEB71296FC92EE92119745
:1058B000D382C282958384830E94D67D0894C11CC2
:1058C000D11CEDB7FEB736960FB6F894FEBF0FBEEB
:1058D000EDBFFBE1CF16D104D9F627C700D087E68C
:1058E00094E0ADB7BEB712969C938E9311970E9429
:1058F000E87D2091B1040F900F902223A9F000D0F1
:1059000000D0EDB7FEB7319684E694E0ADB7BEB7F0
:1059100012969C938E931197228313820E94E87DA6
:105920000F900F900F900F9088E10FB6F89480932E
:105930006000109260000FBE0C94007CF6C60E94BE
:10594000C24DF3C66091B6047091B70480E090E058
:105950000E94527D1C016CEF72E00E94677D0097EF
:1059600049F40E946F548091CE049091CF048160DD
:105970008D7FC4CDC1016FEF72E00E94677D0097FB
:1059800041F40E94D1538091CE049091CF048C7F3A
:10599000B5CD0BE413E0C101B8010E94677D00970B
:1059A00049F40E94D1538091CE049091CF048E7F10
:1059B0008260A4CD8091CE0481FF0BC000D000D0C6
:1059C0008EE096E0EDB7FEB7928381831483038364
:1059D000A3C680FF03C08CEF92E002C08FEF92E07D
:1059E00000D000D02AE036E08DC600D08AE394E0F3
:1059F000EDB7FEB7928381830E94E87D8DB79EB795
:105A000040970FB6F8949EBF0FBE8DBFEDB7FEB79F
:105A100031968CE194E0ADB7BEB712969C938E930D
:105A200011978091832090918420A0918520B0913E
:105A3000862082839383A483B5838091772090917D
:105A40007820A0917920B0917A2086839783A087CF
:105A5000B18780917B2090917C20A0917D20B09196
:105A60007E2082879387A487B58780917F2090913D
:105A70008020A0918120B091822086879787A08B7B
:105A8000B18B0E94E87D2091B104EDB7FEB772960C
:105A90000FB6F894FEBF0FBEEDBF222309F445C632
:105AA00000D000D0EDB7FEB7319689E194E0E8CCA4
:105AB000F89481E090E00E94AF08182F80E090E019
:105AC0000E94AF08082F7894F89483E090E00E9439
:105AD000AF08F82E82E090E00E94AF08E82E78949C
:105AE00000D000D000D02FE034E0EDB7FEB7328315
:105AF0002183209124183091251840912618509127
:105B00002718ADB7BEB713962D933D934D935C9375
:105B100016970E94E87D00D000D0EDB7FEB7319611
:105B200028EE33E0ADB7BEB712963C932E93119793
:105B3000E2821382F482158206831782108711860F
:105B40000E94E87DEDB7FEB73A960FB6F894FEBF17
:105B50000FBEEDBF0E94A51A2091660000D000D0B4
:105B6000EDB7FEB731968CED93E0ADB7BEB71296A8
:105B70009C938E931197228313820E94E87D0F904D
:105B80000F900F900F900E949E0C2091B104222341
:105B900009F4CBC500D000D0EDB7FEB7319689ED42
:105BA00093E06ECC80E090E00E94AA0C81E090E04F
:105BB0000E94AA0C2091B104222309F4B6C500D09A
:105BC00000D0EDB7FEB7319686ED93E059CC0E9438
:105BD00080180E949E0C2091B104222309F4A5C5CF
:105BE00000D000D0EDB7FEB7319683ED93E048CCFE
:105BF0006091B6047091B70480E090E00E94527DFD
:105C00008C016CEF72E00E94677D009731F4809107
:105C1000CE049091CF04886071CCC8016FEF72E020
:105C20000E94677D4091CE045091CF04009731F4DB
:105C3000477F5093CF044093CE0464CC43FF03C00E
:105C40008CEF92E002C08FEF92E000D000D022E112
:105C500036E0EDB7FEB732832183948383835CC53E
:105C60006091B6047091B70480E090E00E94527D8C
:105C700060E573E00E94677D009741F5F89489E044
:105C800097E00E94A7410CC0C8010D960E94F34402
:105C90008EE595E0B8010E946141C8010E946D4205
:105CA000082F192F0115110579F704C089E097E035
:105CB0000E94E84189E097E00E944D420097B1F7C9
:105CC00089E097E00E94A34178944BC089E097E077
:105CD0000E94A741482F592F7A0106E513E03DC0E5
:105CE0008DB79EB70C970FB6F8949EBF0FBE8DBFB1
:105CF000EDB7FEB73196ADB7BEB712961C930E93B3
:105D00001197D70112968C91129782831382139662
:105D10008C9113978483158218968C91189786839B
:105D2000178214968D919C9115979187808716966E
:105D30008D919C911797938782870E94D67DEDB7AE
:105D4000FEB73C960FB6F894FEBF0FBEEDBFC7017D
:105D50000E946D42482F592F7A01E114F10409F095
:105D6000BFCF2091B104222309F4DFC400D000D0BA
:105D7000EDB7FEB7319680ED93E082CB0E948E1B8B
:105D8000D4C46091B6047091B70480E090E00E94A2
:105D9000527D8C016CEF72E00E94677D009751F498
:105DA0008091CE049091CF0498609093CF0480931B
:105DB000CE0410C0C8016FEF72E00E94677D409171
:105DC000CE045091CF04009771F4577F5093CF04C5
:105DD0004093CE048EEC94E064E170E042E050E049
:105DE0000E94387F17C053FF03C08CEF92E002C0BF
:105DF0008FEF92E000D000D026E136E0EDB7FEB79D
:105E000032832183948383830E94E87D0F900F90D7
:105E10000F900F9081E00E94AD0A87C46091B60494
:105E20007091B70480E090E00E94527D8C016EE09A
:105E300073E00E94677D009731F48091CE049091C9
:105E4000CF049B7F5BCBC80163E073E00E94677D5A
:105E50004091CE045091CF04009711F45460E9CEE4
:105E600052FF03C083E093E002C08EE093E000D0D5
:105E700000D02DE733E0ADB7BEB712963C932E931A
:105E8000119714969C938E9313970E94D67D46C4C7
:105E90006091B6047091B70480E090E00E94527D5A
:105EA0000097A9F160E070E040E150E00E94377B8C
:105EB0006093C8047093C9048093CA049093CB0480
:105EC00000D000D000D02DEB33E0EDB7FEB7328329
:105ED0002183ADB7BEB713966D937D938D939C933D
:105EE00016970E94E87DEDB7FEB736960FB6F89488
:105EF000FEBF0FBEEDBF88EC94E06EE070E044E0C2
:105F000050E00E94387F81E00E943C1C0EC480E07B
:105F10000E943C1C0E949E0C00D000D000D088EA59
:105F200093E0ADB7BEB712969C938E931197809174
:105F3000C8049091C904A091CA04B091CB04EDB7F4
:105F4000FEB783839483A583B6830E94E87D8DB7D3
:105F50009EB706960FB6F8949EBF0FBE8DBF81E028
:105F60000E943C1C0E949E0C2091B104222309F443
:105F7000DCC300D000D0EDB7FEB7319685EA93E0E0
:105F80007FCA6091B6047091B70480E090E00E94EF
:105F9000527D009741F160E070E04AE050E00E94DD
:105FA000377B7093CD046093CC0400D000D0EDB764
:105FB000FEB7319628E833E0ADB7BEB712963C93F2
:105FC0002E931197738362830E94E87D0F900F9048
:105FD0000F900F908CEC94E062E170E042E050E0B2
:105FE0000E94387F14C000D000D087E693E0EDB760
:105FF000FEB7928381838091CC049091CD049483E9
:1060000083830E94E87D0F900F900F900F90209156
:10601000B104222309F489C300D000D0EDB7FEB744
:10602000319684E693E02CCA0E9430452091B10459
:10603000222309F47AC300D000D0EDB7FEB7319621
:1060400081E693E01DCA00D081E593E0EDB7FEB78D
:10605000928381830E94E87D0F900F900E94FD192A
:1060600000D08DE493E0ADB7BEB712969C938E93AB
:1060700011970E94E87D0F900F9080E00E94541BC2
:1060800000D087E493E0EDB7FEB7928381830E944E
:10609000E87D0F900F900E9469108091711C80FF25
:1060A00005C081E061E041E00E94A9110E94021A4E
:1060B00000D000D0EDB7FEB731968EE393E0ADB7D8
:1060C000BEB712969C938E9311978091D0048283D1
:1060D00013820E94E87DEDB7FEB7319681E393E02D
:1060E000ADB7BEB712969C938E9311978091E90637
:1060F000828313820E94E87D89E193E0EDB7FEB7C9
:106100009283818380E490E0948383830E94E87D7E
:1061100000D0EDB7FEB7319686E093E0ADB7BEB7DD
:1061200012969C938E9311978091ED248283138213
:106130008091EE24848315820E94E87D0F900F9059
:1061400081EF92E0EDB7FEB7928381838091CC041A
:106150009091CD04948383830E94E87D00D08DEDDF
:1061600092E0ADB7BEB712969C938E931197809133
:10617000C8049091C904A091CA04B091CB04EDB7B2
:10618000FEB783839483A583B6830E94E87D8DB791
:106190009EB706960FB6F8949EBF0FBE8DBF81E0E6
:1061A0000E943C1C0E948B0B00D000D000D020ED40
:1061B00032E0ADB7BEB712963C932E931197EDB770
:1061C000FEB763837483858396830E94E87D8DB7D1
:1061D0009EB706960FB6F8949EBF0FBE8DBF0E9465
:1061E000C20B0E949F0B00D000D000D022EC32E006
:1061F000ADB7BEB712963C932E931197EDB7FEB78D
:1062000063837483858396830E94E87D8DB79EB7F0
:1062100006960FB6F8949EBF0FBE8DBF1D9B03C0A0
:1062200083E193E002C08FEF92E000D000D026EB34
:1062300032E0ADB7BEB712963C932E9311971496E9
:106240009C938E9313970E94E87D2091C8243091EF
:10625000C9244091CA245091CB248091CC249091A0
:10626000CD24A091CE24B091CF2400D000D000D076
:106270000DB71EB70F5F1F4F68E972E0EDB7FEB7AD
:1062800072836183F8012283338344835583868339
:106290009783A087B1870E94E87DEDB7FEB731965E
:1062A00086E792E0ADB7BEB712969C938E93119796
:1062B0008091D5249091D624A091D724B091D82450
:1062C00082839383A483B5838091D9249091DA2427
:1062D000A091DB24B091DC2486839783A087B187CB
:1062E0000E94E87DEDB7FEB738960FB6F894FEBF72
:1062F0000FBEEDBF8CE692E0928381830E94E87D21
:106300008091CE040F900F9081FF0EC000D086E6E2
:1063100092E0ADB7BEB712969C938E9311970E94F0
:10632000E87D0F900F9017C080FF03C08CEF92E0C4
:1063300002C08FEF92E000D000D022E632E0EDB74D
:10634000FEB732832183948383830E94E87D0F907C
:106350000F900F900F908091CE0483FF03C08CEFBD
:1063600092E002C08FEF92E000D000D02FE432E044
:10637000ADB7BEB712963C932E93119714969C938B
:106380008E9313970E94E87D8091CE049091CF0464
:106390000F900F900F900F9093FF03C08CEF92E03F
:1063A00002C08FEF92E000D000D022E432E0EDB7DF
:1063B000FEB732832183948383830E94E87D80919A
:1063C000E4069091E50625E332E0ADB7BEB712963C
:1063D0003C932E93119714969C938E9313970E943F
:1063E000E87D0F900F900F900F90779903C08CEF7E
:1063F00092E002C08FEF92E000D000D02CE232E0B9
:10640000EDB7FEB732832183948383830E94E87DB6
:106410008091CE049091CF040F900F900F900F9029
:1064200092FF03C083E093E002C08EE093E000D0CF
:1064300000D02DE733E0ADB7BEB712963C932E9354
:10644000119714969C938E9313970E94D67D20915A
:10645000B1040F900F900F900F90222309F465C1A3
:1064600000D000D0EDB7FEB7319689E292E00C94EF
:10647000402A0E94CA1A2091B104222309F455C16E
:1064800000D000D0EDB7FEB7319686E292E00C94D2
:10649000402A0E94C6170097B9F500D000D000D05E
:1064A0008BE192E0EDB7FEB79283818380916D1806
:1064B00090916E18A0916F18B09170188383948397
:1064C000A583B6830E94E87D8EE092E0ADB7BEB7AB
:1064D00012969C938E9311978091E9249091EA24CF
:1064E000A091EB24B091EC24EDB7FEB783839483A5
:1064F000A583B6830E94E87D8DB79EB706960FB63A
:10650000F8949EBF0FBE8DBF0E949E0C2091B104D7
:10651000222309F40AC100D000D0EDB7FEB73196AE
:106520008BE092E00C94402A83E061E048E021E0B7
:106530000E94431300D000D000D084E092E0EDB779
:10654000FEB7928381838091601890916118A09129
:106550006218B091631883839483A583B6830E94E5
:10656000E87D00D000D0EDB7FEB7319683EF91E023
:10657000ADB7BEB712969C938E9311978091641815
:1065800090916518A0916618B091671882839383E3
:10659000A483B5838091681890916918A0916A18B6
:1065A000B0916B1886839783A087B1870E94E87D9E
:1065B000EDB7FEB73A960FB6F894FEBF0FBEEDBF2B
:1065C0000E949E0C2091B104222309F4AEC000D099
:1065D00000D0EDB7FEB7319680EF91E00C94402AE1
:1065E0006091B6047091B70480E090E00E94527D03
:1065F00066E873E00E94677D0097B1F46091B6048D
:106600007091B70480E090E00E94527D009709F4F9
:106610008CC00E94497C803108F087C09091520163
:10662000982B9093520181C08091520100D000D0EC
:106630002AE136E0EDB7FEB73283218390E08F7018
:106640009070948383830E94E87D0F900F900F9049
:106650000F900E949E0C69C06091B6047091B704BF
:1066600080E090E00E94527D8C016CEF72E00E940D
:10667000677D009749F40E94B3528091CE049091B7
:10668000CF0490610C947E2AC8016FEF72E00E94E3
:10669000677D0097E9F4F8940E94C15288E10FB633
:1066A000F89480936000109260000FBE84B7877FDB
:1066B00084BF8091600088618093600010926000C8
:1066C00078948091CE049091CF049F7E0C947E2A82
:1066D000C8016BE873E00E94677D4091CE04509141
:1066E000CF04009721F454FF20C0F894FFCF54FF4B
:1066F00003C08CEF92E002C08FEF92E000D000D098
:1067000027E236E0ADB7BEB712963C932E931197B1
:1067100014969C938E9313970E94E87D0F900F9090
:106720000F900F9002C00E94EA18E981FA8111824D
:10673000108283E00F900F90CF91DF911F910F9106
:10674000FF90EF90DF90CF90BF90AF909F908F9091
:106750007F906F905F904F903F902F900895F894A6
:1067600091E2E0E0F0E0909357008491E2E0F0E005
:10677000909357002491E4E0F0E090935700E49167
:1067800090E0A0E0B0E0DC019927882730E040E00D
:1067900050E0542F432F322F2227820F931FA41F24
:1067A000B51F8E0F911DA11DB11D809324189093CC
:1067B0002518A0932618B093271878940895DF938E
:1067C000CF93CDB7DEB727970FB6F894DEBF0FBED5
:1067D000CDBFCE0104966EE070E044E050E00E9430
:1067E0001A7F8C819D81AE81BF818F3F2FEF9207F1
:1067F0002FEFA2072FEFB20749F488EC94E06EE088
:1068000070E044E050E00E94387F08C08093C804E4
:106810009093C904A093CA04B093CB04CE0102960E
:1068200062E170E042E050E00E941A7F8A819B8121
:106830002FEF8F3F920779F48CE390E09093CD0493
:106840008093CC048CEC94E062E170E042E050E094
:106850000E94387F04C09093CD048093CC04CE0175
:10686000029664E170E042E050E00E941A7F8A8163
:106870009B812FEF8F3F920779F48AE090E090930D
:10688000CF048093CE048EEC94E064E170E042E0AB
:1068900050E00E94387F04C09093CF048093CE04D0
:1068A000CE01029660E070E042E050E00E941A7F64
:1068B0008A819B812FEF8F3F920769F41092E50642
:1068C0001092E40684EE96E060E070E042E050E072
:1068D0000E94387F04C09093E5068093E4068DED16
:1068E00094E268E170E049E050E00E941A7F0E9463
:1068F0000D0ECE01049666E070E044E050E00E9488
:106900001A7F8C819D81AE81BF818F3F2FEF9207CF
:106910002FEFA2072FEFB20749F489EA94E066E06F
:1069200070E044E050E00E94387F08C089EA94E0BB
:1069300066E070E044E050E00E941A7FCE010496C9
:106940006AE070E044E050E00E941A7F8C819D81F3
:10695000AE81BF818F3F2FEF92072FEFA2072FEF5E
:10696000B20749F48DEA94E06AE070E044E050E058
:106970000E94387F08C08DEA94E06AE070E044E04D
:1069800050E00E941A7FCE01049662E070E044E07D
:1069900050E00E941A7F8C819D81AE81BF818F3F24
:1069A0002FEF92072FEFA2072FEFB20749F485EAE6
:1069B00094E062E070E044E050E00E94387F08C05C
:1069C00085EA94E062E070E044E050E00E941A7FC3
:1069D000CE01019666E170E041E050E00E941A7F2E
:1069E00089818F3F49F489EE96E066E170E041E0ED
:1069F00050E00E94387F08C089EE96E066E170E0C2
:106A000041E050E00E941A7FCE01019667E170E0FC
:106A100041E050E00E941A7F89818F3F49F480ED68
:106A200094E067E170E041E050E00E94387F08C0E8
:106A300080ED94E067E170E041E050E00E941A7F51
:106A400027960FB6F894DEBF0FBECDBFCF91DF9172
:106A500008950E94A7526C9A6B9A6A9A6F9A729ADA
:106A6000749A739A779A809880B3897F80BB839851
:106A7000849887E080937E00549A0E94AF330E94EE
:106A8000DF3381E00E94AD0A80E090E00E94210E99
:106A90000E94304C8091CE0486FD239A0895CF93B6
:106AA000DF93EC0188819981009731F02AE08938E1
:106AB000920709F099C08FC00E9429358091CE04B9
:106AC00080FD06C081FF02C01D9902C00E94D15303
:106AD000809170008C7F809370008091B6008062FE
:106AE0008093B6001092B20082E08093B100809152
:106AF000B60090E0877090700097C9F780917000A1
:106B000081608093700080E090E066EB78E00E9406
:106B10008A520E94FD1980E00E94541B00D08AEE28
:106B200091E0ADB7BEB712969C938E9311970E94D9
:106B3000E87D0F900F900E9469108091711C86FF74
:106B400002C00E946D4D8091E90690E00E941857A6
:106B50008091D00490E00E9490550E948D558093C2
:106B600017078091D00490E00E94905500D000D08B
:106B700000D0EDB7FEB7319680E993E0ADB7BEB770
:106B800012969C938E93119780911707828313829C
:106B90008091E906848315820E94D67D10921607A3
:106BA00010921507EDB7FEB736960FB6F894FEBFF4
:106BB0000FBEEDBF8DED94E09093E7248093E62423
:106BC00083E290E090930E0780930D0789E89AE0A6
:106BD000998388830DC0633259F485E197E060E0C2
:106BE00070E00E94951FE6CF1982188283E001C0F1
:106BF00081E0DF91CF9108958536910564F1209170
:106C0000E4063091E50620FF10C000D000D022EA53
:106C100033E0EDB7FEB732832183948383830E94F0
:106C2000D67D0F900F900F900F90809183209091C0
:106C30008420A0918520B09186200196A11DB11DD0
:106C40008093832090938420A0938520B093862006
:106C500021E030E002C020E030E0C90108954F9209
:106C60005F926F927F928F929F92AF92BF92CF92DC
:106C7000DF92EF92FF920F931F93DF93CF93CDB7E5
:106C8000DEB7CB58D0400FB6F894DEBF0FBECDBFF5
:106C90002C01633871F485EF96E0C557DF4F6883A8
:106CA000CB58D0400E94E73EC557DF4F6881CB5894
:106CB000D040D2012D913C911197BAE02C333B0783
:106CC00009F4A6C7EAE02D333E0748F42115310543
:106CD00089F0F9E02C333F0709F0E6C716C04AE017
:106CE0002D34340709F4BAC75AE02435350709F0C2
:106CF000DBC7CCC785EF96E061E870E04AE555E078
:106D00000E94CC3E8CE399E07EC7623109F0D2C785
:106D10008091CE049091CF0491FDF4CF8091C8046E
:106D20009091C904A091CA04B091CB0497FD8C9AAC
:106D30000E94C20B8091C8049091C904A091CA041A
:106D4000B091CB0493FF02C00E94C6178091C80483
:106D50009091C904A091CA04B091CB0494FF0AC0D9
:106D60000E948B0B6093D0247093D1248093D22403
:106D70009093D3248091C80480FF5DC062E1C62E49
:106D8000D12CCC0EDD1E00D000D000D0EDB7FEB768
:106D90003196ADB7BEB71296DC92CE92119788E7C6
:106DA00090E09383828386EB93E0958384830E94B3
:106DB000467E082F192F5DEDE52E54E2F52EEDB736
:106DC000FEB736960FB6F894FEBF0FBEEDBF48E78C
:106DD000A42EB12C3FE8832E32E0932ED7012D91C3
:106DE0007D01EDB7FEB738970FB6F894FEBF0FBE22
:106DF000EDBF3196C601800F911FADB7BEB7129699
:106E00009C938E931197B382A2829582848226836B
:106E100017820E94467E080F191FEDB7FEB73896FD
:106E20000FB6F894FEBF0FBEEDBFF5EEEF16F4E21D
:106E3000FF06A1F602C000E010E08091C80481FFC7
:106E40006EC022E1C22ED12CCC0EDD1E00D000D0AF
:106E500000D0EDB7FEB73196C601800F911FADB7D8
:106E6000BEB712969C938E93119788E790E0938318
:106E700082838AEB93E0958384830E94467E080F89
:106E8000191F7E010894E11CF11C80E1F7011192A9
:106E90008A95E9F72DB73EB72A5F3F4F0FB6F894B2
:106EA0003EBF0FBE2DBF80EB68E9A70128E00E941E
:106EB000611199E0A92EB12CAC0EBD1E88E7882E79
:106EC000912CBFE86B2EB2E07B2ED7012D917D0176
:106ED000EDB7FEB738970FB6F894FEBF0FBEEDBF03
:106EE0003196C601800F911FADB7BEB712969C9325
:106EF0008E93119793828282758264822683178291
:106F00000E94467E080F191FEDB7FEB738960FB6E0
:106F1000F894FEBF0FBEEDBFEA14FB04B1F68091FA
:106F2000C8049091C904A091CA04B091CB04009701
:106F3000A105B10581F12DB73EB7285030400FB6FD
:106F4000F8943EBF0FBE2DBFEDB7FEB73196CE0110
:106F50004296800F911FADB7BEB712969C938E9349
:106F6000119788E790E0938382838FEB93E095837A
:106F700084838091E7069091E806978386830E9438
:106F8000467E080F191FEDB7FEB738960FB6F89476
:106F9000FEBF0FBEEDBF8091C80482FF50C089E2E2
:106FA00090E06BE270E04AE250E027E00E94464940
:106FB0008DED94E20E94B64B2DB73EB72A5030407B
:106FC0000FB6F8943EBF0FBE2DBFEDB6FEB60894C7
:106FD000E11CF11C9E012E5E3F4F200F311FADB70B
:106FE000BEB712963C932E93119728E730E0F70135
:106FF0003383228326EC33E0358324839C01B9015B
:10700000882777FD8095982F0E94A47720E030E0B4
:1070100048EC52E40E943A77D70116966D937D931F
:107020008D939C9319970E94467E080F191FEDB708
:10703000FEB73A960FB6F894FEBF0FBEEDBF809133
:10704000C80483FF56C089E290E06BE270E04AE238
:1070500050E026E00E94464981E090E00E94120C38
:107060008093EB068CED97E10E94B64B2DB73EB7AF
:107070002A5030400FB6F8943EBF0FBE2DBFEDB67C
:10708000FEB60894E11CF11C9E012E5E3F4F200FBE
:10709000311FADB7BEB712963C932E93119728E7D8
:1070A00030E0F7013383228320ED33E035832483FE
:1070B0009C01B901882777FD8095982F0E94A477BD
:1070C00020E030E048EC52E40E943A77D70116966F
:1070D0006D937D938D939C9319970E94467E080F24
:1070E000191FEDB7FEB73A960FB6F894FEBF0FBE64
:1070F000EDBF8091C80484FF36C02DB73EB72A503B
:1071000030400FB6F8943EBF0FBE2DBFEDB7FEB7AF
:107110003196CE014296800F911FADB7BEB7129641
:107120009C938E93119788E790E0938382838BEDF5
:1071300093E0958384838091A8179091A917A091DB
:10714000AA17B091AB1786839783A087B1870E9457
:10715000467E080F191FEDB7FEB73A960FB6F894A2
:10716000FEBF0FBEEDBF8091C80485FF31C00E94F5
:107170009F0B2DB73EB72A5030400FB6F8943EBF54
:107180000FBE2DBFEDB7FEB731969E012E5E3F4F6D
:10719000200F311FADB7BEB712963C932E931197B7
:1071A00028E730E03383228329EE33E035832483DC
:1071B00066837783808791870E94467E080F191F18
:1071C000EDB7FEB73A960FB6F894FEBF0FBEEDBF0F
:1071D0008091C80486FF3AC0F8948091C8249091A9
:1071E000C924A091CA24B091CB2478942DB73EB77E
:1071F0002A5030400FB6F8943EBF0FBE2DBF4DB79A
:107200005EB74F5F5F4F9E012E5E3F4F200F311FD5
:10721000EDB7FEB73283218328E730E0FA013383EC
:10722000228327EF33E03583248386839783A087E7
:10723000B1870E94467E080F191F2DB73EB7265F03
:107240003F4F0FB6F8943EBF0FBE2DBF8091C804CC
:1072500087FF92C08091CC049091CD04009709F4EF
:107260008BC0F894C090C824D090C924E090CA2460
:10727000F090CB2478948091D4179091D517A09159
:10728000D617B091D717A7019601281B390B4A0BC7
:107290005B0BCA01B9010E94A277862EA72E682E29
:1072A000B92E6091CC047091CD0480E090E00E94F2
:1072B000A2779B01AC01682D7A2D862D9B2D0E9413
:1072C0003A775C014DB75EB74A5050400FB6F8941C
:1072D0005EBF0FBE4DBFEDB7FEB73196CE014296F1
:1072E000800F911FADB7BEB712969C938E931197E6
:1072F00088E790E09383828380E094E095838483A1
:10730000262F372F4A2D5B2D2683378340875187C1
:10731000C557DF4F6883CB58D040C657DF4F7883BF
:10732000CA58D0400E94467E080F191FC557DF4F2C
:107330006881CB58D040C657DF4F7881CA58D040BB
:10734000862F972FAA2DBB2D8093D5249093D624DA
:10735000A093D724B093D824C092D417D092D51735
:10736000E092D617F092D717EDB7FEB73A960FB660
:10737000F894FEBF0FBEEDBF8091C8049091C90480
:10738000A091CA04B091CB0490FF40C0F8948091C2
:10739000CC249091CD24A091CE24B091CF24789488
:1073A0002DB73EB72A5030400FB6F8943EBF0FBEFF
:1073B0002DBF4DB75EB74F5F5F4F9E012E5E3F4FB3
:1073C000200F311FEDB7FEB73283218328E730E06D
:1073D000FA01338322832DE034E0358324838683CE
:1073E0009783A087B1870E94467E080F191F2DB78B
:1073F0003EB7265F3F4F0FB6F8943EBF0FBE2DBF7E
:10740000C8010E94FC35009709F07CCC8091C8042B
:107410009091C904A091CA04B091CB0491FF92C08D
:107420008091CC049091CD04009709F48BC0F8941E
:10743000C090CC24D090CD24E090CE24F090CF24E6
:1074400078948091D8179091D917A091DA17B091BC
:10745000DB17A7019601281B390B4A0B5B0BCA01EE
:10746000B9010E94A277862EA72E682EB92E6091B0
:10747000CC047091CD0480E090E00E94A2779B0143
:10748000AC01682D7A2D862D9B2D0E943A775C01E8
:107490004DB75EB74A5050400FB6F8945EBF0FBE6E
:1074A0004DBFEDB7FEB73196CE014296800F911FCA
:1074B000ADB7BEB712969C938E93119788E790E074
:1074C0009383828386E194E095838483262F372FEC
:1074D0004A2D5B2D2683378340875187C557DF4F61
:1074E0006883CB58D040C657DF4F7883CA58D04006
:1074F0000E94467E080F191FC557DF4F6881CB5881
:10750000D040C657DF4F7881CA58D040862F972F7A
:10751000AA2DBB2D8093D9249093DA24A093DB2449
:10752000B093DC24C092D817D092D917E092DA1722
:10753000F092DB17EDB7FEB73A960FB6F894FEBFA0
:107540000FBEEDBF8091C8049091C904A091CA04F8
:10755000B091CB0492FF3EC0809173209091742033
:10756000A0917520B09176202DB73EB72A503040BB
:107570000FB6F8943EBF0FBE2DBF4DB75EB74F5F3D
:107580005F4F9E012E5E3F4F200F311FEDB7FEB7BC
:107590003283218328E730E0FA013383228323E218
:1075A00034E03583248386839783A087B1870E9444
:1075B000467E080F191F2DB73EB7265F3F4F0FB607
:1075C000F8943EBF0FBE2DBFC8010E94FC35009746
:1075D00009F098CB8091C8049091C904A091CA0485
:1075E000B091CB0493FF3CC04DB75EB74A505040BA
:1075F0000FB6F8945EBF0FBE4DBFEDB7FEB7319624
:10760000CE014296800F911FADB7BEB712969C93E4
:107610008E93119788E790E0938382838CE294E0C5
:107620009583848380916D1890916E18A0916F1846
:10763000B091701886839783A087B1870E94467E99
:10764000080F191FEDB7FEB73A960FB6F894FEBFB4
:107650000FBEEDBFC8010E94FC35009709F052CB68
:107660008091C8049091C904A091CA04B091CB0440
:1076700094FF3CC02DB73EB72A5030400FB6F89467
:107680003EBF0FBE2DBFEDB7FEB73196CE0142967D
:10769000800F911FADB7BEB712969C938E93119732
:1076A00088E790E09383828387E394E095838483E3
:1076B0008091D0249091D124A091D224B091D32450
:1076C00086839783A087B1870E94467E080F191F83
:1076D000EDB7FEB73A960FB6F894FEBF0FBEEDBFFA
:1076E000C8010E94FC35009709F00CCB8091C804BA
:1076F0009091C904A091CA04B091CB0495FF48C0F1
:1077000081E00E943D0B2DB73EB72A5030400FB6A6
:10771000F8943EBF0FBE2DBFEDB6FEB60894E11C37
:10772000F11C9E012E5E3F4F200F311FADB7BEB73B
:1077300012963C932E93119728E730E0F70133839C
:10774000228324E434E0358324832091A9043091FA
:10775000AA044091AB045091AC040E948078D701F8
:1077600016966D937D938D939C9319970E94467EF8
:10777000080F191FEDB7FEB73A960FB6F894FEBF83
:107780000FBEEDBFC8010E94FC35009709F0BACAD0
:107790008091C8049091C904A091CA04B091CB040F
:1077A00096FF48C082E00E943D0B2DB73EB72A509D
:1077B00030400FB6F8943EBF0FBE2DBFEDB6FEB6FB
:1077C0000894E11CF11C9E012E5E3F4F200F311FDB
:1077D000ADB7BEB712963C932E93119728E730E0D1
:1077E000F7013383228321E534E03583248320911C
:1077F000AD043091AE044091AF045091B0040E94AA
:107800008078D70116966D937D938D939C931997ED
:107810000E94467E080F191FEDB7FEB73A960FB6C5
:10782000F894FEBF0FBEEDBFC8010E94FC35009763
:1078300009F068CA8091C8049091C904A091CA0453
:10784000B091CB0497FF39C083E00E943D0B2DB768
:107850003EB72A5030400FB6F8943EBF0FBE2DBF42
:10786000EDB7FEB731969E012E5E3F4F200F311FC0
:10787000ADB7BEB712963C932E93119728E730E030
:10788000338322832EE534E0358324836683778334
:10789000808791870E94467E080F191F8C98EDB74C
:1078A000FEB73A960FB6F894FEBF0FBEEDBFC80103
:1078B0000E94FC35009709F025CA8091C804909178
:1078C000C904A091CA04B091CB04A0FF06C083E014
:1078D00061E046E020E00E9443138091C80490914B
:1078E000C904A091CA04B091CB04A1FF06C083E0F3
:1078F00061E046E021E00E9443138091C80490912A
:10790000C904A091CA04B091CB04A0FF3CC02DB71C
:107910003EB72A5030400FB6F8943EBF0FBE2DBF81
:10792000EDB7FEB73196CE014296800F911FADB7ED
:10793000BEB712969C938E93119788E790E093833D
:1079400082838BE694E09583848380916418909180
:107950006518A0916618B091671886839783A087F1
:10796000B1870E94467E080F191FEDB7FEB73A9601
:107970000FB6F894FEBF0FBEEDBFC8010E94FC35E4
:10798000009709F0BFC98091C8049091C904A091E3
:10799000CA04B091CB04A1FF3CC02DB73EB72A501A
:1079A00030400FB6F8943EBF0FBE2DBFEDB7FEB707
:1079B0003196CE014296800F911FADB7BEB7129699
:1079C0009C938E93119788E790E09383828383E75B
:1079D00094E0958384838091681890916918A091B0
:1079E0006A18B0916B1886839783A087B1870E942D
:1079F000467E080F191FEDB7FEB73A960FB6F894FA
:107A0000FEBF0FBEEDBFC8010E94FC35009709F014
:107A100079C9779A8091E4069091E50693FD749A6E
:107A20008091E4069091E50682FD08C08091CE0425
:107A300080FD04C081FF31C01D9B2FC000D000D04D
:107A40008EE794E0ADB7BEB712969C938E931197D4
:107A5000CE01429614969C938E9313970E94D67DE6
:107A60002091B1040F900F900F900F902223A9F056
:107A700000D000D0EDB7FEB7319684EE91E0ADB7FF
:107A8000BEB712969C938E931197228313820E9405
:107A9000E87D0F900F900F900F9080910807898BD1
:107AA000FE01E00FF11F128A0F5F1F4F8091E40665
:107AB0009091E50680FF12C000D000D085E894E0E8
:107AC000EDB7FEB792838183C801019694838383C7
:107AD0000E94D67D0F900F900F900F906801089430
:107AE000C11CD11CA1E1EA2EF12CEC0EFD1EC70138
:107AF000B6010E9444488091CE0482FF45C088EBC5
:107B000094E0B701A60128EC30E20E94C94C8091B4
:107B1000E4069091E50692FF37C0F8ECEF2EF0E214
:107B2000FF2EE6E9AE2EE4E0BE2ED7018D917D0159
:107B300000D000D0EDB7FEB73196ADB7BEB7129604
:107B4000BC92AE921197828313820E94D67D0F90D1
:107B50000F900F900F90B8EDEB16B0E2FB0629F7EF
:107B60008AE090E00E94087E00D000D08BE994E08B
:107B7000EDB7FEB792838183D482C3820E94D67D03
:107B80000F900F900F900F908091E4069091E50672
:107B900082FD73980E946F5485EF96E00E94EA3E42
:107BA0008091CE049091CF0490FF43C0E090CC042C
:107BB000F090CD040E948D55C82E1092CD041092E5
:107BC000CC0489E190E00E94A55524C0739880916F
:107BD00008078F5F80930807898BB8016F5F7F4F1D
:107BE000CE0141960E94444885EF96E00E94EA3E0D
:107BF00080919E0E90919F0E65E840E050E00E94BB
:107C0000B0408CE39AE0D20111969C938E9352C0BF
:107C100000E010E02091CE043091CF0430FDD6CFAB
:107C20008C2D90E00E94A555F092CD04E092CC04FA
:107C3000739A8091E7069091E806009711F00E94F0
:107C4000D153809108078F5F809308078091E406E5
:107C50009091E50682FF56C8739A54C880E097E079
:107C60000E949143009731F10E946F548091CE049D
:107C700087FD2B9880E097E060E470E00E94664307
:107C800084E59AE0F2019183808314C080E097E05C
:107C90000E949143009771F00E94D1538091CE04CD
:107CA00087FF30C82B9A2EC8D20111961C921E92C3
:107CB00083E001C081E0C557DF4F0FB6F894DEBF07
:107CC0000FBECDBFCF91DF911F910F91FF90EF902D
:107CD000DF90CF90BF90AF909F908F907F906F90EC
:107CE0005F904F9008950895FC01DB018C91808393
:107CF00011968C91119781830895FC01DB0190818D
:107D00008C91981741F421E030E0918111968C918B
:107D10001197981711F020E030E0C9010895FC0197
:107D200080818093ED2481818093EE240895DC018D
:107D30001996ED91FC911A970280F381E02D30970E
:107D400009F009950895EF92FF920F931F93DF9327
:107D5000CF9300D0CDB7DEB78C0188E10E94BF4839
:107D6000BC017E010894E11CF11CC7010E94743E15
:107D7000D8011996ED91FC911A970190F081E02DB0
:107D8000C801B70109950F900F90CF91DF911F9116
:107D90000F91FF90EF900895EF92FF920F931F9332
:107DA000CF93DF93EC018B017A014AE655E00E9404
:107DB000F83EFA86E986C8016EE675E00E94573FF4
:107DC000DF91CF911F910F91FF90EF9008950E9446
:107DD000113F0895CF93DF93EC0188E16DEE74E2DB
:107DE0000E94B548CE010E94143FDF91CF910895C3
:107DF000EF92FF920F931F93CF93DF93EC018B01D0
:107E00007A010E94303FF886EF82C80162E775E090
:107E10000E94573FDF91CF911F910F91FF90EF90FC
:107E200008950E94393F08950E94465A0895FC0122
:107E3000A781B0852D913C91F90109950895DC0148
:107E40001796ED91FC9118970280F381E02D309701
:107E500009F0099508958AE99EE00E94A3410895DA
:107E6000FC01738362838AE99EE0BF010E942E4277
:107E70000895BC018AE99EE00E94F5410895CF93E0
:107E8000DF93EC018AE99EE00E94A74108C082814D
:107E900093818C179D0739F0CF010E946D42E82F26
:107EA000F92F3097A1F7CF01DF91CF9108950F936C
:107EB0001F93CF93DF938B010E943F3FEC0100970C
:107EC00031F01D830C83C8010E949E5C8E83DF917C
:107ED000CF911F910F9108951F93CF93DF93EC01E2
:107EE000162F888580FF1DC0EC81FD813097C9F079
:107EF000D0939F0EC0939E0E82E08887CE01069697
:107F00000995992787FD909502978230910510F089
:107F1000133829F4CE01BE010E94953F02C081E0D2
:107F20008887DF91CF911F910895CF92DF92EF92D2
:107F3000FF920F931F93CF93DF93EC017B01C090CF
:107F40009E0ED0909F0E00919C0E10919D0EF801F8
:107F500003C00190F081E02DEC17FD0719F0309778
:107F6000C1F746C0209709F443C08885882309F1EA
:107F700018860BC0C017D10729F0C80167E8AE0109
:107F80000E946C3FF801008111810115110591F7E4
:107F9000EC81FD81309769F0CE15DF0551F0D0936B
:107FA0009F0EC0939E0ECE01069663E840E050E01F
:107FB0000995E0919C0EF0919D0ECE17DF0791F48C
:107FC0008881998190939D0E80939C0E0DC0808135
:107FD00091818C179D0729F48881998191838083F1
:107FE00003C0FC01309799F7D0929F0EC0929E0E6D
:107FF000DF91CF911F910F91FF90EF90DF90CF9085
:1080000008951F93CF93DF931092A00EC0919C0E02
:10801000D0919D0E11E00EC08985882341F018870C
:108020001986CE0162E840E050E00E946C3F099062
:10803000D881C02D209781F7DF91CF911F910895AE
:1080400080914B0F982F9F5F90934B0F08956091F5
:108050009E0E70919F0E0E94953F08958AE880932E
:108060004B0F1092A20E1092A10E10929D0E109224
:108070009C0E10929F0E10929E0E08958091A00E5D
:10808000882311F00E9401407091A10E772309F41A
:1080900055C02091A20E30E0F901EE0FFF1FEE0F48
:1080A000FF1FE20FF31FED55F14F608160934A0F00
:1080B000418152815093490F4093480F83819481AD
:1080C0009093470F8093460F2F5F3F4F2F71307073
:1080D0002093A20E71507093A10E009741F58091EC
:1080E0009C0E90919D0E18C08091A00E882311F0D7
:1080F0000E9401404091480F5091490F8091440FD8
:108100009091450F60914A0F0E946C3FE091440F9F
:10811000F091450F808191819093450F8093440F9A
:108120008091440F9091450F0097F1F607C0613898
:1081300019F421E0FC0120870E946C3F8091A00E81
:108140002091A10E30E0280F311DC90108958091C2
:10815000A00E2091A10E30E0280F311DC901089515
:108160007091A10E7032D9F02091A20E270F2F71BD
:108170002093430F30E0F901EE0FFF1FEE0FFF1FBA
:10818000E20FF31FED55F14F6083528341839483D7
:1081900083837F5F7093A10E20E030E002C021E076
:1081A00030E0C9010895CF93DF93C0919E0ED09126
:1081B0009F0E0E946C3FD0939F0EC0939E0EDF9146
:1081C000CF910895FC01AB0190919C0E80919D0E82
:1081D0009C01A32FB22F03C00D90BC91A02DAE1710
:1081E000BF0791F01097C1F7309771F090838183AA
:1081F000F0939D0EE0939C0E81E08087178216829B
:10820000CF0161E80E94D3400895FC01009741F03E
:1082100080858150823020F481E081878093A00E98
:10822000089521E030E0FC018085882311F420E0EE
:1082300030E0C9010895CF93DF93EC014A815B815F
:108240008C819D8160E070E00E94607D4A815B814D
:1082500088819981489F9001499F300D589F300D2A
:1082600011248E819F8160E070E0A9010E94607DF1
:10827000DF91CF910895FC018281938120E030E06D
:1082800019C0A481B581A20FB31F4C91442381F47E
:1082900081E08C9340815181249FC001259F900DE6
:1082A000349F900D112426813781280F391F07C074
:1082B0002F5F3F4F2817390720F320E030E0C90136
:1082C0000895FC01268137814281538180E090E04E
:1082D00018C02617370781F4A481B581A80FB91FEC
:1082E0002C91121614F421502C930480F581E02D6A
:1082F000E80FF91F80810895A081B1812A0F3B1FEB
:1083000001968417950728F38FEF0895FC01CB01A0
:10831000268137816217730790F0A081B181628155
:108320007381A69FA001A79F500DB69F500D1124E9
:10833000420F531F21E030E08417950710F020E032
:1083400030E0C9010895FC01118210820895FC01FA
:10835000808191810895FB0120813181FC0131836D
:1083600020830895FC01208131812115310511F40C
:1083700007C09C01F901808191810097D1F702C06B
:1083800020E030E0C9010895CF93DF93DC012D9107
:108390003C91119721153105A9F0F9018081918156
:1083A000009729F411961C921E920EC0F9012081AB
:1083B0003181D9018D919C9111970097B9F7118264
:1083C000108202C020E030E0C901DF91CF91089512
:1083D000DC01ED91FC911197309729F0808191811A
:1083E00011969C938E93CF010895CF93DF93FC0158
:1083F000A081B1811097D9F0C0E0D0E016C0A617D7
:10840000B70771F48D919C911197209719F491837E
:10841000808302C09983888311961C921E9207C0A4
:10842000ED0198818981A92FB82F109741F7DF912D
:10843000CF9108950F931F93CF93DF938C01EB019E
:108440000E94F541F8018081918199838883D183CD
:10845000C083DF91CF911F910F910895EF92FF920A
:108460000F931F93CF93DF93EC017B010E94F541A3
:10847000F70111821082CE010E94B241FC010097E7
:1084800019F4E882F98202C0F182E082DF91CF9193
:108490001F910F91FF90EF900895DC01ED91FC91F9
:1084A000119720E030E005C02F5F3F4F0190F08131
:1084B000E02D3097C9F7C9010895FB01309721F4E9
:1084C000BA010E941A420895DA01808191811196C1
:1084D0009C938E93518340830895009721F0FC0173
:1084E0002081318102C020E030E0C90108958091EF
:1084F0004C0F90914D0F009729F410924F0F10924E
:108500004E0F08950E943351E0914C0FF0914D0FA2
:108510002281338140815181240F351F281B390B63
:108520000CC04281538160817181460F571F481BE7
:10853000590B4217530708F49A010480F581E02D86
:10854000309779F7280F391F30934F0F20934E0F34
:10855000089580E895E00E9405410895CF92DF924A
:10856000EF92FF920F931F93CF93DF937C01FC0157
:1085700080819181009729F08A35910509F06EC0BC
:108580000BC010924D0F10924C0F8AE590E0F7014E
:108590009183808381E066C0673849F5CA01E09124
:1085A0004C0FF0914D0F03C00480F581E02D309702
:1085B00041F32681378128173907B1F3E0934C0F37
:1085C000F0934D0F0FC016962D913C9117972817D9
:1085D000390739F414962D913C91159735832483EE
:1085E000DF01FD01A481B581109769F7CECF623814
:1085F00061F6C0914C0FD0914D0F00E010E02BC000
:10860000CE010E9496600097F1F08E819F8168E80C
:10861000AE010E94B0400097A1F41F821E828C819F
:108620009D810115110521F0F8019583848304C013
:1086300090934D0F80934C0F1D821C820E947742B5
:10864000D8CF0E94A9428E019C818D81C92EE6015E
:108650006E01D82EE601209799F697CFF701118287
:10866000108283E0DF91CF911F910F91FF90EF90E7
:10867000DF90CF900895CF93DF93EC010E94A94241
:108680008E819F81009769F0E0914C0FF0914D0F22
:1086900006C0EC17FD07A9F00480F581E02D3097A6
:1086A000C1F780919E0E90919F0E9F838E83809143
:1086B0004C0F90914D0F9D838C83D0934D0FC093A1
:1086C0004C0F0E947742DF91CF910895CF93DF93B3
:1086D000EC010E947660CE010E943B43DF91CF9176
:1086E0000895CF93DF93EC010E948260CE010E9437
:1086F0003B43DF91CF910895CF93DF93EC010E942C
:108700008C60CE010E943B43DF91CF910895FC0124
:1087100080819181860F971F918380830E94774289
:10872000089521E030E0FC0186819781009711F0E7
:1087300020E030E0C9010895FC012281338180816D
:108740009181280F391FC9010895FC018081918111
:10875000089521E030E080914C0F90914D0F0097EB
:1087600011F420E030E0C901089580914C0F909100
:108770004D0F009729F020914E0F30914F0F02C0FE
:1087800020E030E0C9010895CF93DF93EC01E09140
:108790004C0FF0914D0F8E179F0741F48C819D81F6
:1087A00090934D0F80934C0F14C0FC01309731F023
:1087B000848195818C179D07C1F707C01D821C829B
:1087C0001F821E82DF91CF9108958C819D819583B8
:1087D00084830E947742F2CFCF92DF92EF92FF9292
:1087E0000F931F93CF93DF938C017A01FC0180815B
:1087F0009181009729F08B34910509F051C01EC07A
:1088000081E59FE00E94A741C82EE6017E01F92E76
:10881000E70109C06C817D81CE0102960E9466430A
:108820000990D881C02D2097A9F781E08093500F3F
:108830008BE490E0F8019183808337C06838A9F514
:1088400081E59FE00E94A741C82EE6016E01D92E66
:10885000E60123C0CE010296E816F906D9F481E5B7
:108860009FE0BE010E94F541E0909E0EF0909F0EA9
:108870008A859B8590939F0E80939E0EEC85FD8547
:10888000309719F08E859F850995F0929F0EE092A2
:108890009E0ECECF0990D881C02D2097D9F6C8CF93
:1088A000F8011182108283E001C081E0DF91CF9155
:1088B0001F910F91FF90EF90DF90CF90089510924D
:1088C000500F81E59FE00E94A34189E995E060E0B7
:1088D00070E00E94E24008950F931F93CF93DF93BF
:1088E000EC0100919E0E10919F0E1B870A875D87F9
:1088F0004C873F872E878091500F882379F089E934
:1089000095E090939F0E80939E0ECE0102960E945A
:10891000664310939F0E00939E0E02C07D836C836E
:1089200081E59FE0BE010E94F54181E59FE0BE0127
:108930000E942E42DF91CF911F910F9108950F93C6
:108940001F93CF93DF93EC018091500F882391F018
:1089500000919E0E10919F0E89E995E090939F0ED5
:1089600080939E0ECE0102960E94714310939F0E3B
:1089700000939E0E81E59FE0BE010E94F54181E5D6
:108980009FE0BE010E942E42DF91CF911F910F9177
:1089900008950F931F93CF93DF93EC018091500FB5
:1089A000882391F000919E0E10919F0E89E995E029
:1089B00090939F0E80939E0ECE0102960E947C4360
:1089C00010939F0E00939E0E81E59FE0BE010E94D2
:1089D000F54181E59FE0BE010E942E42DF91CF91DB
:1089E0001F910F910895CF93DF93EC018091500F69
:1089F000882329F0CE0102960E94C44304C01F823E
:108A00001E821986188681E59FE0BE010E94F5410D
:108A1000DF91CF910895CF93DF93EC018091500FB8
:108A2000882331F0CE0102960E9491439C0114C02C
:108A300081E59FE00E94A741E82FF92F06C0EC17BF
:108A4000FD0741F00190F081E02D3097C1F721E062
:108A500030E002C020E030E0C901DF91CF910895FD
:108A60000F931F930091ED241091EE240E9460510A
:108A70002DB73EB7225530400FB6F8943EBF0FBE1B
:108A80002DBFEDB7FEB731962AE23EE0ADB7BEB7D7
:108A900012963C932E9311970283138214831582AE
:108AA00066837783808791878091E0269091E12685
:108AB000A091E226B091E32682879387A487B587A9
:108AC0008091E4269091E526A091E626B091E726D4
:108AD00086879787A08BB18B8091E8269091E926B5
:108AE000A091EA26B091EB26828B938BA48BB58B59
:108AF0008091EC269091ED26A091EE26B091EF2684
:108B0000868B978BA08FB18F8091F0269091F12664
:108B1000A091F226B091F326828F938FA48FB58F08
:108B20008091F4269091F526A091F626B091F72633
:108B3000868F978FA0A3B1A38091F8269091F926F4
:108B4000A091FA26B091FB2682A393A3A4A3B5A378
:108B50008091FC269091FD26A091FE26B091FF26E3
:108B600086A397A3A0A7B1A7809100279091012782
:108B7000A0910227B091032782A793A7A4A7B5A726
:108B80008091042790910527A0910627B09107278F
:108B900086A797A7A0ABB1AB809108279091092732
:108BA000A0910A27B0910B2782AB93ABA4ABB5ABD6
:108BB00080910C2790910D27A0910E27B0910F273F
:108BC00086AB97ABA0AFB1AF8091102790911127E2
:108BD000A0911227B091132782AF93AFA4AFB5AF86
:108BE000EDB7FEB7FF968091142790911527A091BD
:108BF0001627B091172780839183A283B383EDB7A3
:108C0000FEB7ED5BFF4F8091182790911927A09137
:108C10001A27B0911B2780839183A283B383EDB77A
:108C2000FEB7E95BFF4F80911C2790911D27A09113
:108C30001E27B0911F2780839183A283B383EDB752
:108C4000FEB7E55BFF4F8091202790912127A091EF
:108C50002227B091232780839183A283B383EDB72A
:108C6000FEB7E15BFF4F8091242790912527A091CB
:108C70002627B091272780839183A283B3830E9404
:108C8000E87D0091ED241091EE242DB73EB72E5AC9
:108C90003F4F0FB6F8943EBF0FBE2DBF0E946051EC
:108CA000ADB7BEB7D2970FB6F894BEBF0FBEADBF7B
:108CB000EDB7FEB731962BEB3DE012963C932E9329
:108CC00011970283138214831582668377838087CA
:108CD00091878091282790912927A0912A27B091E8
:108CE0002B2782879387A487B58780912C27909123
:108CF0002D27A0912E27B0912F2786879787A08BAD
:108D0000B18B8091302790913127A0913227B0917B
:108D10003327828B938BA48BB58B809134279091D2
:108D20003527A0913627B0913727868B978BA08F58
:108D3000B18F8091382790913927A0913A27B0912F
:108D40003B27828F938FA48FB58F80913C27909182
:108D50003D27A0913E27B0913F27868F978FA0A3F4
:108D6000B1A38091402790914127A0914227B091D3
:108D7000432782A393A3A4A3B5A3809144279091F2
:108D80004527A0914627B091472786A397A3A0A780
:108D9000B1A78091502790915127A0915227B0916F
:108DA000532782A793A7A4A7B5A780915427909192
:108DB0005527A0915627B091572786A797A7A0AB14
:108DC000B1AB0E94E87D2DB73EB72E5C3F4F0FB68A
:108DD000F8943EBF0FBE2DBF1F910F91089580E301
:108DE0008093530F0895EF92FF92CF93DF932091DA
:108DF000530F30E0C0E3D0E0C21BD30B285A304FF2
:108E0000B901AE010E94577DCE01DF91CF91FF9055
:108E1000EF900895AF92BF92CF92DF92EF92FF92C0
:108E20000F931F93CF93DF937C01C090540FD0908A
:108E3000550F2091530F30E08601005D1F4F021B3C
:108E4000130B01381105E0F4C0E3D0E0C21BD30BD3
:108E5000285A304FB901AE010E94577DCE0DDF1D5B
:108E60002091560F3091570F80910A1090910B105E
:108E7000280F391FCE01B901A6010E94577D02C0FB
:108E800000E010E0C801DF91CF911F910F91FF909A
:108E9000EF90DF90CF90BF90AF9008959091530FD7
:108EA000980F9093530F08954091540F5091550F80
:108EB0009C014817590798F080910A1090910B1067
:108EC000820F931F90930B1080930A10421B530B39
:108ED0005093550F4093540F21E030E002C020E042
:108EE00030E0C90108959093550F8093540F089571
:108EF00020910A1030910B102857304FC901089566
:108F00002091530F30E0285A304FC901089521E0D5
:108F100030E08091560F9091570F4FE088389407BA
:108F200011F420E030E0C90108950E9487470097BE
:108F300071F028E83FE06091560F7091570F409113
:108F4000540F5091550FC9010E94577D0895A0916B
:108F50000A10B0910B101097B9F02091540F309176
:108F6000550F205D3F4FA857B04FE8E8FFE080E382
:108F700090E003C04D914193019682179307D4F37B
:108F800010920B1010920A1008958091560F909134
:108F9000570F08958091540F9091550F0895909117
:108FA000530F80E3891B089580E39091530F891B31
:108FB0002091540F3091550F280F311DC90108958C
:108FC0001F93CF93DF93EC011091530F812F90E00B
:108FD0008C179D076CF00E94D4478C0F9D1F813821
:108FE000910530F41C1B1093530F21E030E002C0B8
:108FF00020E030E0C901DF91CF911F910895CF9318
:10900000DF93E7EFF4E21192119285E2E732F8077D
:10901000D1F7C0E0D0E0CE01880F991F81519B4D60
:1090200068E675E00E94743E2196C430D10599F738
:10903000DF91CF91089510920B1010920A101092A8
:10904000550F1092540F80E38093530F88E89FE0F0
:109050009093570F8093560F0E94FF4708950F93E8
:109060001F93CF93DF93EC018B010E941B48D09399
:10907000570FC093560F1093550F0093540FDF9165
:10908000CF911F910F910895CF92DF92EF92FF92AF
:109090000F931F93DF93CF9300D0CDB7DEB78C0132
:1090A00069837A830E941B4869817A81C62ED72EF4
:1090B00021E8C216D10418F030E8C32ED12C8091DB
:1090C000560F9091570FB801A6010E94577DD0927C
:1090D000550FC092540FC6010F900F90CF91DF91A2
:1090E0001F910F91FF90EF90DF90CF900895282F60
:1090F000392FD901E7EFF4E280E301900D9281501E
:10910000E1F7862F972FDC01EFEEF4E288E0019083
:109110000D928150E1F70895E7EFF4E2282F392FFF
:10912000D90180E30D9001928150E1F7AFEEB4E2F6
:10913000862F972FFC0188E001900D928150E1F776
:109140000895E82FF0E0EE0FFF1FE950FB4D71830B
:10915000608381E090E00895E82FF0E0EE0FFF1FBC
:10916000E950FB4D80819181089590E0880F991F0F
:1091700081549B4D0E94743E81E090E00895282F19
:1091800030E0220F331F21543B4DC9010895811552
:10919000910511F00197F1F70895E0912A25F091DA
:1091A0002B2590818091292589230895E0912725F9
:1091B000F0912825808190912925892B8083E09149
:1091C0002C25F0912D25808190912925892B808354
:1091D0000895E0912725F0912825908180912925F7
:1091E000809589238083E0912C25F0912D25908115
:1091F000809129258095892380830895FF920F937C
:109200001F93E0912725F0912825908180912925B1
:10921000809589238083E0912C25F0912D258081F4
:1092200090912925892B80838FEB93E00E94C7487A
:10923000FFB6F894E0912C25F0912D259081809136
:10924000292580958923808383E890E00E94C74880
:10925000E0912A25F0912B25008110912925FFBE50
:1092600078948BE393E00E94C748E0912A25F0911F
:109270002B25808190912925892319F0802F812326
:1092800001C081E01F910F91FF90089550932D250B
:1092900040932C25709328256093272590932B25A8
:1092A00080932A2581E090E002C0880F991F2A95BB
:1092B000E2F7809329250E94FE4808950F931F939B
:1092C000182F0FB7F894E0912C25F0912D2580816F
:1092D00090912925892B808383E090E00E94C748E4
:1092E000112351F0E0912C25F0912D259081809152
:1092F000292580958923808387E190E00E94C748D3
:10930000E0912A25F0912B258081909129258923B0
:1093100009F410E089E590E00E94C748E0912C250F
:10932000F0912D2590818091292580958923808336
:109330000FBF8BE390E00E94C748812F1F910F91D0
:1093400008950F931F93182F08E0812F81700E94BA
:109350005E491695811110680150B9F7812F1F9150
:109360000F9108958FEF0E94A1490895DF92EF9227
:10937000FF920F931F93CF93DF93182FEB010E945F
:10938000FE48882389F580EF0E94A149EE2400E47D
:1093900098EFD92ED00E81E00E945E49F82E81E030
:1093A0000E945E49882319F0FF2069F020C0FF2049
:1093B00051F4011728F0888180FF05C0101719F0BB
:1093C000E02EFF24F3948F2D0E945E4988818695BC
:1093D0008883FF2011F08068888301500D15D9F62D
:1093E000002339F02196D4CFEE24EA9402C08EEF08
:1093F000E82E8E2DDF91CF911F910F91FF90EF906E
:10940000DF9008950F931F93CF93DF93182FEB01F5
:109410000E94FE48209751F085E50E94A14908E08E
:1094200089910E94A1490150D9F703C08CEC0E9498
:10943000A149812F0E94A149DF91CF911F910F91E6
:1094400008950F931F93CF93DF93FB01DA01E80197
:10945000408150E0718160E0462B572B803171F4E0
:10946000BA016E7F13E0660F771F1A95E1F79681B8
:109470004CE050E0491B5109460F571F57FF06C0EB
:1094800091E09C93509541955F4F01C01C928832AA
:1094900089F4848190E0BC0160767070603671055B
:1094A00049F086FF02C04E7F05C085FF02C04C7F99
:1094B00001C0487FCA0154E0969587955A95E1F717
:1094C000F90180834F70488380E0DF91CF911F9135
:1094D0000F9108950F931F93CF93DF938C01EB01AE
:1094E000F8018081BE010E94B649F8018083815055
:1094F0008D3F28F48881883211F0803189F7DF911F
:10950000CF911F910F9108951F93CF93DF93EC019B
:109510000E94FE4884EBBE010E94024A81E00E9444
:109520005E49182F0E94FE4881E0112309F480E073
:10953000DF91CF911F9108951F93CF93DF93182F41
:10954000EB010E94FE480E94CD48882349F084E444
:10955000BE010E94024A113029F00E94D64802C082
:1095600082E001C080E0DF91CF911F9108956F925A
:109570007F928F929F92AF92BF92CF92DF92EF92A3
:10958000FF920F931F93DF93CF93CDB7DEB7299749
:109590000FB6F894DEBF0FBECDBF7C014B013A0180
:1095A00059010E94FE488EEBB7010E94024A8E01CB
:1095B0000F5F1F4F8AE0C82ED12CCC0EDD1E0E94FB
:1095C000B249F80181938F01EC15FD05C1F78E01B9
:1095D0000F5F1F4FC80169E070E00E944765882354
:1095E00051F4F7018081B801A401930185010E9423
:1095F000214A80E001C083E029960FB6F894DEBFCF
:109600000FBECDBFCF91DF911F910F91FF90EF90D3
:10961000DF90CF90BF90AF909F908F907F906F9092
:1096200008957F928F929F92AF92BF92CF92DF92D6
:10963000EF92FF920F931F93DF93CF93CDB7DEB7D7
:1096400029970FB6F894DEBF0FBECDBF782E5B0111
:109650004A0179018EEB60E070E00E94024A8E01BF
:109660000F5F1F4F9AE0C92ED12CCC0EDD1E0E9439
:10967000B249F80181938F01EC15FD05C1F78E0108
:109680000F5F1F4FC80169E070E00E9447658823A3
:1096900049F4872DB801A501940187010E94214A50
:1096A00080E001C083E029960FB6F894DEBF0FBEBC
:1096B000CDBFCF91DF911F910F91FF90EF90DF9081
:1096C000CF90BF90AF909F908F907F9008950F9311
:1096D0001F93DF93CF93CDB7DEB728970FB6F894DB
:1096E000DEBF0FBECDBF182F062FDE011196EBEAAD
:1096F000F5E088E001900D928150E1F7242F3327A7
:1097000027FD309541E752E0249FC001259F900D31
:10971000349F900D112464E670E00E94527AAB01F0
:1097200064E6069FB0011124460F571FFE013196D3
:10973000CE010996619170E02617370719F44F5F43
:109740005F4F03C0E817F907A9F7112319F05095E7
:1097500041955F4FCA0128960FB6F894DEBF0FBE41
:10976000CDBFCF91DF911F910F9108950F931F935C
:10977000DF93CF93CDB7DEB72B970FB6F894DEBF4C
:109780000FBECDBF182F092F885F612F792F0E9440
:109790009C4A882309F049C066E471E48FE090E0B8
:1097A0000E94234C812F902FBE016F5F7F4FAE012F
:1097B0004E5F5F4F9E012D5F3F4F0E94B74A882347
:1097C000A1F5DE011496E3EAF5E088E001900D9240
:1097D0008150E1F74B81642F70E021E732E0629F16
:1097E000C001639F900D729F900D112464E670E09C
:1097F0000E94527A9A8184E6989FC0011124680FD2
:10980000791FFE013496CE010C962191421719F46E
:109810006F5F7F4F03C0E817F907B9F78981882385
:1098200031F0709561957F4F02C064E371E2CB0126
:109830002B960FB6F894DEBF0FBECDBFCF91DF9150
:109840001F910F910895DC01CB0181159105A105B0
:10985000B10529F081509040A040B040D9F708955B
:109860001092B90080E28093B800089594EA909332
:10987000BC0020EA36E841E050E005C0215030400D
:1098800040405040F1F09091BC0097FFF7CF1DC0D1
:109890009031B9F48093BB0084E88093BC0080EAE7
:1098A00096E8A1E0B0E004C00197A109B10959F020
:1098B0002091BC0027FFF8CF0EC081E0903421F446
:1098C0000FC081E0089581E008959091B900987FDC
:1098D0009830F1F6DFCF9091B900987F983169F711
:1098E00080E0089544EA34E824E94093BC00909174
:1098F000BC0097FFFCCF9091B900987F983011F091
:10990000903199F78093BB003093BC009091BC00DC
:1099100097FFFCCF9091B900987F903211F0983565
:1099200039F42093BC009091BC0094FDFCCFDDCFB6
:1099300008950E94364C089584E98093BC0080917C
:10994000BC0084FDFCCF08958093BB0084E8809325
:10995000BC008091BC0087FFFCCF9091B900987F3C
:1099600081E0983209F480E0089584EC8093BC0093
:109970008091BC0087FFFCCF8091BB00089584E8F4
:109980008093BC008091BC0087FFFCCF8091BB001E
:109990000895E82FF92F80E1919190933F01815034
:1099A000D9F780913C018F7D80933C0180913C01EF
:1099B000877F80933C01862F972FFC0180E1919156
:1099C00090933E018150D9F780913C01806880934B
:1099D0003C0180913D0180FFFCCF4051504080917F
:1099E0003C01806280933C0180913C01877F8093A1
:1099F0003C0114C0862F972FFC0180E19191909338
:109A00003E018150D9F780913C01806880933C01F0
:109A100080913D0180FFFCCF405150401416150647
:109A20004CF3822F932FFC0180E190913E019193A2
:109A30008150D9F781E090E008950F931F93CF9361
:109A4000DF938C018CE70E94724C8CE70E94A44C3F
:109A5000C0E0D0E0F80181918F010E94A44C2196D2
:109A6000C031D105B9F70E949C4CDF91CF911F9175
:109A70000F910895813039F48CE790E060E070E058
:109A800040E050E006C08CE790E060E070E040EC21
:109A900050E00E9449110895813039F48CE790E03C
:109AA00060E070E04EE050E006C08CE790E060E0DF
:109AB00070E048E050E00E94491108958CE790E082
:109AC00060E070E041E050E00E9449116AE67AE00F
:109AD00080E090E00E94234C08958CE790E060E0E5
:109AE00070E048E350E00E9449118CE790E060E0AC
:109AF00070E049E350E00E9449118CE790E060E09B
:109B000070E044E150E00E9449118CE790E060E091
:109B100070E048E750E00E9449118CE790E060E077
:109B200070E04EE550E00E9449118CE790E060E063
:109B300070E04DE650E00E9449116CE17AE186E068
:109B400090E00E94234C8CE790E060E070E04CE0F5
:109B500050E00E9449118CE790E060E070E041E045
:109B600050E00E9449118CE790E060E070E046E030
:109B700050E00E9449116AE67AE080E090E00E949D
:109B8000234C0895DF93CF93CDB7DEB7A2970FB6DE
:109B9000F894DEBF0FBECDBFDE011196E3EBF5E01A
:109BA00081E101900D928150E1F7DE015296E4ECE3
:109BB000F5E081E101900D928150E1F70E946D4D39
:109BC000CE0101960E941D4D82E00E943A4D6AE648
:109BD0007AE080E090E00E94234CCE0142960E9401
:109BE0001D4D60E17EEA88E290E00E94234C80E017
:109BF0000E944C4D60E17EEA88E290E00E94234C96
:109C000081E00E944C4DA2960FB6F894DEBF0FBEC5
:109C1000CDBFCF91DF910895E6E4F1E0808120810E
:109C200090813081829586958695837022952F70DC
:109C3000822B832B92959F70892B0895DF92EF9250
:109C4000FF920F931F93DF93CF9300D0CDB7DEB772
:109C500080E06CE046E00E94F45189E18093C4000A
:109C60001092C50082E08093C00080E00E949E5266
:109C70000E94235184B784B784B784B784B7EEEACF
:109C8000FDE222E432E4318320833A968DB79EB719
:109C90000A97E817F907B8F300D000D087E79FE0EC
:109CA000ADB7BEB712969C938E93119785ED95E054
:109CB00014969C938E9313970E94E87D0F900F90BB
:109CC0000F900F900E9460610E942E4080E895E006
:109CD00060E070E00E94E2400E945F44E091200654
:109CE000F091210609950E940C4E90E00E949E6121
:109CF000CE0101960E945150882359F000D087E58B
:109D00009FE0EDB7FEB7928381830E94E87D0F90BC
:109D10000F908E010F5F1F4FC8010E948F3E0E945F
:109D20005B507C010E946050BC01C701A8010E94E9
:109D3000AB550E94B94F0E9490550E9465500E94F9
:109D4000185700D08AE49FE0ADB7BEB712969C9337
:109D50008E9311970E94E87D00D0EDB7FEB7319643
:109D600006E41FE0ADB7BEB712961C930E93119791
:109D70008A81828313820E94E87DEDB7FEB7319617
:109D8000ADB7BEB712961C930E931197898182834B
:109D900013820E94E87D0F900F9084E49FE0EDB75E
:109DA000FEB7928381830E94E87D0F900F900E94FE
:109DB000A461E091A306F091A4060995E0918A06BA
:109DC000F0918B060995E0914C06F0914D060995AE
:109DD000E0908806F09089060091A1061091A206F5
:109DE0000E948D55D82E0E9420572DB73EB72A507D
:109DF00030400FB6F8943EBF0FBE2DBFEDB7FEB793
:109E0000319629E23FE0ADB7BEB712963C932E9350
:109E10001197F382E28215830483D68217828087AA
:109E200011860E94E87DE091AD06F091AE062DB757
:109E30003EB7265F3F4F0FB6F8943EBF0FBE2DBF13
:109E40003097D1F00995BC0100D000D086E19FE0A9
:109E5000ADB7BEB712969C938E93119780E890E0B1
:109E60000E943E7AEDB7FEB7748363830E94E87D5B
:109E70000F900F900F900F9000D084E19FE0ADB74E
:109E8000BEB712969C938E9311970E94E87D0F9017
:109E90000F908CEC96E060E070E00E94E2408EE46F
:109EA00095E00E944A6000D08CE09FE0EDB7FEB7DD
:109EB000928381830E94E87D0F900F900F900F9006
:109EC000CF91DF911F910F91FF90EF90DF90089558
:109ED000EF92FF920F931F9380E88093610010929E
:109EE00061000E941E4E0E943E400E94BF5280911F
:109EF0002E2590912F25009729F0019790932F25DB
:109F000080932E25E0903025F09031250091322568
:109F1000109133250E946051E616F70608071907CD
:109F200011F30E9460516093302570933125809326
:109F3000322590933325D7CF00D000D000D0EDB795
:109F4000FEB7319626E03FE0ADB7BEB712963C9320
:109F50002E93119793838283758364830E94E87D97
:109F60008DB79EB706960FB6F8949EBF0FBE8DBFF5
:109F700008950F931F93DF93CF93CDB7DEB7A297CA
:109F80000FB6F894DEBF0FBECDBF83E490E00E9411
:109F9000327F89839A83982F9B50903108F08A836F
:109FA0009A819095891709F470C000D082EB9FE0E8
:109FB000ADB7BEB712969C938E9311970E94E87D21
:109FC0008E010D5F1F4F0F900F90D80180E090E041
:109FD000FC01EE56F04FE491ED9301968830910527
:109FE000B9F7F894CE01039661E270E048E050E0E2
:109FF0000E94387FD80180E090E0FC01E656F04FE7
:10A00000E491ED9301968E309105B9F7CE01039658
:10A0100069E270E04EE050E00E94387F80E090E01E
:10A02000FC01E855F04FE491D801ED938D010196C4
:10A030008A309105A9F7CE01039667E370E04AE004
:10A0400050E00E94387F85E490E06DEC7BEA0E944E
:10A05000507F87E490E060E070E00E94507F89E4E8
:10A0600090E060E00E94427F81E490E060E070E078
:10A070000E94507F8AE1898385EE8A8369817A8193
:10A0800083E490E00E94507F78948981A2960FB675
:10A09000F894DEBF0FBECDBFCF91DF911F910F911E
:10A0A0000895F89461E270E042E050E00E941A7F67
:10A0B000789480E0089585E490E00E94327F0895CE
:10A0C00087E490E00E94327F089589E490E00E9446
:10A0D0002A7F089520913C2530913D2540913E25D1
:10A0E00050913F2590E0A0E0B0E0280F391F4A1FB3
:10A0F0005B1F20933C2530933D2540933E25509394
:10A100003F25209138253091392540913A255091AD
:10A110003B25280F391F4A1F5B1F2093382530939A
:10A12000392540933A2550933B252091DC26222364
:10A13000A1F020913425309135254091362550915C
:10A140003725280F391F4A1F5B1F20933425309372
:10A150003525409336255093372508951F920F9249
:10A160000FB60F920BB60F9211242F933F934F937C
:10A170005F936F937F938F939F93AF93BF93EF936F
:10A18000FF9380910C1090910D10019690930D10FB
:10A1900080930C1080910E108F5F80930E10809131
:10A1A0000E108038A9F410920E1080913C259091E9
:10A1B0003D25A0913E25B0913F250196A11DB11DE1
:10A1C00080933C2590933D25A0933E25B0933F2559
:10A1D0008091DC268823F1F080910F108F5F8093AF
:10A1E0000F1080910F108038A9F410920F108091F9
:10A1F000342590913525A0913625B09137250196CB
:10A20000A11DB11D8093342590933525A09336254B
:10A21000B09337250E94A943009711F00E94A942EC
:10A22000FF91EF91BF91AF919F918F917F916F912E
:10A230005F914F913F912F910F900BBE0F900FBEEA
:10A240000F901F901895F8941092B60016BC83EFEB
:10A2500087BD82E084BD94E095BD95B395BB8093A6
:10A260006E007894089520910C1030910D1080911B
:10A270000C1090910D1028173907A9F7C9010895FE
:10A2800007C022E330E0000021503040E1F70197A1
:10A290000097B9F708950F931F93CF93DF938C0125
:10A2A0000E943351EC010E9433518C1B9D0B80178F
:10A2B0009107C8F3DF91CF911F910F9108950895F1
:10A2C00020913C2530913D2540913E2550913F25E0
:10A2D00080913C2590913D25A0913E25B0913F2550
:10A2E000281739074A075B0759F7B901CA010895CA
:10A2F0001F920F920FB60F9211241092F9050F9032
:10A300000FBE0F901F9018951F920F920FB60F92CD
:10A310000BB60F9211242F933F934F935F936F933C
:10A320007F938F939F93AF93BF93EF93FF93E091AE
:10A33000EF05F091F0058081E091FA05F091FB05C1
:10A34000309709F00995FF91EF91BF91AF919F91DF
:10A350008F917F916F915F914F913F912F910F90CE
:10A360000BBE0F900FBE0F901F9018951F920F926B
:10A370000FB60F921124109206060F900FBE0F9089
:10A380001F9018951F920F920FB60F920BB60F9257
:10A3900011242F933F934F935F936F937F938F93EA
:10A3A0009F93AF93BF93EF93FF93E091FC05F091E0
:10A3B000FD058081E0910706F0910806309709F0CD
:10A3C0000995FF91EF91BF91AF919F918F917F91EF
:10A3D0006F915F914F913F912F910F900BBE0F9016
:10A3E0000FBE0F901F90189590E02DE030E0829FF7
:10A3F000F001839FF00D929FF00D1124E151FA4F6F
:10A40000A281B3811C92A481B5816C93A681B7818E
:10A4100088ED8C93A085B1854C93128614861386A3
:10A42000089590E02DE030E0829FF001839FF00DD1
:10A43000929FF00D1124E151FA4F81E08287A081B3
:10A44000B1816C933A9680818823E9F708951F9330
:10A45000182F8A3031F4809110106DE00E94115253
:10A4600002C08D3029F080911010612F0E9411528E
:10A4700080E090E01F910895EF92FF921F93CF9399
:10A48000DF93182FE62EE7017E01F72EE7010CC0BF
:10A490008A3021F4812F6DE00E94115269916D3054
:10A4A00019F0812F0E9411528881882389F7DF914A
:10A4B000CF911F91FF90EF9008950F931F93DF931B
:10A4C000CF93CDB7DEB7FE013A9601E110E1C801A6
:10A4D00060E470E0488559859F010E94847E8F81E9
:10A4E000B8010E943C52CF91DF911F910F910895C6
:10A4F0001F93CF93DF93182FEB0104C0812F0E948D
:10A5000011522196FE0164916623C1F7DF91CF912C
:10A510001F91089590E02DE030E0829FF001839F2D
:10A52000F00D929FF00D1124E151FA4F748763876B
:10A530000895682F80E00E941152089580931010B2
:10A5400081EE95E09093A92D8093A82D089584B76E
:10A55000877F84BF88E10FB6F894809360001092E3
:10A5600060000FBE08952FE088E190E00FB6F894E8
:10A57000A895809360000FBE209360000895A89571
:10A58000089588E10FB6F8948093600010926000FF
:10A590000FBE0895F89428E088E190E00FB6F89493
:10A5A000A895809360000FBE20936000FFCF80913C
:10A5B0004F2590E0FC01EE0FFF1F9695982F8827FE
:10A5C00097958795E80FF91FE05BFA4D1082089583
:10A5D000809147258091472590E008958091390129
:10A5E00081FD0CC081E491E06FE140E00E94C15820
:10A5F000813039F021E030E0813129F020E030E095
:10A6000002C021E030E0C90108958091390181FD47
:10A6100012C081E491E06FE140E00E94C158982FA0
:10A620008151823050F09F3141F0913041F081E012
:10A63000923031F402C081E0089580E0089580E016
:10A6400008950E9405538823E1F3089581E491E081
:10A650006FE140E00E94C1580895E9E3F1E0808194
:10A6600080818D7F80838DE090E00197F1F782E417
:10A6700091E06FE140E023E00E94CB5883E090E05E
:10A680000197F1F708950E9421531092DC260E9451
:10A690002D538091390182608093390180915F2729
:10A6A0008823E9F180919400909195002091702782
:10A6B0003091712782179307A0F480913C279091E5
:10A6C0003D27A0913E27B0913F278C57914EAF4F29
:10A6D000BF4F80933C2790933D27A0933E27B09394
:10A6E0003F278091940090919500821B930BA0E0EE
:10A6F000B0E020913C2730913D2740913E2750917A
:10A700003F27820F931FA41FB51F80933C27909370
:10A710003D27A0933E27B0933F2710925F2780915B
:10A7200061278823E9F18091940090919500209110
:10A7300074273091752782179307A0F480914427DE
:10A7400090914527A0914627B09147278C57914E6D
:10A75000AF4FBF4F8093442790934527A093462740
:10A76000B09347278091940090919500821B930BA2
:10A77000A0E0B0E020914427309145274091462742
:10A7800050914727820F931FA41FB51F8093442722
:10A7900090934527A0934627B093472710926127AF
:10A7A00008958091DC26882381F0809151108823C0
:10A7B00021F40E940553882331F481E08093D41062
:10A7C00021E030E004C00E94435320E030E0C901A2
:10A7D00008950F931F93182F883049F0863039F071
:10A7E000893029F0863119F0893109F041C0809112
:10A7F000390181FD40C00E9421530E942653082F39
:10A80000181709F43BC0183019F40E942D5329C0C1
:10A81000193141F48631A9F482E491E06FE140E01E
:10A8200029E009C0163169F4893159F482E491E0D4
:10A830006FE140E026E00E94CB58E3E0F0E0319782
:10A84000F1F782E491E06FE140E0212F0E94CB58C4
:10A85000083019F4E9E6F1E002C0E3E0F0E03197F6
:10A86000F1F70E942653811749F023E430E008C035
:10A8700022E430E005C024E430E002C020E430E00F
:10A88000C9011F910F9108958091940090919500B6
:10A89000909375278093742721E0209361278091FE
:10A8A000390181FF15C02093DB268091940090919F
:10A8B0009500909371278093702720935F27809154
:10A8C00039018D7F809339018091DB268823E1F760
:10A8D00086E10E94E95381E08093DC26089580910F
:10A8E000DC26882351F480915110882321F081E0E7
:10A8F0008093D31002C00E94445481E090E00895F8
:10A900001F93DF93CF930F92CDB7DEB78FB78983B5
:10A9100080915110882331F5F8948091DC268823AA
:10A9200051F08091390181FD1BC00E94055388239D
:10A93000B9F080E003C00E946F5481E0909147011C
:10A940009E3010F010E001C01FEF882311F00E942C
:10A95000D15316FF05C089818FBF21E030E004C0CC
:10A9600089818FBF20E030E0C9010F90CF91DF9146
:10A970001F9108958091D310882321F00E944454A0
:10A980001092D3108091D410882321F00E94435359
:10A990001092D410109251100895EF92FF92CF931D
:10A9A000DF93B82FA92FF62FE72F81E08093511066
:10A9B0002091202730912127409122275091232751
:10A9C0002F5F3F4F4F4F5F4F20932027309321271A
:10A9D0004093222750932327862F8E5F87FF0CC03A
:10A9E0008091D9269091DA2601969093DA26809369
:10A9F000D926CFEFDFEF0BC022E530E1C9016B2F85
:10AA00007A2F4F2F5E2F0E94577DC0E0D0E00E942A
:10AA1000BA54CE01DF91CF91FF90EF9008959091BD
:10AA2000390191FD0AC0282F803108F02FE085E41C
:10AA300091E06FE040E00E94CB5808958093D610DB
:10AA400008950E9426538250813130F4E82FF0E0BF
:10AA5000EC5CF94F8081089581E0089508958FEFAF
:10AA600080934E018CE691E060EF44E022E00E948A
:10AA7000CB588CE290E06EE041E025E00E94CB589C
:10AA800080E880936F018091460180936D0184E49A
:10AA900091E060E245E021E00E94CB580895CF9319
:10AAA000DF93CDEFD3E0CE010197F1F70E94B758C5
:10AAB000109250251092D2251092542610924F25B4
:10AAC00010924E25E9E3F1E080818E7F80838081C2
:10AAD0008D7F80838DE090E00197F1F78081816028
:10AAE000808382E491E06FE140E023E00E94CB5854
:10AAF0002197F1F780915D0180915E010E942F55B1
:10AB000086E196E060E070E00E94E2400E944454DA
:10AB100081E090E0DF91CF9108958091D510089564
:10AB2000DF93CF930F92CDB7DEB789830E94215375
:10AB300029812093D51088E491E06FE140E00E94E4
:10AB4000CB580F90CF91DF9108950E94905586E0E9
:10AB50000E94E9530895809362019093630160938A
:10AB60006001709361014115510531F1FA01819144
:10AB700080936B01DA0111968C9180936A01DF0159
:10AB80001196818180936901FD01319611968C9116
:10AB900080936801DF011196818180936701FD0137
:10ABA000319611968C9111978093660181818093E3
:10ABB0006501828180936401089586E196E00E9498
:10ABC000054181E080934725809148259091492552
:10ABD0000196909349258093482581E090E008955F
:10ABE000EF92FF92CF93DF9350914F25252F30E0C6
:10ABF000F901EE0FFF1F3695322F22273795279543
:10AC0000E20FF31FE05BFA4D4081442309F4CEC00C
:10AC10002091390121FDCAC02091DC26222309F4AC
:10AC2000C5C047FF16C00E94D7528091102790914F
:10AC30001127A0911227B09113270196A11DB11DD4
:10AC40008093102790931127A0931227B093132776
:10AC5000ADC04330B0F40E94D75280910C27909140
:10AC60000D27A0910E27B0910F270196A11DB11DB0
:10AC700080930C2790930D27A0930E27B0930F2756
:10AC800095C0C42FD0E022976C177D07B0F40E94C6
:10AC9000D7528091082790910927A0910A27B09157
:10ACA0000B270196A11DB11D8093082790930927BA
:10ACB000A0930A27B0930B2779C0652F70E09B0102
:10ACC000220F331F7695762F662777956795260F87
:10ACD000371F2F5A3A4DB90150E00E94577D2091FD
:10ACE0004F25822F90E0FC01EE0FFF1F9695982FC5
:10ACF000882797958795E80FF91FE053FA4D8081D3
:10AD000080934025822F90E0FC01EE0FFF1F969567
:10AD1000982F882797958795E80FF91FE05BFA4DE4
:10AD200010822F5F20934F25233010F010924F2573
:10AD300080914F2590E0FC01EE0FFF1F9695982F14
:10AD4000882797958795E80FF91FE05BFA4D80817A
:10AD5000882311F00E94DD556091470160934125E1
:10AD600080914625882311F0681710F460934625DA
:10AD700084E070E00E94A1486091402583E070E08B
:10AD80000E94A1488091242790912527A0912627F1
:10AD9000B09127270196A11DB11D80932427909380
:10ADA0002527A0932627B093272702C0C0E0D0E034
:10ADB000CE01DF91CF91FF90EF900895CF93DF9375
:10ADC000EC0188819981009729F024E08B3F92075C
:10ADD00039F505C08BEF94E09983888325C06238EC
:10ADE00019F5109247250E941B480E94784760E899
:10ADF00070E00E94F0551816190644F40E9473473B
:10AE0000E091A706F091A8060995E4CF809144252A
:10AE10009091452501969093452580934425DACF5E
:10AE20001982188283E001C081E0DF91CF910895FB
:10AE300091E0909351100E940F550E94BA540895CA
:10AE40008091390181FD07C085E491E06FE040E029
:10AE50000E94C158089580E10895CF92DF92EF9249
:10AE6000FF920F931F93CF93DF93182F21E020932E
:10AE700051100091DC268091390181FF16C080912C
:10AE80009400909195009093712780937027209360
:10AE90005F272093DB26809139018D7F80933901D4
:10AEA0008091DB268823E1F700E00E942153809106
:10AEB000DC26882309F441C0809161278823E9F1C9
:10AEC000209194003091950080917427909175277E
:10AED00028173907A0F42091442730914527409145
:10AEE0004627509147272C57314E4F4F5F4F2093A5
:10AEF0004427309345274093462750934727209176
:10AF0000940030919500281B390B40E050E0C09030
:10AF10004427D0904527E0904627F09047272C0DF6
:10AF20003D1D4E1D5F1D20934427309345274093C0
:10AF30004627509347271092612789E10E94E953E1
:10AF400086E00E94AC48009751F00E942057C82F1D
:10AF500086E00E94AC4881500E940F5502C0C0E0BC
:10AF6000D0E0809194009091950090937327809306
:10AF7000722781E080936027F89480913901826084
:10AF800080933901809139018D7F80933901612F40
:10AF90006E5F82E590E10E94FC5878948091D626FD
:10AFA0009091D72601969093D7268093D6260E941B
:10AFB000215382E491E060EE45E00E94C158182FD1
:10AFC00086E00E94AC48009719F08C2F0E940F5524
:10AFD000002319F00E94445402C00E944353809100
:10AFE00060278823E9F18091940090919500409129
:10AFF00072275091732784179507A0F480914027FA
:10B0000090914127A0914227B09143278C57914EB0
:10B01000AF4FBF4F8093402790934127A093422783
:10B02000B09343272091940030919500241B350B59
:10B0300040E050E08091402790914127A091422725
:10B04000B0914327280F391F4A1F5B1F20934027C9
:10B050003093412740934227509343271092602713
:10B060008091DC26882361F0809194009091950076
:10B07000909375278093742781E08093612707C0A0
:10B0800082E491E06FE140E023E00E94CB580E940F
:10B09000BA541130E1F01330A9F48091182790913F
:10B0A0001927A0911A27B0911B270196A11DB11D48
:10B0B0008093182790931927A0931A27B0931B27E2
:10B0C00012E00AC0153029F0173031F404C010E046
:10B0D00003C013E001C011E0812F90E0DF91CF9118
:10B0E0001F910F91FF90EF90DF90CF900895CF9335
:10B0F000DF93EB010E94CD549C01009731F4CE0107
:10B100000E942D579C01009749F08091D92690917B
:10B11000DA2601969093DA268093D926C901DF9129
:10B12000CF9108950F931F938091DC26882321F4FB
:10B130000E946F5411E001C010E00E942653863136
:10B1400011F0813119F40091470109C086E491E0C2
:10B150006FE140E00E94C158082F000F080F112333
:10B1600011F00E94D153802F1F910F9108951092DA
:10B17000D8101092D710EFE6F0E0808180628083D3
:10B180000895FC018081862390E002C09595879503
:10B190004A95E2F70895F894FC019081862F8095F6
:10B1A000892330E002C0220F331F4A95E2F726239D
:10B1B000282B208378940895DC01119620917B013F
:10B1C000FC012083215030E0A9014F575E4FE0E899
:10B1D000F1E061916D93E417F507D9F7FC01E058B0
:10B1E000FF4F2F573E4FD9012C9120838F579F4FF0
:10B1F00021E0FC0120830895FC0160938001019609
:10B200006350860F911DA1E8B1E021912D93E817BD
:10B21000F907D9F708951F920F920FB60F920BB648
:10B220000F9211242F933F934F935F936F937F93CC
:10B230008F939F93AF93BF93EF93FF9380914701B9
:10B240008093412520914E2530E0C901880F991F38
:10B250003695322F222737952795820F931F805BD3
:10B260009A4D0E94DC5880914E258F5F80934E2529
:10B27000833010F010924E250E94DD55FF91EF9122
:10B28000BF91AF919F918F917F916F915F914F91FE
:10B290003F912F910F900BBE0F900FBE0F901F90FC
:10B2A00018951F920F920FB60F9211240F900FBE98
:10B2B0000F901F9018951F920F920FB60F921124A6
:10B2C0000F900FBE0F901F9018951F920F920FB600
:10B2D0000F9211240F900FBE0F901F9018951F9280
:10B2E0000F920FB60F9211241092DB260F900FBE13
:10B2F0000F901F9018951F920F920FB60F92112466
:10B300001092DB260F900FBE0F901F9018951F9282
:10B310000F920FB60F9211248F9381E080934725EF
:10B320008F910F900FBE0F901F9018951F920F9244
:10B330000FB60F9211241092DB260F900FBE0F90C4
:10B340001F9018951F920F920FB60F9211248F9392
:10B350009F938091D7109091D81001969093D81018
:10B360008093D7109F918F910F900FBE0F901F90D9
:10B3700018950F931F93CF93DF938091E4269091BC
:10B38000E526A091E626B091E7260196A11DB11D04
:10B390008093E4269093E526A093E626B093E726D3
:10B3A0000E946A5CEC0189ED90E10E94A7410BC00C
:10B3B000D8011296ED91FC911397309709F00995F9
:10B3C000C8010E946D42082F192F0115110581F740
:10B3D000209719F0CE010E94173FDF91CF911F9166
:10B3E0000F9108950E94A4610E941B480E94745A04
:10B3F00088E896E09093DF268093DE260E94675CC3
:10B4000082E090E060E074E040E05EE12FEF31E048
:10B410000E94285C0895CF92DF92EF92FF920F93E3
:10B420001F93CF93DF936C01EB018A0189ED90E1CB
:10B430000E94A7410CC0D7011496ED91FC9115977D
:10B44000309711F0CE010995C7010E946D42E82E98
:10B45000F92EE114F10479F7C601BE01A8010E949A
:10B460001F3FDF91CF911F910F91FF90EF90DF90E1
:10B47000CF900895BC0189ED90E10E942E4208957D
:10B48000BC0189ED90E10E94F5410895CF93DF93CF
:10B49000EC018091E0269091E126A091E226B09106
:10B4A000E3260196A11DB11D8093E0269093E1262D
:10B4B000A093E226B093E326CE010E94815C009720
:10B4C00069F00E949547E0918C06F0918D068BE023
:10B4D0009AE5BE01099521E030E002C020E030E0AD
:10B4E000C901DF91CF9108958BED90E10E94A341B6
:10B4F00008950F93CF93DF93EC017B836A831886C3
:10B500005F834E838BED90E1BE010E942E42E0915D
:10B51000DD10F091DE10309749F04C815D818A8119
:10B520009B81688520E030E001E00995DF91CF91B3
:10B530000F910895BC018BED90E10E94F5410895B3
:10B540000F93DC0118961C921897E091DD10F09192
:10B55000DE10309759F012968D919C91139760E010
:10B5600040E050E020E030E000E009950F910895C0
:10B570000F93DC01AB0114962D913C91159781E05E
:10B5800018968C93189715967C936E931497E09168
:10B59000DD10F091DE10309739F012968D919C916C
:10B5A000139761E000E009950F9108950F93DC0176
:10B5B000E091DD10F091DE10309769F014962D9136
:10B5C0003C91159712968D919C91139718966C91BA
:10B5D000A90101E009950F910895E091DF10F09124
:10B5E000E010309709F0099508959093E01080934A
:10B5F000DF1008959093DE108093DD1008958BED99
:10B6000090E10E94A7410895EF92FF920F931F933C
:10B61000CF93DF938C01EB017A018BED90E10E94D7
:10B62000A74115C0DC0112962D913C9113972C1760
:10B630003D0759F41696ED91FC911797309761F0FC
:10B64000B801AE019701099507C00E946D42282FED
:10B65000392FC901009731F7DF91CF911F910F91D9
:10B66000FF90EF9008950895AF92BF92CF92DF922E
:10B67000EF92FF920F931F93DF93CF9300D0CDB73C
:10B68000DEB75B010E947847FC01008111811A83BB
:10B6900009830C30110518F4EE24FF242EC000D0CD
:10B6A00000D080E596E0EDB7FEB7928381831483E6
:10B6B00003830E94D67D0F900F900F900F9020C0B3
:10B6C0000E947847F701EE0FFF1FEE0FFF1FE80FF4
:10B6D000F91FC280D3800E9478470894E11CF11CB6
:10B6E000F701EE0FFF1FEE0FFF1FE80FF91F40815C
:10B6F0005181C501B6010E94045BE016F10600F31A
:10B700000F900F90CF91DF911F910F91FF90EF90CD
:10B71000DF90CF90BF90AF900895CF93DF93CCEFA1
:10B72000D0E16091121170911311CE014FEB5BE5E6
:10B7300020E030E00E946C440E94A16160911211EF
:10B74000709113110E943E7ABC01CE01409744EDE6
:10B750005BE520E030E00E946C44DF91CF910895DA
:10B760000F93013051F480910C1190910D11909331
:10B770001311809312110E948D5B0F910895809197
:10B780001211909113112091101130911111880F05
:10B79000991F2817390708F4C90190931311809352
:10B7A00012110E948D5B0895EF92FF92CF93DF9369
:10B7B0000E941B480E947847E82EE7017E01F92E7F
:10B7C000E701198218820E94FF5A26C02881398118
:10B7D000F901EE0FFF1FEE0FFF1FEC0FFD1FDC0145
:10B7E00012964D915C911397538342832F5F3F4F85
:10B7F000F901EE0FFF1FEE0FFF1FEC0FFD1F149658
:10B800004D915C91159751834083398328830E9421
:10B810006D42282F392FC901009721F0FC012085A6
:10B820002223A1F688819981880F991F880F991F7B
:10B8300002960E94734788819981009721F081EEDA
:10B8400090E10E94EA3EDF91CF91FF90EF90089542
:10B85000EF92FF920F931F93CF93DF93FC018B0125
:10B860007A01E90181EE90E1BF014DE656E00E94C8
:10B87000CC3E10930D1100930C11F0920F11E09239
:10B880000E11D0931111C093101180EB9BE50E9413
:10B89000FA5ADF91CF911F910F91FF90EF90089589
:10B8A000CF93DF93CCEFD0E1CE010E94F344CE01E1
:10B8B00040970E94F344CE014B970E94E73EDF91F0
:10B8C000CF910895809112119091131108950E94C3
:10B8D0002B3F0895EF92FF92CF93DF93E091710693
:10B8E000F09172060995EC01009729F06A817B813D
:10B8F00081E00E94A148CE01DF91CF91FF90EF90AF
:10B9000008950F931F93CF93DF938C01E0917306FB
:10B91000F09174060995EC01F8016281738181E070
:10B920000E94A14821E030E0209711F420E030E0AF
:10B93000C901DF91CF911F910F910895E091750694
:10B94000F091760609950895FC0120E030E004C0EE
:10B950008181280F311D329680818823C9F7C90162
:10B960000895FC01818190E0308120E0822B932BAF
:10B9700002C0880F991F6A95E2F7892F9927FA016B
:10B98000E958F94F208130E08223932328E030E00A
:10B99000241B350B02C0969587952A95E2F70895EA
:10B9A0006F927F928F929F92AF92BF92CF92DF92CF
:10B9B000EF92FF920F931F93CF93DF936C017B0164
:10B9C0005A0189012830310544F4CB01BA01A9019B
:10B9D0000E94B15CF601808341C0390133E0759467
:10B9E00067943A95E1F74115510521F04C01C0E00B
:10B9F000D0E016C0DB01FC01C0E0D0E08D91819366
:10BA00002196C615D705D4F3A8014770507041158B
:10BA1000510521F1C7018C0F9D1F60E070E019C036
:10BA2000C7018C0F9D1FB50148E050E00E94B15C3A
:10BA3000F40181934F012196C615D7058CF3A80117
:10BA4000477050704115510549F0C7018C0F9D1F7B
:10BA5000B5010E94B15CCC0DDD1D8883DF91CF91D3
:10BA60001F910F91FF90EF90DF90CF90BF90AF901C
:10BA70009F908F907F906F9008954F925F926F92FA
:10BA80007F928F929F92AF92BF92CF92DF92EF926E
:10BA9000FF920F931F93DF93CF9300D000D0CDB7C9
:10BAA000DEB70E947847E82E092F82E090E00E94DE
:10BAB0005447009709F464C0EE2DF02F918180E087
:10BAC0002081820F911D0E943F3F7C01009709F465
:10BAD00059C00E9478473C01F7014681242F30E08D
:10BAE0002770307081E090E02115310511F480E07D
:10BAF00090E0469546954695840F911D0E945447C7
:10BB00000097F1F1F70104811581CC24DD2453E085
:10BB1000452E512C4C0E5D1E4E010894811C911C2B
:10BB20002AC0F801A180BB24B60143E07595679552
:10BB30004A95E1F7660D771DA60147705070883170
:10BB400050F0C40195010E94D05CF8018081B401DD
:10BB50000E94B5480CC01C821B82C20195010E9444
:10BB6000D05C6B817C81F80180810E94A148CA0C65
:10BB7000DB1C0E5F1F4FF8018081882391F602C005
:10BB8000EE24FF24C7010F900F900F900F90CF91DC
:10BB9000DF911F910F91FF90EF90DF90CF90BF90BA
:10BBA000AF909F908F907F906F905F904F9008958F
:10BBB000FC0150E080E190E0861B970B821B930B09
:10BBC00002C0440F551F8A95E2F78081852B808340
:10BBD0008181842B818308956F927F928F929F92AF
:10BBE000AF92BF92CF92DF92EF92FF920F931F938B
:10BBF000CF93DF938C015B016A0179012830310515
:10BC000024F4C801FA01408156C0390163E07594FB
:10BC100067946A95E1F7A114B10421F04A01C0E0EC
:10BC2000D0E021C0DA01F80180E090E02D9121936D
:10BC3000019686159705D4F397012770307021156A
:10BC40003105D9F1F601E80FF91F408150E068E0B5
:10BC500070E0621B730B02C0559547956A95E2F739
:10BC6000800F911F26C0F40141914F01C8018C0F34
:10BC70009D1FB50128E030E00E94D85D2196C615D1
:10BC8000D7058CF397012770307021153105A9F085
:10BC9000F601EC0FFD1F408150E0C5010896821BA4
:10BCA000930B02C0559547958A95E2F7C8018C0F12
:10BCB0009D1F60E070E00E94D85DDF91CF911F91E1
:10BCC0000F91FF90EF90DF90CF90BF90AF909F903B
:10BCD0008F907F906F9008954F925F926F927F92B6
:10BCE0008F929F92AF92BF92CF92DF92EF92FF928C
:10BCF0000F931F93DF93CF9300D0CDB7DEB78C01A6
:10BD0000DC0116964C911697842F90E08770907006
:10BD100021E030E0009711F420E030E046954695B0
:10BD200046957901E40EF11CC70102960E94E04796
:10BD3000009709F453C00E948047FC01D801129675
:10BD40008C911297808313968C9181830E948047F7
:10BD5000F2E06F2E712C680E791EC30160E070E076
:10BD6000A7010E94607DF801C480D58000E010E04A
:10BD70002E010894411C511C2AC0D60111968C90AA
:10BD8000119799247801E3E0F594E794EA95E1F7B7
:10BD9000E60CF71C77E0A72EB12CA022B122883147
:10BDA00030F00E94BF48AC01C701B50107C00E9436
:10BDB000AC489A838983C701B501A20194010E940E
:10BDC000EC5D080D191DE2E0F0E0CE0EDF1ED6019D
:10BDD0008C91882391F621E030E002C020E030E031
:10BDE000C9010F900F90CF91DF911F910F91FF909C
:10BDF000EF90DF90CF90BF90AF909F908F907F900B
:10BE00006F905F904F900895E091A506F091A6067F
:10BE100009950895E0914E06F0914F060995089511
:10BE2000E091A906F091AA0609950895E091AB0664
:10BE3000F091AC060995089580E090E0089508958A
:10BE4000E0913006F091310609950895009731F0A0
:10BE5000E0913006F091310609950895E09132069F
:10BE6000F09133060995089580E090E008950F93CE
:10BE70001F93DF93CF93CDB7DEB7E0970FB6F8945B
:10BE8000DEBF0FBECDBF0E94CA478C010E9478471B
:10BE9000602FAE014F5F5F4F0E946A67882309F4ED
:10BEA00045C088A99801281B3109C9010E9454473F
:10BEB0000097E1F12E81222371F18A859B853BEA6F
:10BEC0008D3C930721F03FEF8F3F930779F52230A8
:10BED00041F088E090E007C0019722912F3F41F0A8
:10BEE0000BC082E090E0FE01E80FF91F3C96F4CF12
:10BEF000181619068CF30FC089E1BE01645F7F4FED
:10BF00000E94B54889E10E94BF486DEE74E20E942C
:10BF10007D3E009759F088E1BE016A5E7F4F0E9426
:10BF2000B548E0918E06F0918F060995E0960FB620
:10BF3000F894DEBF0FBECDBFCF91DF911F910F915F
:10BF40000895AF92BF92CF92DF92EF92FF920F933C
:10BF50001F93DF93CF93CDB7DEB7E0970FB6F8947A
:10BF6000DEBF0FBECDBF6C018B01FE01319680E3B9
:10BF7000DF011D928A95E9F781E089838CE00E94B8
:10BF8000AC488C831D821F828091161189878F5F38
:10BF90008093161183E0E82EE8868DEC9BEA9B8760
:10BFA0008A8789E10E94BF4868E675E00E947D3E6D
:10BFB000009731F082E08E838FEF8C878D8709C0E8
:10BFC00089E10E94BF48BC01CE010C960E94743EDC
:10BFD000EE828DEC9BEA9D8B8C8BCE0146966DEEAE
:10BFE00074E20E94743E0E9478479FA78EA70E9429
:10BFF000CA4788AB7E010894E11CF11CC7010E946E
:10C000006166A82E90E00E94E047009741F10E94EF
:10C010008047BC01C7014A2D0E947F66A09026067A
:10C02000B09027060E9480477C010E94D447BC0143
:10C03000C701F5010995C114D10489F0009721F0D9
:10C040008130910561F404C0C80160E070E003C074
:10C05000C80164E070E041E050E0F6010995E09627
:10C060000FB6F894DEBF0FBECDBFCF91DF911F9109
:10C070000F91FF90EF90DF90CF90BF90AF90089519
:10C080000E94A16180931611E0913006F091310673
:10C0900009950895EF92FF92CF93DF93E82EE70181
:10C0A0007E01F92EE70104C060E070E00E94E240EA
:10C0B000899199910097C1F7DF91CF91FF90EF900F
:10C0C0000895EF92FF92CF93DF93E82EE7017E0170
:10C0D000F92EE70102C00E942740899199910097AB
:10C0E000D1F7DF91CF91FF90EF900895CF93DF9339
:10C0F000EC017B836A830E94335199838883DF91AB
:10C10000CF910895FC018081918122813381820F3A
:10C11000931F918380830895CF93DF93EC010E9456
:10C12000335199838883DF91CF910895CF93DF9323
:10C13000EC010E94335128813981821B930B0196B7
:10C1400021E030E04A815B814817590710F020E078
:10C1500030E0C901DF91CF910895EF92FF92CF9324
:10C16000DF93FC01C281D38180819181C80FD91FE7
:10C170000E943351C81BD90BCE01DF91CF91FF90A4
:10C18000EF900895CF93DF93E6E6F7E2C8E2D7E2B7
:10C19000AAE5B7E211921192199219921992199285
:10C1A0001D9287E2EE37F807A9F7DF91CF91089546
:10C1B0000F931F93CF93DF93FC01DC01A65AB84D78
:10C1C0008C91882339F10091940010919500EF0132
:10C1D000CC0FDD1FCC0FDD1FC85DD84DDF01AA0FCE
:10C1E000BB1FAA59B84D8D919C9111979801281B9E
:10C1F000390B40E050E0688179818A819B81260F6C
:10C20000371F481F591F288339834A835B83119640
:10C210001C930E93EE0FFF1FEE0FFF1FE85DF84D0E
:10C220006081718182819381DF91CF911F910F9104
:10C23000089560E070E0CB010895FC01EE0FFF1F50
:10C24000EE0FFF1FE85DF84D4083518362837383D7
:10C250000895EF92FF920F931F93CF93DF932AE5F8
:10C2600037E2C8E2D7E2E6E6F7E2D9018D919D0117
:10C270008823C9F04091940050919500808191816C
:10C280007A01E81AF90A00E010E088819981AA8110
:10C29000BB818E0D9F1DA01FB11F88839983AA8328
:10C2A000BB835183408324963296B7E226363B0700
:10C2B000E1F6DF91CF911F910F91FF90EF900895DC
:10C2C0000E94DE6508950F931F93FC01CB014091FE
:10C2D00017115091181133832283158304837183BE
:10C2E0006083F0931811E09317114115510511F473
:10C2F0000E94F86580E090E01F910F910895809171
:10C300001711909118110097C1F010921811109206
:10C310001711DC0114966D917C9115971296ED9191
:10C32000FC9113970995E0911711F091181130972E
:10C3300021F0808191810E94F86508950E942C7BF4
:10C3400008950E94277B08958FEA96E00E941B4182
:10C3500087EB96E00E941B410895EF92FF92CF93E6
:10C36000DF930E9487470097C9F087EB96E00E9411
:10C370003B41E82EE7017E01F92EE701209731F1DC
:10C380000E94CA47998388830E94C5479B838A83FA
:10C39000C70104960E94F3468CAB18C08FEA96E062
:10C3A0000E943B41EC017E01F92EE701209771F0DC
:10C3B000C70102960E940A4799838883B7016E5489
:10C3C0007F4FC7018E579F4F0E947748CE01DF9164
:10C3D000CF91FF90EF900895BC016E547F4F8E5720
:10C3E0009F4F0E9477480895CF93DF93EC018FEA27
:10C3F00096E0BE010E948641009719F08FEA96E010
:10C4000009C087EB96E0BE010E948641009729F0A3
:10C4100087EB96E0BE010E946141DF91CF910895C4
:10C42000EF92FF92CF93DF93EC018FEA96E0BE018B
:10C430000E948641009779F068817981CE01029649
:10C440000E944448BE016E547F4FCE018E579F4FCD
:10C450000E948C481BC087EB96E0BE010E9486417B
:10C460000097A1F00E941B48688179818A819B8195
:10C470000E9444488CA990E00E94E0470E948047B7
:10C480004CA92496BE0150E00E94577DDF91CF91C8
:10C49000FF90EF900895EF92FF92CF93DF93EC011E
:10C4A0008FEA96E0BE010E948641009711F0229625
:10C4B0000DC087EB96E0BE010E948641009721F0F7
:10C4C0000A80DB81C02D02C0C0E0D0E0CE01DF9148
:10C4D000CF91FF90EF900895FC01808191810895A4
:10C4E00070E06F5B7F4F660F771F680F791FCB017E
:10C4F0000895E62FF0E0EF5BFF4FEE0FFF1FE80F10
:10C50000F91F80819181089508958FE697E10E9437
:10C510009143009721F08FE697E10E947C430895B4
:10C52000E0917C17F0917D17309711F009950895EF
:10C5300080E00895EF92FF920F931F93CF93DF93C4
:10C54000EC018A0188819981009731F023E08C30D9
:10C55000920709F006C12BC080E00BC0E82FF0E085
:10C56000EE0FFF1FEE0FFF1FE35AF84E11821082ED
:10C570008F5F843098F38093771780919E0E90910F
:10C580009F0E90936E1780936D170E9420408093AA
:10C590007E278FE697E160E470E00E9466430E9488
:10C5A000F9688CE093E09983888381E0DDC0623094
:10C5B00009F4B9C0633030F4662309F489C06130EE
:10C5C00081F79CC0673819F0683859F741C010925C
:10C5D00078174DE5E42E47E1F42E18C0F70182816B
:10C5E00093818017910749F4808191810E94406A6C
:10C5F000F701118210821382128284E090E0E80E2B
:10C60000F91E809178178F5F809378178091781743
:10C61000843020F3EEE8FCE2848D958D801791073D
:10C6200019F4158E148E118EB0969DE2EE30F90736
:10C6300099F7E4E2FDE2818592858017910711F474
:10C64000158214823D962DE2E63AF207A1F7A9CFB2
:10C6500087E14F36580709F0A4CFCA010E949143E1
:10C66000009709F49ECF109278172DC0F0E035E0C6
:10C67000EE0FFF1F3A95E1F7E257F34D818D8823C6
:10C68000E9F08FE697E10E947C438091781790E073
:10C6900025E0880F991F2A95E1F78257934D9093D3
:10C6A0008D2C80938C2C82E00E94746A80917F276D
:10C6B00090918027009711F00E94906280917817E6
:10C6C0008F5F80937817E0917817E43078F269CF24
:10C6D0004115510509F465CF50938D2C40938C2C56
:10C6E00083E00E94746A80917F2790918027009751
:10C6F00011F00E9490620E94856253CF411551054E
:10C7000009F44FCF5093892C4093882C85E00E94E8
:10C71000746A80917F2790918027009709F441CF18
:10C720000E9490623ECF80917F2790918027009752
:10C7300009F437CF80919027863031F48091A82773
:10C7400081FF02C00E94856281E00E94746A80912C
:10C750007F2790918027009709F423CF0E94C3641C
:10C7600020CF1982188283E0DF91CF911F910F9122
:10C77000FF90EF90089590937D1780937C17089514
:10C7800020919E0E30919F0E60E0EDE5F7E113C021
:10C79000408151814817590761F442815381421702
:10C7A000530739F460937B17118210820E94406A0C
:10C7B000089534966F5F643058F360937B17089543
:10C7C00040E0EDE5F7E116C0542F5F5F2081318135
:10C7D0002115310569F440937A1791838083209164
:10C7E0009E0E30919F0E338322830E945A6A0895D1
:10C7F0003496452F443040F340937A170895FC0156
:10C8000080919E0E90919F0E958F848F778F668F6B
:10C810000895FC0180919E0E90919F0E92878187D2
:10C82000748763870895CF93DF93EA010E94BC6900
:10C83000FC01009741F080919E0E90919F0E92878F
:10C840008187D487C387CF01DF91CF9108950F935C
:10C850001F93DF93CF9300D000D0CDB7DEB78C010C
:10C86000AB018FEF89838A838B838C83CE01019602
:10C87000B8010E941364FC01009711F01583048332
:10C88000CF010F900F900F900F90CF91DF911F91DC
:10C890000F9108958CEC96E062E040E050E00E9439
:10C8A000D3401092802710927F270895AC018CEC22
:10C8B00096E061E00E94B0400895AC018CEC96E0F7
:10C8C00060E00E94B04008950F931F93CF93DF93D1
:10C8D000EA010E9432698C01009761F080919E0EFE
:10C8E00090919F0EF801958F848FD78FC68FC801C6
:10C8F0000E945D64C801DF91CF911F910F9108954F
:10C90000CF93DF93A0918C2CB0918D2C109719F0C0
:10C91000ED016C9605C0C091882CD091892C299688
:10C920008091872C86FF22C01092791740E0EDE5B8
:10C93000F7E116C02081318114968D919C91159755
:10C940002817390759F482819381009739F0409371
:10C950007917998388831B821A8206C034964F5FA9
:10C96000443040F3409379170E9485628881998111
:10C97000009731F04A815B8160917E270E94D3400D
:10C98000DF91CF9108950F931F93CF93DF93809101
:10C990009027863009F074C080917F27909180277E
:10C9A00025E08030920709F06BC0C4E9D2E0D09353
:10C9B0008027C0937F2702E00093892714E9109312
:10C9C0008A271092AC271092AB270E94F1688095BD
:10C9D00090959093AC278093AB271092922710925A
:10C9E00091270E94E068809590959093922780937C
:10C9F00091270E949062D0938027C0937F27009355
:10CA0000892710938A2790918A2C80918B2CE92F6B
:10CA1000F82FDF01A459BD4F8CE692E00D900192F2
:10CA20000197E1F78FE997E26CE672E00E94846873
:10CA30008091832780939F27809184278093A027CC
:10CA4000809185278093A127809186278093A227B4
:10CA50001092AC271092AB270E94F16880959095B8
:10CA60009093AC278093AB27109292271092912736
:10CA70000E94E068809590959093922780939127EB
:10CA80000E949062DF91CF911F910F910895282FFE
:10CA9000392FF90120E030E080E0A8E112C0419197
:10CAA00098E0542F5827B52FB17050FD8A278695EE
:10CAB000B13009F48068915011F04695F2CF2F5FA4
:10CAC0003F4F2617370759F708951F920F920FB659
:10CAD0000F920BB60F9211242F933F934F935F93B6
:10CAE0006F937F938F939F93AF93BF93EF93FF9336
:10CAF000809194009091950090936B2780936A2782
:10CB000081E080935C2780917100807D809371002B
:10CB10000E947F6180915C278823E9F180919400D5
:10CB20009091950020916A2730916B278217930787
:10CB3000A0F48091302790913127A0913227B091B5
:10CB400033278C57914EAF4FBF4F80933027909330
:10CB50003127A0933227B09333278091940090918E
:10CB60009500821B930BA0E0B0E02091302730911C
:10CB700031274091322750913327820F931FA41FF2
:10CB8000B51F8093302790933127A0933227B0931D
:10CB9000332710925C27FF91EF91BF91AF919F9146
:10CBA0008F917F916F915F914F913F912F910F9056
:10CBB0000BBE0F900FBE0F901F9018959FB7F89463
:10CBC000E1E7F0E08081807D808388B38F6288BB5D
:10CBD00010929000E1E9F0E0108210929200109221
:10CBE0009500109294008081856080839FBF089596
:10CBF0002FB7F894909399008093980088B38F6230
:10CC000088BBE1E7F0E08081826080832FBF0895D8
:10CC1000EF92FF92CF93DF93FC01DB0185E0EB0104
:10CC200019928A95E9F7858190E08370907000975A
:10CC300011F082E08C93878190E083709070009770
:10CC400021F082E012968C931297858190E0837098
:10CC50009070009799F0878190E0837090700097B2
:10CC600069F023893489818592852817390731F441
:10CC700081E0848312961C92129701C014828581F0
:10CC800083708250823030F4C82FD0E0CA52D94F1E
:10CC9000888101C080E011968C931197E781E37041
:10CCA000E250E23028F4F0E0EA52F94F808101C00E
:10CCB00080E013968C931397DF91CF91FF90EF90C4
:10CCC0000895DF93CF9300D000D00F92CDB7DEB799
:10CCD000BE016F5F7F4F0E94086689819A81890F2C
:10CCE0008D5F9B81890F9C81890F9D81890F0F909A
:10CCF0000F900F900F900F90CF91DF910895AF920A
:10CD0000BF92CF92DF92EF92FF920F931F93DF9328
:10CD1000CF9300D000D000D0CDB7DEB78C017B011F
:10CD2000BE016F5F7F4F4E830E940866C9809A8163
:10CD3000A92EBB24DB808C81682F70E095012C0D1F
:10CD4000311D2D5F3F4F2D0D311D260F371F5D818A
:10CD5000250F311D4E8150E0421753070CF4A8C037
:10CD6000D80111964C91119750E041705070E3E05A
:10CD7000440F551FEA95E1F712962C91129730E077
:10CD80002170307054E0220F331F5A95E1F7242BA5
:10CD90003C913770232B13963C911397E32FF0E0CF
:10CDA000E170F07045E0EE0FFF1F4A95E1F72E2B82
:10CDB00014963C911497E32FF0E0E170F07036E0A8
:10CDC000EE0FFF1F3A95E1F72E2BF7012083159602
:10CDD0004C91159750E043705070440F551F440F0D
:10CDE000551F16962C91169730E02370307054E042
:10CDF000220F331F5A95E1F7242B17963C91179772
:10CE00003295330F330F307C322B318318962C91AF
:10CE100018972283FC2DF23069F419962C91D701D2
:10CE200013962C931397F801228514962C9314973C
:10CE300045E001C043E0E92FF0E03B96E00FF11F31
:10CE4000542F0AC09701250F311DC290D901CC92F1
:10CE50005F5F0894A108B108A114B10499F7940F79
:10CE6000BD2DB23089F4F701E90FF11DD8015396B9
:10CE70002C91539720839F5FF701E90FF11D549682
:10CE80002C91549720839F5FE82FF0E07596E00F78
:10CE9000F11F292F08C0D701A20FB11D32913C9379
:10CEA0002F5F6150704061157105A9F7890F01C0AE
:10CEB00080E026960FB6F894DEBF0FBECDBFCF91AF
:10CEC000DF911F910F91FF90EF90DF90CF90BF9077
:10CED000AF900895BF92CF92DF92EF92FF920F939F
:10CEE0001F93CF93DF937C01D62EEA01633008F4C1
:10CEF000ADC0FC018081B82EB294B694B694B3E074
:10CF0000BB22F1E0BF22F7019181292F26952695BA
:10CF10002370C92EC294C694C694A3E0CA22382FA7
:10CF200037703883382F369536953695317039837A
:10CF3000382F329531703A838295869581708B8334
:10CF4000BC822D83892F829583708E83CF828281CC
:10CF5000888787010D5F1F4F222361F1F8019181BE
:10CF600080E0F7013381830F911D9A8789878701BC
:10CF70000B5F1F4F223081F4CA010B9668E675E003
:10CF80000E94743EF80181818B87F70185818C872F
:10CF90008701095F1F4F16C02330A1F4F7013D96AA
:10CFA000DA011B9682918D93E017F107D9F7085F9C
:10CFB0001F4F08C0CA010B9668E675E00E94743ED8
:10CFC0001A861986CC2089F1BB2059F4F801918189
:10CFD00080E02081820F911D9C8B8B8B0E5F1F4FF9
:10CFE00004C089859A859C8B8B8BFC2DF23071F463
:10CFF000CE01459668E675E00E94743EF801818195
:10D000008D8B80818E8B0E5F1F4F17C0FC2DF330F0
:10D01000A1F4085F1F4FD801FE01759680E09E9134
:10D0200091938F5F8830D9F708C0CE01459668E6A6
:10D0300075E00E94743E1C8A1B8A802F8E199D2DDC
:10D04000981B9FA71EA70DA7D81608F480E0DF91B4
:10D05000CF911F910F91FF90EF90DF90CF90BF90F5
:10D0600008959C0141505040460F571FDB0110C0EE
:10D07000FC91E0E011968C911197BF01680F711D32
:10D08000260F371F2617370710F42F5F3F4F1296D2
:10D09000A417B50768F3A417B50749F49C9180E07D
:10D0A000280F391F2817390710F42F5F3F4FC90188
:10D0B0000895CF93DF9390918A27C92FD0E064978A
:10D0C0003091892720E0C20FD31F9E01280F311D08
:10D0D000C90163E977E248E050E00E9431686BE9FA
:10D0E00077E2AE010E943168009719F0382F292F9E
:10D0F00002C02FEF3FEFC901DF91CF9108959093C8
:10D100008D1780938C170895FC014381460F40933F
:10D110008627872F99272281280F20938527A18191
:10D12000A093842750815093832730E02817390734
:10D1300048F48A2F8F5F80938427882319F45F5FD8
:10D1400050938327842F90E070708617970798F488
:10D15000809185278F5F80938527882361F4809154
:10D1600084278F5F80938427882329F480918327E5
:10D170008F5F809383270895BC0180918C2C9091C0
:10D180008D2C08960E948468E0918C2CF0918D2C57
:10D19000809183278087809184278187809185274C
:10D1A000828780918627838708959C01AB0180E068
:10D1B00090E0B9010E943168382F292FC9010895E4
:10D1C00080E090E067E877E244E150E00E94316857
:10D1D000009719F0382F292F02C02FEF3FEFC90118
:10D1E000089586E00E945968089581E10E94596877
:10D1F000089580E009C0E82FF0E0EE0FFF1FE25F26
:10D20000F24D118210828F5F8430A8F380E00BC052
:10D21000E82FF0E095E0EE0FFF1F9A95E1F7E25757
:10D22000F34D118E8F5F843098F380E094E09093FB
:10D230008F1780938E1740E08DE090E00EC0242F72
:10D2400030E0289FF001299FF00D389FF00D112448
:10D25000EC5DF24D158214824F5F4A3080F34093AB
:10D260008A17089520918E1730918F172F5F3F4FA7
:10D270004DE72030340710F020E030E1522F432FEB
:10D28000A0E013C0EA2FF0E0B5E0EE0FFF1FBA9563
:10D29000E1F7E257F34DB18DBB2331F00480F58106
:10D2A000E02DE417F50711F3AF5FA43059F7309381
:10D2B0008F1720938E1710928A1720E0E0E0F0E09D
:10D2C0001EC0A22FB0E035E0AA0FBB1F3A95E1F7D0
:10D2D000A257B34D59963C915997332321F420938B
:10D2E0008A17FD0110C0373049F4309731F05A9653
:10D2F0004C915A97328D341708F4FD012F5F24307A
:10D3000000F320938A173097A9F122E0218F209112
:10D3100084172487209185172587209186172687D3
:10D3200020918717278728ED34E0338B228B358BAC
:10D33000248B21E030E0318B208B138E21E0228F73
:10D3400023E0208F168A20E1278B20918E173091C1
:10D350008F173227232732273583248377836683E9
:10D36000DC012D913D914D915C9113972083318388
:10D3700042835383CF0108950F931F93CF93DF937D
:10D3800020918E1730918F174DE050E02F5F3F4F67
:10D39000ADE720303A0710F020E030E1B22FA32FA4
:10D3A00010E012C0C12FD0E0C49FF001C59FF00D66
:10D3B000D49FF00D1124EC5DF24D0480F581E02D39
:10D3C000EA17FB0719F31F5F1A3061F730938F17C5
:10D3D00020938E1710E02DE030E01AC0012F0F5F70
:10D3E000C12FD0E0C29FF001C39FF00DD29FF00D7E
:10D3F0001124EC5DF24DDF011496448155814115F5
:10D40000510529F410938A17309749F433C0102F2F
:10D410001A3020F310938A17E0E0F0E02BC020913F
:10D420008E1730918F1732272327322711963C937E
:10D430002E9377836683009729F4108211821282DB
:10D44000138209C0DC012D913D914D915C912083A7
:10D450003183428353838DE090E0C89FD001C99F00
:10D46000B00DD89FB00D1124AC5DB24D80E418967C
:10D470008C931897CF01DF91CF911F910F91089551
:10D4800040E013C0E42FF0E0542F5F5FEE0FFF1F6A
:10D49000E25FF24D208131812817390729F440934A
:10D4A0008A17118210820895452F443058F3409313
:10D4B0008A17089540E013C0E42FF0E0542F5F5F17
:10D4C000EE0FFF1FE25FF24D208131812115310502
:10D4D00029F440938A17918380830895452F44301F
:10D4E00058F340938A170895EF92FF920F931F937A
:10D4F000CF93DF93C0918C2CD0918D2C843009F484
:10D50000F7C10FEA17E210938B2C00938A2C10932B
:10D51000822700938127833071F4898D90E08F708A
:10D5200090708330910509F074C0888999890097BB
:10D5300009F02FC78DC0823009F08EC08091871707
:10D540008F5F80938717882399F4809186178F5F68
:10D5500080938617882361F4809185178F5F80936D
:10D560008517882329F4809184178F5F809384170F
:10D570001092802710927F271092232D1092222D37
:10D58000898D873011F0853041F48A8D8F5F8A8FC5
:10D59000843109F0FEC6198EFCC6882309F4F9C649
:10D5A000288939892115310509F44EC09A8D292F12
:10D5B00021502A8F992309F0ECC69B8D983031F0C9
:10D5C000282F2150223048F4953039F4198E80E804
:10D5D0008093872C0E94806495C5953048F423E0A1
:10D5E00030E0092E02C0220F331F0A94E2F701C077
:10D5F00020E32A8F9F5F9B8F90E08F709070833025
:10D600009105E1F0843091054CF48130910509F4E5
:10D6100061C38230910509F0BCC60DC0863091050A
:10D6200009F40CC58830910509F408C584309105CA
:10D6300009F0AFC603C51092A8274FC384E08093BA
:10D64000872C0E94806490C58F70833009F0A1C63A
:10D6500088E08093872C4BC5853019F5E091882CA4
:10D66000F091892C84819581009709F492C61092DB
:10D670008D2C10928C2C0C50104010938B2C0093FE
:10D680008A2C10938227009381271092232D1092C9
:10D69000222D1092802710927F2788E08093872C7C
:10D6A00025C10852104080918727853409F071C642
:10D6B0009091892780E020918A277C01E20EF11C5D
:10D6C00080917F27909180278E159F0508F461C671
:10D6D000F0928027E0927F2780918D2790E08F73D2
:10D6E0009070009709F055C680918E27882309F025
:10D6F00050C680911E2D90911F2DC091DC06D091B7
:10D70000DD068C179D0759F44091202D5091212D55
:10D710002091DE063091DF0642175307A1F02091D9
:10D720009727309198272817390709F032C620919A
:10D73000992730919A278091202D9091212D28179B
:10D74000390709F026C60E94E0682FEF8F3F920745
:10D7500009F01FC680919027863009F431C18131CC
:10D76000E9F1813009F015C680919B27883009F0D6
:10D7700010C610929B2780919D2790919E274FEF76
:10D78000873F940710F0099601C0089690939E2752
:10D7900080939D278091932790919427A09195271E
:10D7A000B09196278093972790939827A0939927D5
:10D7B000B0939A2780911E2D90911F2DA091202D1E
:10D7C000B091212D8093932790939427A093952730
:10D7D000B093962780E4F8018087B8C5C7014C97BD
:10D7E0009093802780937F2783EA97E290938B2CF6
:10D7F00080938A2C8091A1279091A227009739F0DD
:10D800000E94F568FFEF8F3F9F0709F0C2C5209186
:10D810009D2730919E272115310509F4BAC584E270
:10D820009DE29093892C8093882C6091DE06709104
:10D83000DF064091D8065091D9060091DA06109182
:10D84000DB0639C084819581009781F1281739075B
:10D8500069F586819781009739F0A0919B27B09157
:10D860009C27A817B90711F5808191818C179D0716
:10D8700029F4A281B381A617B70739F18417950758
:10D8800029F4A281B381A017B107F9F0A0919327E1
:10D89000B0919427A817B90749F4A0919527B091A2
:10D8A000962782819381A817B90779F03D96F09366
:10D8B000892CE093882CE091882CF091892C8DE2C2
:10D8C000E63AF80708F4BECF64C510928D2C10928A
:10D8D0008C2C82E08093872C83EA97E290938227B6
:10D8E000809381271092232D1092222D0E94806414
:10D8F0008091222D9091232D009709F44AC59C0117
:10D90000245E3F4F3093802720937F2730938927D1
:10D9100020938A27E091882CF091892C20852093F0
:10D920008F2721E120939027089698278927982709
:10D930009093A02780939F271092A2271092A1274F
:10D940008481958190939C2780939B2786819781E2
:10D9500090939E2780939D2780911E2D90911F2D3F
:10D96000A091202DB091212D8093932790939427FF
:10D97000A0939527B093962780819181A281B3814E
:10D980008093972790939827A0939927B0939A27ED
:10D990008FEA97E290938B2C80938A2C0E94F568F3
:10D9A000809590959093A2278093A127009709F0E6
:10D9B000CDC48FEF9FEF9093A2278093A127C6C479
:10D9C0000E94F168EFEF8F3F9E0709F0E2C480915B
:10D9D0009D2790919E27009709F4DBC420919B27F7
:10D9E00030919C272115310509F4D3C4CEE8DCE23F
:10D9F000498D4423E9F06C817D8186179707C1F436
:10DA00006E817F812617370799F4E0919327F09173
:10DA1000942768817981E617F70751F4E0919527FB
:10DA2000F09196276A817B81E617F70709F46DC1AB
:10DA3000A096FDE2CE30DF07D9F62091A8272F73FC
:10DA40002230B9F4909389178093881740E00DC075
:10DA5000E42FF0E0EE0FFF1FE25FF24D20813181F5
:10DA60004F5F8217930709F46EC0443088F34093E8
:10DA70008A178091A82782FD8CC484E1F80181A3D4
:10DA800088E290E09093802780937F2780E580A3B1
:10DA90008091A2279091A627938F3091A1279091F2
:10DAA000A527928F368F2091A0279091A427918F40
:10DAB000258F90919F2790938A174091A327408F9D
:10DAC000948F8F5F878F882361F4832F8F5F868F7A
:10DAD000882339F4822F8F5F858F882311F49F5F0D
:10DAE000948F80919B2790919C2790938917809386
:10DAF000881720919D2730919E27F801358B248B24
:10DB0000978B868B8091932790919427A09195274E
:10DB1000B09196278093972790939827A093992761
:10DB2000B0939A2780911E2D90911F2DA091202DAA
:10DB3000B091212D8093932790939427A0939527BC
:10DB4000B0939627E8C310928A1780E0C0E0D0E037
:10DB500022C0E82FF0E075E0EE0FFF1F7A95E1F7A5
:10DB6000E257F34D918D992321F480938A17EF01A9
:10DB700016C0973079F4209721F0228D9A8D921754
:10DB800048F4C82FD0E065E0CC0FDD1F6A95E1F7BF
:10DB9000C257D34D8F5F8430E0F280938A1720976D
:10DBA00009F4F7C3D0938D2CC0938C2C83E08A8F1B
:10DBB000888F1E8A84E08F8B1B8E80919D27909189
:10DBC0009E279D838C8380919B2790919C279F8388
:10DBD0008E838091932790919427A0919527B0915F
:10DBE000962788839983AA83BB8381E0898F80915C
:10DBF00084178C87809185178D87809186178E87F3
:10DC0000809187178F8781E090E0998B888B809136
:10DC1000A2278B878091A1278A878091A027898757
:10DC200080919F27888781E090E00E94BC68809166
:10DC3000A727282F30E0207F3070213531050CF4E4
:10DC400049C082958F7090E00597880F991F880FC3
:10DC5000991F50918B1740E034C0F901E957F84DF6
:10DC600050A5552329F440938A1710928B1732C080
:10DC7000513011F44F5F25C05230E1F461A564309A
:10DC8000C9F440938A1750938B1732A520E083A5DF
:10DC900090E0822B932B9093891780938817F4E060
:10DCA000893D9F0710F088ED94E09B8B8A8B9D8BBC
:10DCB0008C8B10C02957384DF90121A5222331F052
:10DCC000420F242F30E0281739073CF240938A177F
:10DCD00050938B1780E18093A8278091A8278260BA
:10DCE0008093A82782E08093AF2784E08093B027B9
:10DCF0008093B12788ED8093B2278CE290E09093D7
:10DD0000802780937F2780E6B3C2D0938D2CC09369
:10DD10008C2C1092872C8091A82790E082FF03C062
:10DD2000198E80E24EC22091A72722952F70220FD4
:10DD3000220F20938A17B701621B71099B0124519E
:10DD400030403093802720937F2750E04F705070F1
:10DD50004230510539F4AC014F73507042315105D6
:10DD600051F42AC04130510531F4AC014F73507069
:10DD70004230510509F12115310531F49C01237020
:10DD8000307021153105C1F030919F272885321759
:10DD900009F064C23091A0272985321709F05EC2CC
:10DDA0003091A1272A85321709F058C23091A22755
:10DDB0002B85321709F052C284FF4AC068897989DD
:10DDC0006115710509F444C0CE010C960E94846867
:10DDD0003091A327809183273817D1F52091A4276C
:10DDE000809184272817A1F59091A52780918527F8
:10DDF000981771F58091A62740918627841741F5E1
:10DE00003C872D879E878F878B8D8823D1F42E8921
:10DE1000888D9A8D891B922F969596959695891B3C
:10DE2000280F2E8B87FD81959F89392F3695369542
:10DE3000931B980F9F8B822F869586958695890FC9
:10DE4000888F81E08093872C888D8A8F198A188A21
:10DE5000298D30E0C9018F7090708430910509F4EC
:10DE6000B5C18530910564F482309105C9F18330E4
:10DE700091050CF0B9C08130910509F08AC211C03A
:10DE80008630910509F4E2C1863091050CF4BEC1DB
:10DE90008730910509F4E2C18830910509F079C213
:10DEA0008AC18091872C80FF14C083E0898F80E431
:10DEB0008093872C198A188A80917F2790918027D8
:10DEC000009709F410C122E42093872C0E94BC68BB
:10DED0000AC18091A8278F73823009F05AC2FACE06
:10DEE0008091872C80FF75C08091A8278F73823125
:10DEF00009F06FC08091A727282F30E0207F307075
:10DF0000213531050CF449C082958F7090E005975A
:10DF1000880F991F880F991F50918B1740E034C0CC
:10DF2000F901E957F84D50A5552329F440938A1774
:10DF300010928B1732C0513011F44F5F25C0523010
:10DF4000E1F461A56430C9F440938A1750938B17AC
:10DF500032A520E083A590E0822B932B9093891724
:10DF60008093881774E0893D970710F088ED94E05E
:10DF70009B8B8A8B9D8B8C8B10C02957384DF90158
:10DF800021A5222331F0420F242F30E02817390732
:10DF90003CF240938A1750938B1783E0898F8091CE
:10DFA0009F2788878091A02789878091A1278A87CA
:10DFB0008091A2278B8781E090E00E94BC6882E478
:10DFC0008093872C198A188A1092802710927F27B5
:10DFD0008AC080E28093872C0E948064E0918C2C20
:10DFE000F0918D2C118E45CD8091A82780FF2AC0FD
:10DFF00024FD28C088899989009709F0CAC18091B9
:10E000007F279091802701960E94BC682091872CE1
:10E01000822F80618093872C80917F279091802729
:10E02000009719F022612093872C0E94806481E080
:10E0300090E0998B888B88E0898F1B8E81E180939B
:10E04000A8270FC185FF1CC05091AD2740E08091EB
:10E05000AE2790E0842B952B40918A2C50918B2CED
:10E06000480F591F50938B2C40938A2C40917F2747
:10E0700050918027481B590B5093802740937F274E
:10E0800080917F2790918027009749F024FD07C059
:10E090002091872C22602093872C0E94BC6890914D
:10E0A000A92780E02091AA27820F911D90938917BC
:10E0B000809388172C893D892817390710F000971D
:10E0C00021F43093891720938817809188179091B5
:10E0D00089179B8B8A8B8091872C90E0837090703E
:10E0E000009709F456C11092232D1092222D0E9400
:10E0F00080648091872C85FF07C01092232D109299
:10E10000222D198E84E19BCF84FF0AC01092232D0B
:10E110001092222D81E090E0998B888B84E08CCF47
:10E120002091222D3091232D21153105E1F080FF22
:10E1300002C0198A188A88899989009781F48A8986
:10E140009B898217930720F49093232D8093222D8F
:10E150008091222D9091232D998B888B04C09093D0
:10E16000232D8093222D1B8E8091812790918227D1
:10E1700090938B2C80938A2C8091222D9091232D2B
:10E18000009759F088899989009739F0889690937B
:10E19000802780937F2788E10BC08091872C81FFA7
:10E1A000F8C088E290E09093802780937F2780E1F9
:10E1B0008093A8275CC08091872C80FFEAC0198ECD
:10E1C00080E18093872C0E948064E3C080917F2748
:10E1D00090918027009711F00E94BC689091A82729
:10E1E0008091872C90FF0BC080FF06C087E0898F4D
:10E1F0001A8E198A188A19C086E0898F16C080FF86
:10E200001EC085E0898F198A188AC3C080917F2734
:10E2100090918027009711F00E94BC688091A827F8
:10E2200080FF0DC087E0898F1A8E81E090E00E9408
:10E23000BC6880E18093872C0E9480640FC080912D
:10E240007F2790918027009749F4A3C08091872C65
:10E2500080FF9FC087E0898F1A8E9BC080E1F80104
:10E2600081A388E290E09093802780937F2780E5C8
:10E270008093A72788858093A32789858093A427E7
:10E280008A858093A5278B858093A6278C8580938C
:10E290009F278D858093A0278E858093A1278F85CA
:10E2A0008093A22786E0809390278C819D81909314
:10E2B0009C2780939B278E819F8190939E2780939C
:10E2C0009D2780911E2D90911F2DA091202DB09102
:10E2D000212D8093932790939427A0939527B09313
:10E2E000962788819981AA81BB81809397279093F3
:10E2F0009827A0939927B0939A27898D84FF05C00A
:10E300001092AA271092A92706C084E08093A9271B
:10E3100088ED8093AA2780E480938F2780917F27C0
:10E32000909180279093892780938A271092AE2717
:10E330001092AD271092AC271092AB270E94F16883
:10E34000809590959093AC278093AB2785E480933C
:10E3500087271092882710928E2710928D27809100
:10E360008C1790918D17019690938D1780938C1731
:10E3700090938B2780938C2710929227109291274D
:10E380000E94E068809590959093922780939127C2
:10E3900004C01092802710927F271092872CDF9163
:10E3A000CF911F910F91FF90EF900895382F292F53
:10E3B000C9010895382F292F40E050E076276727BC
:10E3C000762780E090E0CB0177276627262B372B36
:10E3D000482B592BB901CA010895AC01E09181275E
:10E3E000F0918227222733272E1B3F0B2957334DCD
:10E3F000621773070CF49B011216130664F4209342
:10E40000222D3093232D4E175F0729F0CF01BA013B
:10E41000A9010E94577D08950F93DF93CF93CDB745
:10E42000DEB760970FB6F894DEBF0FBECDBF0023F6
:10E4300009F459C029833A834B835C836D837E83BF
:10E440008F839887E0E2E01B29813A814B815C81D0
:10E450001E16BCF019861A861B861C868E2F9927DD
:10E4600087FD9095909581959F4F04C0220F331F93
:10E47000441F551F8A95D2F72D873E874F87588BAB
:10E480002AC0CA01B901002E04C0660F771F881F79
:10E49000991F0A94D2F769877A878B879C87DA015C
:10E4A000C90104C0B695A79597958795EA95D2F7C7
:10E4B0002D813E814F81588504C0220F331F441F98
:10E4C000551F0A95D2F7822B932BA42BB52B8D8742
:10E4D0009E87AF87B88B29853A854B855C856D858E
:10E4E0007E858F85988960960FB6F894DEBF0FBE43
:10E4F000CDBFCF91DF910F910895A0E1B0E0E3E8A7
:10E50000F2E70C94AA7A29833A834B835C836D8368
:10E510007E838F839887A986BA86CB86DC86ED8634
:10E52000FE860F87188B2D813E814F8158858D8502
:10E530009E85AF85B889281739074A075B07C8F059
:10E5400082179307A407B50790F029813A814B8180
:10E550005C8189859A85AB85BC85281739074A0770
:10E560005B0738F082179307A407B50720F482E011
:10E5700003C080E001C081E06096EAE00C94C67AB6
:10E580002F923F924F925F926F927F928F929F92C3
:10E59000AF92BF92CF92DF92EF92FF920F931F93B1
:10E5A000DF93CF93CDB7DEB763970FB6F894DEBF96
:10E5B0000FBECDBF6C017F876E87FC01178216826C
:10E5C000838181FD04C06FC34C855D8504C01E013D
:10E5D0000894211C311CF6019381EE85FF8593FD83
:10E5E000859193FF8191FF87EE87882309F457C3B4
:10E5F000853241F493FD859193FF8191FF87EE87EA
:10E60000853259F490E0B6014A8B5B8B0E94AA7D5B
:10E610004A895B895D874C87D7CF10E0FF2400E0F3
:10E620000032B0F48B3269F08C3228F4803251F031
:10E63000833271F40BC08D3239F0803349F40160BC
:10E640002CC00260046029C0086027C0006125C09A
:10E6500007FD2EC0282F20532A3098F406FF08C04B
:10E66000812F880F182F110F110F180F120F15C0BF
:10E670008F2D880FF82EFF0CFF0CF80EF20E0062A3
:10E680000CC08E3221F406FD0AC3006406C08C362D
:10E6900011F4006802C0883659F4EE85FF8593FDB9
:10E6A000859193FF8191FF87EE87882309F0B8CF8A
:10E6B000982F9554933018F40061805E06C0982F0F
:10E6C0009556933008F09BC10F7E06FF16E06FE36E
:10E6D000E62EE022853619F4F0E4EF2A07C08636EC
:10E6E00019F420E8E22A02C011111150E7FE06C019
:10E6F0001C3340F4912E939427E00BC0183030F473
:10E70000212F06C027E03CE3932E03C027E017E04B
:10E710009924CA0104969D878C87FA0160817181D2
:10E7200082819381A101092D0E94677C5C0169802F
:10E73000262D30E0398B288B60FE03C0388933FFEB
:10E7400006C0E1FC06C0E2FE06C000E205C00DE224
:10E7500003C00BE201C000E0888999898C70907039
:10E760000097C1F1002311F084E001C083E08F1510
:10E7700058F4F81AE3FC09C080E290E0B6010E9468
:10E78000AA7DFA94C9F701C0FF24002329F0802F45
:10E7900090E0B6010E94AA7D888983FD03C003EE44
:10E7A0001FE00EC00FED1FE00BC0A114B10409F073
:10E7B000805290E0B6010E94AA7D0F5F1F4F05C0F6
:10E7C000AE2CBB2490E1A922BB24F80184918823BC
:10E7D00061F762C2E7FE0EC09A0CF889F4FF04C02C
:10E7E0008A81813309F49A94191454F5292D29301A
:10E7F00050F52DC0E6FC2BC0812F90E08A159B05BB
:10E800004CF03CEFA3163FEFB30624F080E8E82A73
:10E8100001C01150112349F0E2E0F0E0EC0FFD1FC0
:10E82000E10FF11D80818033A1F3E7FE10C0912E2E
:10E830009394812F90E0A816B90644F41A1907C0E2
:10E840009924939404C098E0992E01C010E0E7FE4B
:10E8500007C01A141B043CF495012F5F3F4F05C0FD
:10E8600025E030E002C021E030E0002311F02F5F0E
:10E870003F4F112329F0812F90E00196280F391F77
:10E880008F2D90E02817390714F4F21A01C0FF24E5
:10E890004E2C5524C20189709070009749F406C02F
:10E8A00080E290E0B6010E94AA7DFA94FF20C1F7B1
:10E8B000002329F0802F90E0B6010E94AA7D43FC3E
:10E8C00009C006C080E390E0B6010E94AA7DFA94D8
:10E8D000FF20C1F7E7FE46C03501B7FE02C066243F
:10E8E000772425010894411C511C46185708420CF6
:10E8F000531CF501E919F1094F01812F90E0002720
:10E900001127081B190BFFEF6F16FFEF7F0629F485
:10E910008EE290E0B6010E94AA7DA614B70434F0FE
:10E92000861497041CF4F201808101C080E30894EE
:10E93000610871080894411C511C601671062CF086
:10E9400090E0B6010E94AA7DDECF6A147B0441F4F8
:10E950009A81963320F4953319F4F889F4FF81E312
:10E9600090E049C08A81813311F02FEE622290E05D
:10E97000B6010E94AA7D112389F08EE290E0B601D3
:10E980000E94AA7D02E0F101E00FF11D0F5F80817E
:10E9900090E0B6010E94AA7D1150A9F744FE03C081
:10E9A00085E490E002C085E690E0B6010E94AA7D71
:10E9B000B7FC05C0A114B10441F464FE06C0B094D4
:10E9C000A194B108B3948DE201C08BE290E0B6014E
:10E9D0000E94AA7D80E305C08F5FE6EFFFEFAE0ED9
:10E9E000BF1EFAE0AF16B104BCF790E0B6010E947A
:10E9F000AA7DC501C096B6010E94AA7D4DC183368D
:10EA000031F0833789F0833509F059C022C09A016B
:10EA10002E5F3F4F3D872C87FA018081898331012A
:10EA200081E0A82EB12C13C09A012E5F3F4F3D8785
:10EA30002C87FA016080718006FF03C0612F70E0AF
:10EA400002C06FEF7FEFC3010E94707D5C010F7702
:10EA500014C09A012E5F3F4F3D872C87FA016080DA
:10EA6000718006FF03C0612F70E002C06FEF7FEF7F
:10EA7000C3010E94477D5C01006803FD1CC006C005
:10EA800080E290E0B6010E94AA7DFA948F2D90E07A
:10EA9000A816B906A8F30FC0F30107FD859107FF7B
:10EAA00081913F0190E0B6010E94AA7DF110FA9495
:10EAB0000894A108B108A114B10471F7EDC084361F
:10EAC00011F0893661F507FF0BC09A012C5F3F4FAB
:10EAD0003D872C87FA0160817181828193810CC00E
:10EAE0009A012E5F3F4F3D872C87FA01608171812B
:10EAF000882777FD8095982F0F7697FF08C090950F
:10EB00008095709561957F4F8F4F9F4F0068A10151
:10EB10002AE030E00E94BC7E982E921841C08537D2
:10EB200021F40F7E2AE030E020C0097F8F36A9F063
:10EB3000803720F4883509F0B2C00BC0803721F04F
:10EB4000883709F0ACC001C0006104FF09C004604F
:10EB500007C004FF08C0066006C028E030E005C01A
:10EB600020E130E002C020E132E007FF0AC0CA0124
:10EB700004969D878C87FA016081718182819381DF
:10EB800009C0CA0102969D878C87FA016081718154
:10EB900080E090E0A1010E94BC7E982E92180F7731
:10EBA00006FF09C00E7F911630F404FF06C002FD77
:10EBB00004C00F7E02C0E92C01C0E12E802F90E03E
:10EBC00004FF0CC0FE01E90DF11D2081203311F47A
:10EBD000097E09C0E39402FF06C004C086789070E5
:10EBE000009709F0E394A02EBB2403FD14C000FF9E
:10EBF0000FC0EF1428F4192D1F0D1E19EF2C08C09B
:10EC0000192D06C080E290E0B6010E94AA7DE3942F
:10EC1000EF14C0F304C0EF1410F4FE1801C0FF2479
:10EC2000A4FE0FC080E390E0B6010E94AA7DA2FE80
:10EC30001FC0A1FE03C088E590E010C088E790E007
:10EC40000DC0C50186789070009791F0A1FC02C0BC
:10EC500080E201C08BE207FD8DE290E0B6010E94E8
:10EC6000AA7D06C080E390E0B6010E94AA7D115003
:10EC70009116C0F39A94F101E90DF11D808190E0A5
:10EC8000B6010E94AA7D9920A9F706C080E290E013
:10EC9000B6010E94AA7DFA94FF20C1F795CCF60137
:10ECA0002681378102C02FEF3FEFC90163960FB66F
:10ECB000F894DEBF0FBECDBFCF91DF911F910F91B2
:10ECC000FF90EF90DF90CF90BF90AF909F908F908C
:10ECD0007F906F905F904F903F902F900895505885
:10ECE000BB27AA270ED0CBC1BCD130F0C1D120F0B8
:10ECF00031F49F3F11F41EF48CC10EF4E095E7FB54
:10ED000082C1E92FCDD180F3BA1762077307840758
:10ED1000950718F071F49EF5E5C10EF4E0950B2E01
:10ED2000BA2FA02D0B01B90190010C01CA01A0015D
:10ED30001124FF27591B99F0593F50F4503E68F1B8
:10ED40001A16F040A22F232F342F4427585FF3CFF9
:10ED5000469537952795A795F0405395C9F77EF4CA
:10ED60001F16BA0B620B730B840BBAF09150A1F013
:10ED7000FF0FBB1F661F771F881FC2F70EC0BA0F99
:10ED8000621F731F841F48F4879577956795B79521
:10ED9000F7959E3F08F0B3CF9395880F08F0992719
:10EDA000EE0F9795879508955CD158F080E891E033
:10EDB00009F49EEF5DD128F040E851E059F45EEF90
:10EDC00009C027C18FC1E92FE0786AD168F3092E05
:10EDD000052AC1F3261737074807590738F00E2EC2
:10EDE00007F8E02569F0E025E0640AC0EF6307F862
:10EDF000009407FADB01B9019D01DC01CA01AD01F4
:10EE0000EF9347D03CD10AD05F91552331F02BEDE1
:10EE10003FE049E450FD49EC63CF0895DF93DD27DF
:10EE2000B92FBF7740E85FE31616170648075B0760
:10EE300010F4D92F5ED19F938F937F936F930FD24E
:10EE4000E0E2F1E0E9D01BD12F913F914F915F912A
:10EE500063D1DD2349F09058A2EA2AED3FE049EC66
:10EE60005FE3D0785D274DDFDF9109C1A8D008F4BA
:10EE700081E008950CD003C1FBD040F0F2D030F017
:10EE800021F45F3F19F0BFC051112DC1C2C008D19C
:10EE900098F39923C9F35523B1F3951B550BBB2761
:10EEA000AA2762177307840738F09F5F5F4F220F0E
:10EEB000331F441FAA1FA9F333D00E2E3AF0E0E807
:10EEC00030D091505040E695001CCAF729D0FE2F53
:10EED00027D0660F771F881FBB1F261737074807E5
:10EEE000AB07B0E809F0BB0B802DBF01FF2793589B
:10EEF0005F4F2AF09E3F510568F085C0F4C05F3F28
:10EF0000ECF3983EDCF3869577956795B795F79582
:10EF10009F5FC9F7880F911D9695879597F908957A
:10EF2000E1E0660F771F881FBB1F62177307840716
:10EF3000BA0720F0621B730B840BBA0BEE1F88F725
:10EF4000E0950895E89409C097FB3EF4909580956C
:10EF5000709561957F4F8F4F9F4F9923A9F0F92F9F
:10EF600096E9BB279395F695879577956795B7951D
:10EF7000F111F8CFFAF4BB0F11F460FF1BC06F5F03
:10EF80007F4F8F4F9F4F16C0882311F096E911C015
:10EF9000772321F09EE8872F762F05C0662371F036
:10EFA00096E8862F70E060E02AF09A95660F771F4A
:10EFB000881FDAF7880F9695879597F90895990F26
:10EFC0000008550FAA0BE0E8FEEF16161706E80733
:10EFD000F907C0F012161306E407F50798F0621B54
:10EFE000730B840B950B39F40A2661F0232B242B29
:10EFF000252B21F408950A2609F4A140A6958FEF48
:10F00000811D811D089597F99F6780E870E060E099
:10F0100008959FEF80EC0895DF93CF931F930F9394
:10F02000FF92EF92DF927B018C01689405C0DA2E8B
:10F03000EF0172D0FE01E894A5912591359145919B
:10F040005591AEF3EF015DDEFE019701A801DA9460
:10F0500079F7DF90EF90FF900F911F91CF91DF91A3
:10F06000089500240A94161617061806090608952E
:10F0700000240A9412161306140605060895092E94
:10F080000394000C11F4882352F0BB0F40F4BF2B03
:10F0900011F460FF04C06F5F7F4F8F4F9F4F089543
:10F0A00057FD9058440F551F59F05F3F71F0479539
:10F0B000880F97FB991F61F09F3F79F0879508951E
:10F0C000121613061406551FF2CF4695F1DF08C03D
:10F0D000161617061806991FF1CF8695710561055A
:10F0E00008940895E894BB2766277727CB0197F902
:10F0F00008959B01AC0160E070E080E89FE3BACE28
:10F100000BD0BDCFAEDF28F0B3DF18F0952309F0A8
:10F110007ACF7FCF1124E7CFC3DFA0F3959FD1F340
:10F12000950F50E0551F629FF001729FBB27F00DB5
:10F13000B11D639FAA27F00DB11DAA1F649F66270A
:10F14000B00DA11D661F829F2227B00DA11D621F59
:10F15000739FB00DA11D621F839FA00D611D221F13
:10F16000749F3327A00D611D231F849F600D211DF7
:10F17000822F762F6A2F11249F5750408AF0E1F09A
:10F1800088234AF0EE0FFF1FBB1F661F771F881FE3
:10F1900091505040A9F79E3F510570F034CFA3CF56
:10F1A0005F3FECF3983EDCF3869577956795B795CE
:10F1B000F795E7959F5FC1F7FE2B880F911D9695F8
:10F1C000879597F90895FA01EE0FFF1F30962105F4
:10F1D000310599F16115710561F48038BFE39B0732
:10F1E00049F168949038810561F08038BFEF9B0742
:10F1F00041F0992342F5FF3FE1053105210511F169
:10F20000E8940894E795D901AA2329F4AB2FBE2FDF
:10F21000F85FD0F310C0FF5F70F4A695E0F7F73900
:10F2200050F019F0FF3A38F49F779F930CD00F906D
:10F2300007FC905808953EF0ECCE60E070E080E866
:10F240009FE308954FE79F775F934F933F932F93EB
:10F2500075D02F913F914F915F9152DF08C09B0174
:10F26000AC014ECF19F40EF0CECE3CCFD2CE20DF83
:10F27000C8F39638C0F707F80F92E8942BE33AEA00
:10F2800048EB5FE74BDF0F920F920F924DB75EB7DF
:10F290000F9294D0EDE4F1E0BFDE4F915F91EF91DA
:10F2A000FF91E595EE1FFF1F49F0FE57E0684427E8
:10F2B000EE0F441FFA95E1F74195550B06D00F90DC
:10F2C00007FE17CF08959FCEACC0F2DEE8F3992376
:10F2D000D9F3940F511DBBF39150504094F059F065
:10F2E000882332F0660F771F881F91505040C1F776
:10F2F0009E3F510544F7880F911D9695879597F984
:10F3000008955F3FACF0983E9CF0BB2786957795BB
:10F310006795B79508F4B1609395C1F7BB0F58F79F
:10F3200011F460FFE8CF6F5F7F4F8F4F9F4FE3CFA8
:10F33000DACE0EF076C06DCE689465CEB9DEC8F335
:10F340009923D1F3C6F3DF93CF931F930F93FF92CB
:10F35000C92FDD2788232AF02197660F771F881F82
:10F36000DAF720E030E040E85FEB9FE3883920F0F7
:10F37000803E30F021968F77B3DCE5E7F1E003C003
:10F38000AFDCE2EAF1E048DE8B01BE01EC01FB2ECE
:10F390006F5771097595771F880B990BD5DD28E19B
:10F3A00032E741E35FE3B8DEAF2D9801AE01FF9095
:10F3B0000F911F91CF91DF91A4DC61CEFA01DC01A6
:10F3C000AA0FBB1F9B01AC01BF5728F4222733278C
:10F3D000442750781FC0B75188F4AB2F00244695BE
:10F3E00037952795011CA395D2F3002069F0220FD1
:10F3F000331F441FB395DAF30DD071CC6130710522
:10F40000A0E88A07B94630F49B01AC01662777274C
:10F4100088279078309621F020833183428353836C
:10F4200008959F3F31F0915020F487957795679527
:10F43000B795880F911D9695879597F90895629FC6
:10F44000D001739FF001829FE00DF11D649FE00DDC
:10F45000F11D929FF00D839FF00D749FF00D659F3D
:10F46000F00D9927729FB00DE11DF91F639FB00D3C
:10F47000E11DF91FBD01CF0111240895AA1BBB1B7B
:10F4800051E107C0AA1FBB1FA617B70710F0A61BA4
:10F49000B70B881F991F5A95A9F780959095BC01C5
:10F4A000CD01089597FB092E07260AD077FD04D0D9
:10F4B000E5DF06D000201AF4709561957F4F08951E
:10F4C000F6F7909581959F4F0895A1E21A2EAA1BF9
:10F4D000BB1BFD010DC0AA1FBB1FEE1FFF1FA21704
:10F4E000B307E407F50720F0A21BB30BE40BF50B01
:10F4F000661F771F881F991F1A9469F7609570958A
:10F50000809590959B01AC01BD01CF01089597FBBB
:10F51000092E05260ED057FD04D0D7DF0AD0001CD7
:10F5200038F450954095309521953F4F4F4F5F4FA0
:10F530000895F6F790958095709561957F4F8F4F60
:10F540009F4F08952F923F924F925F926F927F92BA
:10F550008F929F92AF92BF92CF92DF92EF92FF92E3
:10F560000F931F93CF93DF93CDB7DEB7CA1BDB0B8F
:10F570000FB6F894DEBF0FBECDBF09942A88398834
:10F5800048885F846E847D848C849B84AA84B9843B
:10F59000C884DF80EE80FD800C811B81AA81B98147
:10F5A000CE0FD11D0FB6F894DEBF0FBECDBFED015B
:10F5B0000895AF92BF92CF92DF92EF92FF920F9396
:10F5C0001F93CF93DF93EC01688179818A819B81BE
:10F5D000611571058105910521F464E279ED8BE5F2
:10F5E00097E02DE133EF41E050E00E94877A790106
:10F5F0008A0127EA31E440E050E00E941F7A5B0173
:10F600006C01C801B7012CEE34EF4FEF5FEF0E94A1
:10F610001F7A6A0D7B1D8C1D9D1D97FF04C06150D4
:10F62000704080409048688379838A839B837F778A
:10F63000CB01DF91CF911F910F91FF90EF90DF9061
:10F64000CF90BF90AF9008950E94D97A089580EE30
:10F6500096E00E94D97A0895A0E0B0E08093E00699
:10F660009093E106A093E206B093E30608952F92EB
:10F670003F924F925F926F927F929F92AF92BF9212
:10F68000CF92DF92EF92FF920F931F93CF93DF936E
:10F690003B01EA016115710519F0FB01808391833B
:10F6A000209739F09E01225030402332310508F076
:10F6B000D5C0C82ED92EF60111916F017F01812F7F
:10F6C00090E00E943F7D0097B1F71D3231F4F601C2
:10F6D00011917F019924939406C01B3219F4F6010D
:10F6E00011917F019924209719F0C031D105D1F4EF
:10F6F000103389F4F7018081883711F0883559F487
:10F70000F701118182E090E0E80EF91E92E0992A5B
:10F71000C0E1D0E007C0209729F41033B1F0CAE06F
:10F72000D0E02BC0CA30D10541F1C031D10521F064
:10F73000C830D105A9F409C02FEFA22E2FEFB22EA9
:10F740002FEFC22E2FE0D22E20C0C8E0D0E09FEFD6
:10F75000A92E9FEFB92E9FEFC92E9FE1D92E15C07C
:10F760009E01442737FD4095542F6FEF7FEFCB016B
:10F770000E94657A59016A0108C089E9A82E89E9C1
:10F78000B82E89E9C82E89E1D82E60E020E030E06B
:10F79000A9011E01442437FC4094542C012F00532E
:10F7A0000A3060F0812F81548A3110F4075006C06E
:10F7B000812F81568A3150F5012F0755802F90E017
:10F7C0008C179D071CF56F3FE9F0A216B306C4061F
:10F7D000D506A8F0CA01B901A20191010E941F7AC1
:10F7E0009B01AC01802F90E0A0E0B0E0280F391F12
:10F7F0004A1F5B1F281739074A075B0710F46FEF92
:10F8000001C061E0F70111917F01C8CF611471045B
:10F8100081F0662339F00894E108F108F301F182E0
:10F82000E08207C091FE05C0C7010297F3019183F2
:10F83000808390FE07C050954095309521953F4FAD
:10F840004F4F5F4F67FF0DC082E290E09093AD2D68
:10F850008093AC2D2FEF3FEFA90103C020E030E0F3
:10F86000A901B901CA01DF91CF911F910F91FF90BA
:10F87000EF90DF90CF90BF90AF909F907F906F9070
:10F880005F904F903F902F900895662777270C94B4
:10F89000557FFC0188279927E89421912032E9F3CC
:10F8A000293010F02E30C8F32B3241F02D3239F4CC
:10F8B000689404C00E94A27D820F911D2191205363
:10F8C0002A30C0F31EF4909581959F4F08952830FB
:10F8D00008F027E03327DA01990F311D87FD916089
:10F8E00000966105710539F432602E5F3D9330E377
:10F8F0002A95E1F708959F3F30F080387105610542
:10F9000009F03C5F3C5F3D93913008F08068911DA9
:10F91000DF93CF931F930F93FF92EF92192F987F4E
:10F920009695E92F96959695E90FFF27EF5BFF4E89
:10F9300099273327EE24FF24A701E70105900894B7
:10F94000079428F4360FE71EF81E491F511D660F55
:10F95000771F881F991F0694A1F70590079428F434
:10F96000E70EF81E491F561FC11D770F881F991FEC
:10F97000661F0694A1F70590079428F4F80E491F16
:10F98000561FC71FD11D880F991F661F771F06942A
:10F99000A1F70590079420F4490F561FC71FD81FE1
:10F9A000990F661F771F881F0694A9F784911095F9
:10F9B000177041F0D695C79557954795F794E794FA
:10F9C0001A95C1F7E7EEFFE068941590159135910F
:10F9D0006591959105907FE27395E118F10A430BCB
:10F9E000560BC90BD009C0F7E10CF11E431F561F7F
:10F9F000C91FD01D7EF4703311F48A95E6CFE894C8
:10FA0000015030F0080F0AF40027021708F4202FE5
:10FA10002395022F7A3328F079E37D932A95E9F72D
:10FA200010C07D932A9589F606949795679537952A
:10FA300017951794E118F10A430B560BC90BD0091F
:10FA400098F023957E9173957A3308F070E37C9358
:10FA50002013B8F77E9170617D9330F0839571E348
:10FA60007D9370E32A95E1F71124EF90FF900F91B9
:10FA70001F91CF91DF91992787FD9095089591115E
:10FA8000A2C3803219F089508550D0F70895FC0147
:10FA90000590615070400110D8F7809590958E0FB9
:10FAA0009F1F089540E957E10E947B7D0895FB0167
:10FAB000DC0102C001900D9241505040D8F70895EA
:10FAC000DC0101C06D9341505040E0F70895FB0107
:10FAD000DC018D91019080190110D9F3990B0895E3
:10FAE000FC016150704001900110D8F7809590950D
:10FAF0008E0F9F1F0895FA01A191B081009719F40C
:10FB00001097E1F0CD01DC01CD010D90002011F442
:10FB1000C00113C0FB012191222319F02015D9F750
:10FB2000F3CFFB012191201519F41E92119606C006
:10FB30002223C1F70D900020A1F7D001FA01A19373
:10FB4000B08308957AE0979F902D879F802D910D27
:10FB5000112408950F931F93CF93DF938C01EB0132
:10FB60008B8181FF1BC082FF0DC02E813F818C8164
:10FB70009D812817390764F4E881F9810193F9839D
:10FB8000E88306C0E885F985802F0995009731F450
:10FB90008E819F8101969F838E8302C00FEF1FEF9E
:10FBA000C801DF91CF911F910F910895DF93CF93FB
:10FBB000CDB7DEB7FE013596619171918091A82D88
:10FBC0009091A92DAF010E94C072CF91DF9108954D
:10FBD000DF93CF93CDB7DEB7FE013596619171917A
:10FBE0008091A82D9091A92DDC0113962C9113974B
:10FBF000286013962C93AF010E94C072E091A82D4B
:10FC0000F091A92D2381277F2383CF91DF91089540
:10FC10006091A82D7091A92D0E94AA7D0895EF9260
:10FC2000FF920F931F93CF93DF938C01E091A82D48
:10FC3000F091A92D838181FF1FC0C0E0D0E00AC0F0
:10FC4000DB011896ED91FC9119970995009711F039
:10FC5000CFEFDFEFF80181918F016091A82D7091B6
:10FC6000A92D882369F7DB011896ED91FC9119976E
:10FC70008AE00995009711F0CFEFDFEFCE01DF9119
:10FC8000CF911F910F91FF90EF9008950F931F93C5
:10FC9000DF93CF93CDB7DEB72E970FB6F894DEBFC4
:10FCA0000FBECDBF0D891E898F89988D26E02C83CC
:10FCB0001A83098397FF02C080E090E801979E8332
:10FCC0008D839E01255E3F4FCE010196698D7A8D11
:10FCD000A9010E94C0724D815E8157FD0AC02F812B
:10FCE0003885421753070CF49A01020F131FF801CD
:10FCF00010822E960FB6F894DEBF0FBECDBFCF9107
:10FD0000DF911F910F9108950F931F93DF93CF936E
:10FD1000CDB7DEB72E970FB6F894DEBF0FBECDBFBE
:10FD20008C01CB01BA0146E04C831A83098397FF0B
:10FD300002C080E090E801979E838D83CE010196FA
:10FD4000A9010E94C0724D815E8157FD0AC02F81BA
:10FD50003885421753070CF49A01020F131FF8015C
:10FD600010822E960FB6F894DEBF0FBECDBFCF9196
:10FD7000DF911F910F910895FA01AA27283051F1C0
:10FD8000203181F1E8946F936E7F6E5F7F4F8F4FCC
:10FD90009F4FAF4FB1E03ED0B4E03CD0670F781F2B
:10FDA000891F9A1FA11D680F791F8A1F911DA11D10
:10FDB0006A0F711D811D911DA11D20D009F4689449
:10FDC0003F912AE0269F11243019305D3193DEF6F1
:10FDD000CF010895462F4770405D4193B3E00FD0A7
:10FDE000C9F7F6CF462F4F70405D4A3318F0495D92
:10FDF00031FD4052419302D0A9F7EACFB4E0A69575
:10FE00009795879577956795BA95C9F70097610596
:10FE1000710508959B01AC010A2E069457954795EC
:10FE200037952795BA95C9F7620F731F841F951FE1
:10FE3000A01D0895DC01CB01FC01F999FECF06C09D
:10FE4000F2BDE1BDF89A319600B40D924150504098
:10FE5000B8F70895F999FECF92BD81BDF89A992718
:10FE600080B50895A8E1B0E042E050E00C941C7F1A
:10FE7000DC01CB0103C02D910E94437F41505040D3
:10FE8000D0F70895262FF999FECF1FBA92BD81BDF4
:10FE900020BD0FB6F894FA9AF99A0FBE019608950C
:10FEA0000E94427F272F0C94437F6F927F928F9204
:10FEB0009F92AF92BF92CF92DF92EF92FF920F93F9
:10FEC0001F93DF93CF930F92CDB7DEB75B01611520
:10FED000710521F0DB018C9311969C93482F592FCB
:10FEE0006A01F601E1906F018F018E2D90E00E9472
:10FEF0003F7D0097B1F7FE2DFD3229F4D601ED903C
:10FF00008D0121E007C0BE2DBB3219F4F601E1904E
:10FF10008F0120E068010894C108D108C60161EE94
:10FF200070E143E050E029830E94E6802981009738
:10FF300011F572E0E72EF12CE00EF11EC70164EE20
:10FF400070E145E050E00E94E6802981009729F4A5
:10FF500067E0E62EF12CE00EF11EA114B10421F0B1
:10FF6000D5011196FC92EE9220FF0FC130E020E007
:10FF700090E88FEF12C1C60169EE70E143E050E0F6
:10FF800029830E94E6802981009731F060E070E0CB
:10FF9000CB01662477240AC0A114B10409F4F9C086
:10FFA0000E5F1F4FF50111830083F3C03E2D3053C8
:10FFB0003A30A0F52260E22FF0E0AF0148705070B7
:10FFC00022FF07C04115510571F50894611C711C91
:10FFD0002AC04115510519F00894610871086B0198
:10FFE0007C0152E0CC0CDD1CEE1CFF1C5A95D1F7B5
:10FFF0006C0D7D1D8E1D9F1D660F771F881F991F1D
:020000021000EC
:10000000630F711D811D911D6839F9E97F07F9E9B9
:100010008F07F9E19F0738F0246005C03E3F39F4AF
:1000200023FD3FC02860D801ED908D01BFCF35334F
:1000300011F03531B1F5F80131913D3211F4206103
:1000400002C03B3241F4D80111963C911197319690
:1000500042E050E002C041E050E030533A3020F03E
:100060008F01041B150B1DC040E050E0BCE0403880
:100070005B075CF4DA01AA0FBB1FAA0FBB1F4A0F74
:100080005B1F440F551F430F511D319130538F019A
:100090003A3060F324FF03C0509541955F4F640EE2
:1000A000751EC22EDD2421FF08C0A114B10429F061
:1000B00001501040F501118300830E94A2777B015B
:1000C0008C01F3E0CF22DD2433E0C316D10421F408
:1000D00017FB109517F91095C801B70120E030E023
:1000E000A9010E943677882309F44AC077FE09C027
:1000F00040E0C42E41E1D42E709461947108739451
:1001000004C038E1C32E31E1D32E26E0822E912C9B
:1001100090E2A92EB12C0FC0F601259135914591A1
:100120005491C801B7010E948078E62EF72E082F5F
:10013000192F6A187B086A147B0474F7B594A79486
:100140000894810891088114910429F08CEF9FEFA5
:10015000C80ED91EF0CFB701C801282F220F292FB2
:10016000221F2F3F39F020E030E0A9010E943677AE
:10017000882331F482E290E09093AD2D8093AC2DF2
:100180003E2D2F2D902F812F08C030E020E090E8E9
:1001900003C030E020E090EC8FE7F901AC016F2F55
:1001A000722F852F942F0F90CF91DF911F910F9178
:1001B000FF90EF90DF90CF90BF90AF909F908F9087
:1001C0007F906F900895992788270895FB01DC019F
:1001D0004150504088F08D9181341CF08B350CF4E7
:1001E000805E659161341CF06B350CF4605E861B9B
:1001F000611171F3990B0895881BFCCFF894FFCF20
:10020000263A202573205B414444523D252D642E1F
:10021000252D64205345513D252D642052535349CB
:100220003D252D75204C51493D252D7520445250BA
:100230003D252D642E253032645D0A00523D252D6A
:1002400075204C3D252D7520533D252D64200054EF
:10025000696D656F757420414444523D252D642EAF
:10026000252D64205345513D252D6420525353497B
:100270003D252D75204C51493D252D750A002845F9
:10028000787450777229000065756936343D002511
:1002900030327800253032780A00736E3D00413AE2
:1002A000202564202564202564200A00433A202567
:1002B0006420256420256420613D25352E31660AA1
:1002C000007374617475733D3078253032780A207C
:1002D00000312E30204669726D7761726520566557
:1002E000722E2053322D342E3020323031332D30C7
:1002F000362D303900656570726F6D006F6E006F5E
:10030000666600666F7263655F69646C650064654C
:100310006570004F6E006131007265736574006E28
:100320006F6E6500613200765F696E0031003200E9
:100330003300340035003600636820706B7473003E
:1003400025327520252D3130750A006175746F00D6
:10035000666C75736800414444523D252D642E251A
:100360002D64205345513D252D6420525353493D62
:10037000252D75204C51493D252D750A0070777249
:10038000733D25730A007472696D0074657374009F
:1003900043683D252D642054785077723D252D64A7
:1003A0000A004572726F72205458204C656E677453
:1003B000683D25640A0049443D004536343D00202F
:1003C00050533D25640020543D252D362E326600C5
:1003D0002054313D252D362E32660020545F4D438A
:1003E000553D252D352E31660020565F4D43553D38
:1003F000252D342E3266002050303D252D6C5800BE
:100400002050305F543D252D372E3366002050316B
:100410003D252D6C58002050315F543D252D372E41
:100420003366002055503D252D6C58002052483D24
:10043000252D342E31660020565F494E3D252D3541
:100440002E32660020565F41313D252D352E326615
:100450000020565F41323D252D352E326600205654
:100460005F41333D252D352E30660020503D252D32
:100470006C64002050413D252D372E326600263A0F
:100480002025730A00545820706B74206C656E2010
:100490003D2025640A0025303258006C656E3D25EC
:1004A000640A000100D734EF3C22FFCC3B22FFCC92
:1004B0003B1A20090D00B2046162636465666768D7
:1004C000696A6B6C6D6E6F70269400003C000A00C8
:1004D0001A636D642070726F63657373000000D1DE
:1004E000044F3500000000737464696E2070726FF1
:1004F00063657373000000E704550F00000000629D
:10050000726F6164636173742070726F636573737B
:10051000000000FF042F3600000000536C6565707A
:100520002070726F636573730000001B0545100037
:10053000000000506572696F6469632070726F63B8
:100540006573730000003305411700000000DD04EF
:10055000F5041105440529050000D10800001D001F
:1005600040001A075A0710000000A33E973E1810DB
:10057000000000004576656E742074696D65720038
:1005800000007405AE42000000004374696D65729E
:100590002070726F636573730000008A05EC43007E
:1005A000000000020306070A0B0E0F020306070AEB
:1005B0000B0E0F2843292032303132204865726AF1
:1005C000756C660055747665636B6C696E67202088
:1005D0002020202000436F6E74696B6920322E3515
:1005E000000000000200000000275200000000C6CA
:1005F00000C500C400C100C200000000CE00CD0054
:10060000CC00C900CA0000000052463233302064DA
:1006100072697665720000000906DE56000000006F
:100620004F55CD542D577758F0558054EE52E8521F
:100630006F54D153000101010101010101010101C8
:10064000010101010052696D65004506F259B95971
:1006500061646174612E6E756D20776179206F75AC
:10066000742074686572653A2025640A00345B332F
:100670005B3D5D6C5EA45C0080C0E0F0F8FCFEFFBA
:100680006E756C6C6D61630080061F5F045F0A5FAE
:10069000105F165F1C5F736963736C6F776D6163C6
:1006A0000096064060A15F375F205F265F345FBA27
:1006B0000008001911211135000200F116F316543B
:1006C00043502F495020737461636B000000BF06D4
:1006D0009A62000000000208FFFFFFFF0000000018
:0406E0000100000015
:00000001FF
